:100000000C940C0A0C942B0A0C942B0A0C94E70BFE
:100010000C94210C0C942B0A0C942B0A0C942B0A94
:100020000C942B0A0C942B0A0C942B0A0C942B0A7C
:100030000C942B0A0C942B0A0C942B0A0C943B0F57
:100040000C942B0A0C942B0A0C942B0A0C942B0A5C
:100050000C948A740C94386C0C942B0A0C942B0A14
:100060000C942B0A0C940B6D0C942B0A0C94FF6CC3
:100070000C942B0A0C942B0A0C942B0A0C942B0A2C
:100080000C94BB7F0C942B0A0C942B0A0C942B0A17
:100090000C94496D0C942B0A0C943D6D0C942B0A16
:1000A0000C942B0A0C942B0A0C942B0A0C942B0AFC
:1000B0000C942B0A0C942B0A0C942B0A0C942B0AEC
:1000C0000C942B0A0C942B0A0C942B0A0C942B0ADC
:1000D0000C942B0A0C942B0A0C942B0A0C942B0ACC
:1000E0000C942B0A0C9443740C944D740C94397436
:1000F0000C94F9730C947E740C946F740C94637468
:100100000C9457740C942B0A0C942B0A0C942B0A05
:100110000C942B0A0C942B0A0C942B0A0C942B0A8B
:10012000F0880F8989897B8A9B8ABB8AC38A708AF7
:10013000084AD73B3BCE016E84BCBFFDC12F3D6C4E
:1001400074319ABD56833DDA3D00C77F11BED9E4B4
:10015000BB4C3E916BAAAABE000000803F076342E1
:1001600036B79BD8A71A39685618AEBAAB558C1D4E
:100170003CB7CC5763BD6DEDFD753EF6177231BFD0
:10018000000000803F08000000BE922449123EABF0
:10019000AAAA2ABECDCCCC4C3E00000080BEABAAA1
:1001A000AAAA3E00000000BF000000803F0000003F
:1001B0000000084178D3BB4387D1133D190E3CC3DF
:1001C000BD4282AD2B3E68EC8276BED98FE1A93E5E
:1001D0004C80EFFFBE01C4FF7F3F00000000000025
:1001E00025630025630025730A005854414C5F5471
:1001F00052494D3D25640025730A0025730A0054B9
:1002000065737420362025730A0054657374203595
:100210002025730A005465737420342025730A0066
:100220005465737420332025730A00546573742059
:10023000322025730A005465737420312025730A17
:10024000006368616E3D25640A0074787077723DC2
:1002500025640A003530306B0A003235306B0A00F5
:100260003131356B0A0035366B0A0033386B0A00C2
:1002700025730A00765F6C6F773D252D332E32662D
:100280000A0025730A0073656E743D252D75206480
:1002900075703D252D752069676E6F7265643D250B
:1002A0002D752074746C5F7A65726F3D252D750A0B
:1002B0000025372E33662025372E33660025352E50
:1002C000326620004572726F72203020566F6C7457
:1002D000004E6F7420737570706F727465640A00DD
:1002E0004572726F72203020566F6C7400457272C6
:1002F0006F72203020566F6C740062756C6B5F6497
:10030000656C61793D252D750062756C6B3D252D01
:10031000750056616C7565206E6F7420616C6C6F32
:100320007765640062756C6B3A206D61783D257568
:100330002073746172743D25752C20656E643D25B3
:10034000752C20696E5F7573653D25750A007062B6
:10035000323D25730A007062313D25730A00256C19
:100360007500416C6C6F77656420737065656420FF
:10037000312F31302F3130302F343030206B6269E3
:10038000742F730025630074746C3D252D64200068
:1003900074746C3D252D6420004E65772074746C58
:1003A0003D252D6420002563004D53353631312025
:1003B000503D252D372E326620252D372E32666D85
:1003C0000A00424D5030383520256C6420506120A1
:1003D00020252D372E32666D00256300545F484579
:1003E00041545F4944583D252D352E326620005436
:1003F0005F4445573D252D352E3266200041483D4E
:10040000252D352E32662000545F53485432583D16
:10041000252D352E3266200052485F5348543258FD
:100420003D252D352E32662000545F52483D252D46
:10043000342E3166200052483D252D342E31662061
:100440000025630025630025630025630025630004
:100450007265706F72745F616C6C3D007265706F75
:1004600072743D0025630025630025630025630049
:10047000204F534343414C3D256420002046757373
:10048000653A2065653D253032782068663D253027
:100490003278206C663D25303278206C623D253004
:1004A0003278004D43553D2530366C780025630089
:1004B00074785F6C656E3D252D6C752C765F6C6F66
:1004C000773D252D6C752C73687432783D252D6C25
:1004D000752C62756C6B3D252D6C75002563004F86
:1004E0004B0A002563002563002563002563002572
:1004F00063002563002563002563006465627567FA
:100500005F616C6C3D0064656275673D00646562A7
:1005100075673D0025730A00646565700A006E6F9B
:100520006E650A00707772733D007062323D25730C
:100530000A007062313D25730A00696E74725F7340
:1005400065635F70313D252D372E33660A00696E75
:1005500074725F70313D252D6C640A00696E74728F
:100560005F7365635F70303D252D372E33660A005B
:10057000696E74725F70303D252D6C640A00765F81
:100580006D63753D252D352E32660A00745F6D63EF
:10059000753D252D352E32660A00707077723D2527
:1005A000730A0064656275673D0072636D643D2582
:1005B000730A0025730A006175746F0A006C6F6717
:1005C0005F6D6F64653D007573625F7077723D2586
:1005D000730A0072656C61793D25730A0074746C4E
:1005E0003D252D640A0052494D455F616464723DAA
:1005F000252D642E252D640A006E65696768626F7B
:10060000725F7461626C655F73697A653D25640A27
:1006100000765F6C6F773D252D332E32660A0074AD
:100620007870773D25640A006368616E3D25640A31
:100630000069643D006932635F6275733D00693231
:10064000635F73706565643D252D6C750A00747871
:10065000743D25730A0053797374656D2053756D6D
:100660006D6172790A002530366C780041744D65F1
:100670006761323536524652320041744D656761CA
:10068000313238524652320041744D65676136341A
:10069000524652320041744D6567613132385246DC
:1006A0004131004D43553D006D61736B3D002C00A1
:1006B000696E74657276616C3D252D750023252D5C
:1006C000642C007062320070623100745F68656192
:1006D000745F69647800745F6465770061680070B6
:1006E0005F6D73353631310072685F7368743278CC
:1006F00000745F7368743278007061007000616428
:10070000340061643300616432006164310061333C
:1007100000613200613100765F696E0072680065C9
:10072000727200757074696D650070315F6C7374FE
:100730000070315F740070310070305F6C73740052
:1007400070305F7400703000765F6D637500745FA9
:100750006D6375007431007400696400653634009F
:10076000747874002D002B006175746F006E6F6ECD
:10077000650062756C6B00706F7765725F73617690
:10078000655F6C656472790072656C61795F6C6538
:10079000647900636F6D7061737300616363656C8E
:1007A000007072657300705F70777200616573002E
:1007B00070315F6C6564790070305F6C65647200E5
:1007C0006576656E74006C6564006F7700706B749D
:1007D0000074785F6C6564790072785F6C65647230
:1007E000006F706572006E6F6E65002530327800A4
:1007F000765F6164343D252D382E36660020007604
:100800005F6164333D252D382E3666002000765F0B
:100810006164323D252D382E3666002000765F61FA
:1008200064313D252D382E3666002000765F6C69D8
:100830006768743D252D382E3666002000765F618E
:10084000323D252D372E3366002000765F61313D25
:10085000252D372E3366002000765F696E3D252DED
:10086000352E326600204E657665722D757365648F
:1008700020737461636B203E202564206279746567
:10088000730A00757074696D653D252D642D646172
:1008900079732D253032643A253032643A2530326E
:1008A000642D686F7572730A0074657374205B6FD2
:1008B00066667C317C327C337C347C355D20202044
:1008C00020202020202D2074657374206D6F6465B6
:1008D000730A0D007478205B706B74207061796C02
:1008E0006F61645D202020202020202020202020F7
:1008F0002D2073656E6420726164696F20706B7463
:10090000206B6579626F6172640A0D0077647420F0
:100910005B6F6E7C6F66667C746573745D202020EF
:1009200020202020202020202D20776174636864FF
:100930006F670A0D00765F6C6F77205B765F6C6F78
:10094000775D202020202020202020202020202013
:10095000202D206C6F77657374207265706F7274D0
:1009600020766F6C746167650A0D00757067722080
:100970002020202020202020202020202020202077
:10098000202020202020202D207265626F6F74208F
:1009900076696120626F6F746C6F616465720A0DB5
:1009A0000075617274205B33386B7C35366B7C313B
:1009B00031356B7C3235306B7C3530306B5D202DC2
:1009C00020736574207465726D2F75617274207365
:1009D000706565640A0D00626F6F7420202020200E
:1009E0002020202020202020202020202020202007
:1009F0002020202D207265626F6F740A0D007077C1
:100A00007273205B646565707C6E6F6E655D20201F
:100A1000202020202020202020202D206D637520E4
:100A2000736C656570206D6F64650A0D0072657387
:100A30007420656570726F6D20202020202020209A
:100A40002020202020202020202D20726573746F0C
:100A5000726520656570726F6D0A0D007070777237
:100A6000205B6F6E7C6F66665D202020202020203A
:100A700020202020202020202D2070726F6772619E
:100A80006D6D61626C65207077720A0D0070623264
:100A900020205B6F6E7C6F66665D2020202020200A
:100AA0002020202020202020202D2070726F6772AF
:100AB000616D6D61626C652070696E2062320A0D35
:100AC0000070623120205B6F6E7C6F66665D202057
:100AD000202020202020202020202020202D2062C7
:100AE000756C6B204750494F2070696E0A0D007479
:100AF0007874205B737472696E675D2020202020FB
:100B000020202020202020202020202D205365740C
:100B1000207265706F7274207465787420737472BB
:100B2000696E670A0D0074787077205B31352D305F
:100B30005D20202020202020202020202020202078
:100B400020202D205458205077722E204869676845
:100B5000657374203020283364426D290A0D0074B7
:100B6000746C205B302D31355D202020202020202A
:100B700020202020202020202020202D2074696D7E
:100B8000652D746F2D6C69766520666F72207061BB
:100B9000636B6574730A0D0073732020202020207E
:100BA0002020202020202020202020202020202045
:100BB000202020202D2073797374656D2073756D4E
:100BC0006D6172790A0D0072732020202020202090
:100BD0002020202020202020202020202020202015
:100BE0002020202D20726164696F207374617473FA
:100BF0000A0D007269205B236E5D205B696E745D77
:100C00002020202020202020202020202020202DD7
:100C1000207265706F727420696E74657276616C93
:100C20000A0D0072636D64205B6F6E7C6F66665D9B
:100C30002020202020202020202020202020202DA7
:100C400020616C6C6F7720636D642066726F6D201D
:100C50006E65746F726B0A0D007265205B236E5DAA
:100C6000205B2B7C2D5D205B6D61736B7C617574EB
:100C70006F2C6D61736B5D202D206D6F746520721C
:100C800065706F7274207365742F6D6F6469667917
:100C90000A0D006F772020202020202020202020F7
:100CA0002020202020202020202020202020202D37
:100CB000206F6E652D776972652073656E736F7234
:100CC000730A0D006C6F67205B6175746F7C6F6ECB
:100CD0007C6F66665D2020202020202020202020A0
:100CE0002D206D6F7465732064617461206F6E20B8
:100CF0005553420A0D006E65205B666C7573685D26
:100D000020202020202020202020202020202020E3
:100D100020202D206E65696768626F7220746162A1
:100D20006C650A0D00657272202020202020202092
:100D300020202020202020202020202020202020B3
:100D4000202D206572726F722073746174730A0DA6
:100D5000006D6375202020202020202020202020CE
:100D6000202020202020202020202020202D206D29
:100D7000637520696E666F0A0D00693263205B70CF
:100D8000726F62657C737065656420236E5D2020E0
:100D90002020202020202D206932632070726F6275
:100DA00065206275737C736574206275732073703F
:100DB0006565640A0D006964205B72657365745D26
:100DC0002020202020202020202020202020202023
:100DD00020202D2069642068616E646C696E670A4A
:100DE0000D0068756D20202020202020202020204C
:100DF00020202020202020202020202020202D20E6
:100E000068756D69646974792073656E736F720AB1
:100E10000D0072656C6179205B6F6E7C6F66667C1D
:100E200073746174735D20202020202020202D20E9
:100E300072656C6179206E6574776F726B20726574
:100E4000706F7274730A0D006465205B6D61736B63
:100E50005D20202020202020202020202020202055
:100E6000202020202D2064656275670A0D006368CC
:100E7000616E205B31312D32365D20202020202014
:100E8000202020202020202020202D206368616E3B
:100E90002031312D32362028322E3430352D323467
:100EA0003830204D687A290A0D0063616C69205B37
:100EB0005B765F696E7C61317C61325D20766F6C40
:100EC000747C72657365747C6E6F6E655D202D2019
:100ED00063616C6962726174650A0D0062756C6BA6
:100EE000205B5B73686F777C666C7573685D205BF5
:100EF0007365742074687273682064656C61795DD1
:100F00005D20202D2062756C6B696E6720706163B7
:100F10006B657473200A0D0061646320202020201B
:100F200020202020202020202020202020202020C1
:100F3000202020202D2073686F7720765F696E2C2B
:100F40002061312C20613220766F6C74616765738B
:100F50000A0D007520202020202020202020202085
:100F60002020202020202020202020202020202D74
:100F700020757074696D650A0D0076202020202090
:100F80002020202020202020202020202020202061
:100F90002020202020202D2076657273696F6E0A34
:100FA0000D0068202020202020202020202020202C
:100FB00020202020202020202020202020202D2024
:100FC00068656C700A0D00256300756E6B6E6F7737
:100FD0006E20636D640A00484D4335383833002570
:100FE0007300257300202573002025362E326620DD
:100FF00000253032780074656D705F6578746572B5
:101000006E3D252D362E32660020257300202536B4
:101010002E3266204F6E2D426F6172640025303291
:10102000780074656D705F626F6172643D252D3666
:101030002E3266000A0042756C6B2072656D3A2094
:1010400073746172743D25752C20656E643D257541
:101050002C20696E5F7573653D25750A0042756CBD
:101060006B206164643A2073746172743D25752C41
:1010700020656E643D25752C20696E5F7573653D36
:1010800025750A0042756C6B207468726573683A46
:101090002074696D65723D25750A00503A20256CF3
:1010A000642050612020252D372E3266206D0A00E5
:1010B0004932433A2000452025642E256420636C84
:1010C0006F636B20256C752063707520256C75200F
:1010D0006C706D20256C752069727120256C7520EF
:1010E000676C656420256C7520796C656420256CBF
:1010F0007520726C656420256C7520747820256CD1
:1011000075206C697374656E20256C752073656E2F
:10111000736F727320256C752073657269616C2022
:10112000256C750A00532025642E256420636C6F9E
:10113000636B20256C7520747820256C752072787F
:1011400020256C752072747820256C752072727859
:1011500020256C75207265786D697420256C75206A
:1011600061636B747820256C75206E6F61636B749E
:101170007820256C752061636B727820256C752052
:1011800074696D65646F757420256C752062616487
:1011900061636B727820256C7520746F6F6C6F6E55
:1011A0006720256C7520746F6F73686F72742025CB
:1011B0006C752062616473796E636820256C75209C
:1011C00062616463726320256C7520636F6E746561
:1011D0006E74696F6E64726F7020256C7520736514
:1011E0006E64696E6764726F7020256C75206C6C1C
:1011F000747820256C75206C6C727820256C750ACB
:1012000000257325730A004F6E6C696E650A000A2B
:10121000002C20636865636B2072617465202575FE
:1012200020487A0025732025732C206368616E6E38
:10123000656C20257520706F776572202575000A12
:101240000025783A004D41432061646472657373F0
:10125000200052616E646F6D20455549363420611F
:101260006464726573732067656E6572617465642A
:101270000A000A2A2A2A2A2A2A2A426F6F74696EC9
:10128000672025732A2A2A2A2A2A2A0A0045455035
:10129000524F4D20697320636F72727570742C20E9
:1012A000726577726974696E672077697468206403
:1012B000656661756C74732E0A006C6F63616C688F
:1012C0006F73740041544D45474131323872666145
:1012D0003100020000FFFE0000016E616E00696EC9
:1012E000660000407A10F35A00A0724E18090010F0
:1012F000A5D4E80000E87648170000E40B5402008B
:1013000000CA9A3B000000E1F505000080969800B5
:10131000000040420F000000A086010000001027DE
:1013200000000000E803000000006400000000006E
:101330000A00000000000100000000002C76D888A0
:10134000DC674F0823DFC1DFAE59E1B1B796E5E3B3
:10135000E453C63AE651997696E8E6C28426EB89CC
:101360008C9B62ED407C6FFCEFBC9C9F40F2BAA569
:101370006FA5F490055A2AF75C936B6CF9676DC101
:101380001BFCE0E40D47FEF520E6B500D0ED902E05
:101390000300943577050080841E080000204E0A63
:1013A000000000C80C333333330F986E12831141A1
:1013B000EF8D2114893BE65516CFFEE6DB18D1846C
:1013C0004B381BF77C1D901DA4BBE4242032847293
:1013D0005E228100C9F124ECA1E53D274E414E4932
:1013E0004E495459494E46CDCCCC3D0AD7233C17E3
:1013F000B7D13877CC2B329595E6241FB14F0A0030
:101400000020410000C84200401C4620BCBE4CCA1F
:101410001B0E5AAEC59D740011241FBECFEFD1E440
:10142000DEBFCDBF1AE0A0E0B2E0EEE3FCE301E0F6
:101430000BBF02C007900D92AA34B107D9F72DE374
:10144000AAE4BAE001C01D92A437B207E1F70E94F6
:10145000928B0C941D9E0C9400008115910511F047
:101460000197F1F7089584E295E09F938F930E948E
:10147000FC9A8091620290916302A0916402B09103
:1014800065020F900F9093FF03C08EE195E002C0BC
:1014900088E195E09F938F930E94FC9A0F900F90A4
:1014A0000895E091111CEF73F0E0EE59F34E808344
:1014B0008091111C8F5F8093111C8091B2348860E1
:1014C0008093B23448E452E061E1CA010E94F75BC4
:1014D00080E090E00895CF93DF93EC018091550A6E
:1014E0009091560AA091570AB091580A86FF1DC0E4
:1014F0008E811F928F938D811F928F938C811F926B
:101500008F938B811F928F938A811F928F9381E794
:1015100093E09F938F930E94E89A8DB79EB70C96A5
:101520000FB6F8949EBF0FBE8DBFBE0186E99AE04C
:101530000E942B5DBE0184E092E0DF91CF910C947C
:101540009F5C52985A981DBAE9E6F0E0808180626B
:101550008083EA9A53985B98EB9A808180688083B5
:10156000E8E6F0E08081816080830895E7ECFCE1AB
:101570001182128210820895CF92DF92EF92FF9231
:101580000F931F93CF93DF93EC019B018091C71CB6
:10159000843108F0BBC08091C91C64E10E94DA93D9
:1015A0009093C91CC090E42FD090E52FE090E62FD7
:1015B000F090E72F092F10E08DE8989FD0011124BB
:1015C000A953B34E1396CD92DD92ED92FC921697ED
:1015D0004115510559F0FA018081FD01EA57FF4F8D
:1015E0008083FA018181A957BF4F8C932097A9F07E
:1015F00089819DE8909FF001919FF00D1124E9539E
:10160000F34EDF01A657BF4F8C93E557FF4F8881FC
:101610008F70808388818F70808321153105E1F17F
:10162000D90116964C9116975DE8509FC001519FC5
:10163000900D11248953934EFC01E757FF4F4083CF
:1016400015964C9115973197408334961B964D9182
:101650005D916D917C911E97452F562F672F7727AF
:10166000518340837C01BEE8EB0EF11CF901238518
:10167000348545855685A4E6B0E00E947D94672FA9
:10168000782F892F992724E630E040E050E00E942F
:101690000E94D7016D937C938DE8809FD001819F3C
:1016A000B00D1124A253B34EFE0132968FE7019084
:1016B0000D928A95E1F78091C91C8F5F8093C91CB8
:1016C0009091C71C9F5F9093C71C4091550A509101
:1016D000560A6091570A7091580A60FF2DC01F92F8
:1016E0009F931F928F938091C81C1F928F938DE5BB
:1016F00090E19F938F930E94FC9AEDB7FEB73896C6
:101700000FB6F894FEBF0FBEEDBF16C08091F42F48
:101710009091F52FA091F62FB091F72F0196A11D72
:10172000B11D8093F42F9093F52FA093F62FB093D3
:10173000F72F80E090E002C081E090E0DF91CF9150
:101740001F910F91FF90EF90DF90CF90089520911F
:10175000C71C222361F18091C81C8F5F2150209308
:10176000C71C64E10E94DA939093C81C4091550A0B
:101770005091560A6091570A7091580A60FF1AC03A
:101780001F922F938091C91C1F928F931F929F933A
:1017900086E390E19F938F930E94FC9A8DB79EB74A
:1017A00008960FB6F8949EBF0FBE8DBF03C080E0B1
:1017B00090E0089581E090E0089581110C94A10AD1
:1017C000109269005A9AEA985B9AEB9808951F92D2
:1017D0000F920FB60F9211248F939F93AF93BF93E5
:1017E0008091680080FF24C080918D3490918E3468
:1017F000A0918F34B09190340196A11DB11D8093BA
:101800008D3490938E34A0938F34B0939034809124
:10181000550A9091560AA091570AB091580A87FF2D
:1018200007C0749882E090E090938F0280938E02BC
:10183000BF91AF919F918F910F900FBE0F901F900E
:1018400018951F920F920FB60F9211248F939F93AA
:10185000AF93BF938091680080FF24C08091913442
:1018600090919234A0919334B09194340196A11D3B
:10187000B11D8093913490939234A0939334B0939C
:1018800094348091550A9091560AA091570AB091CC
:10189000580A90FF07C0739882E090E090938F02FF
:1018A00080938E02BF91AF919F918F910F900FBE49
:1018B0000F901F90189580937C0080917B00877F0C
:1018C00080937B0080917C00806C80937C0085E01D
:1018D00080937A0080917A00806880937A0080916A
:1018E0007B0087FFFCCF80917B0085FFFCCF809140
:1018F0007A00806480937A0080917A0086FDFCCF24
:10190000109279001092780084E090E060E070E03E
:1019100020917A00206420937A0020917A0026FD9D
:10192000FCCF2091780030917900620F731F0197EE
:1019300079F710927C0080917A008F7780937A00FB
:10194000769567957695679580E090E00E94019185
:10195000089580E00E945B0C2091860230918702FE
:1019600040918802509189020E94FB9221EE3AE751
:1019700044E95EE30E946C8F08950F931F93CF9309
:10198000DF930FE110E0CBE5DEE00093510187EC3F
:1019900090E00E942D0A8091510185FD0DC000311B
:1019A000110521F02CF0CB54D10903C0C4ECD9E0CF
:1019B000E29701501109E9CFBE0180E090E00E945A
:1019C000019120E030E04AE754E40E944F90DF911B
:1019D000CF911F910F910895CF93DF93EC018881F0
:1019E0009981009799F08F3F914121F019821882D7
:1019F00083E011C0623171F40E94BD0C6093E02F4E
:101A00007093E12F8093E22F9093E32F8FEF91E17A
:101A10009983888381E0DF91CF91089580917B0045
:101A2000886080937B0089EC80937C0085E08093C4
:101A30007A0080917A00806880937A0080917B00A0
:101A400087FFFCCF80917B0085FFFCCF80917A00DF
:101A5000806480937A0080917A0086FDFCCF80912B
:101A60007A00806480937A0080917A0086FDFCCFB2
:101A7000609178007091790080917A008F778093DF
:101A80007A0080E090E00E94019127ED33EA40E97E
:101A90005FE30E94FB9226E636E648E853E40E94A4
:101AA0006B8F0895CF92DF92EF92FF921F93CF93A7
:101AB000DF93CDB7DEB729970FB6F894DEBF0FBE20
:101AC000CDBF6C0110924E0A8FEF89878AE1E82E14
:101AD0008CE1F82E10E089858823E9F11830D9F1DE
:101AE000BE016F5F7F4FCE0109960E947A6599858E
:101AF0009F3F11F09E3F19F490934E0A2CC0CE01E7
:101B00000196C114D10481F40E9494658093AF348E
:101B1000A7EAB4E3FE01319688E08E0F91919D9380
:101B20008E13FCCF81E018C00E949465F701808776
:101B3000FE01319620E030E08191D701A20FB31F62
:101B40008C932F5F3F4F28303105B1F71F5FF9E0CD
:101B5000EF0EF11CC0CF812F29960FB6F894DEBF8F
:101B60000FBECDBFDF91CF911F91FF90EF90DF901F
:101B7000CF90089584E390E19F938F930E94FC9A05
:101B80000F900F9008952F923F924F925F926F9215
:101B90007F928F929F92AF92BF92CF92DF92EF92FD
:101BA000FF920F931F93CF93DF93EC015B0100979C
:101BB00011F427E003C0019749F426E04AE250E01F
:101BC0006BE270E089E290E00E945464CE010E94D2
:101BD000520D9E01215B354F6901D9018C93CD2BAC
:101BE00069F0CAE1DCE1E12CF12C89EE282E8FE0CE
:101BF000382E95EE892E9FE0992E9EC087EA94E3B9
:101C00000E94C366BC01990F880B990B0E94039137
:101C10006B017C01AB2869F020E030E048EC52E435
:101C20000E944F909F938F937F936F9382E290E1F6
:101C3000A4C0C7EAD4E30DE110E189911F928F930C
:101C40001F930F930E94FC9A0F900F900F900F908C
:101C5000B4E3CF3ADB0789F720E030E048EC52E408
:101C6000C701B6010E944F909F938F937F936F930C
:101C70008DE090E19F938F930E94FC9A0F900F90BC
:101C80000F900F900F900F908091AF34811103C08F
:101C900084E194E002C080EA93E09F938F9389E00F
:101CA00090E19F938F930E94FC9A0F900F900F905A
:101CB0000F906DC000E010E0FE01E00FF11F808189
:101CC0001F928F93A1EFBFE0BF93AF930E94FC9A46
:101CD0000F5F1F4F0F900F900F900F90083011055E
:101CE00059F720E030E048EC52E4C301B2010E9411
:101CF0004F909F938F937F936F933F922F920E9469
:101D0000FC9A0F900F900F900F900F900F90888576
:101D1000811151C084E194E09F938F939F928F92A1
:101D20000E94FC9A0E94BA0DFFEFEF1AFF0A299653
:101D30000F900F900F900F90D6018C9190E0E816C5
:101D4000F906E4F5CE010E94C366BC01990F880B29
:101D5000990B0E9403912B013C01A114B10409F4D9
:101D6000A9CF20E030E048EC52E40E944F909F93CE
:101D70008F937F936F9386EF9FE09F938F930E9443
:101D8000FC9A0F900F900F900F900F900F90DF9193
:101D9000CF911F910F91FF90EF90DF90CF90BF9068
:101DA000AF909F908F907F906F905F904F903F90FB
:101DB0002F900C94BA0D80EA93E0AECFDF91CF91D3
:101DC0001F910F91FF90EF90DF90CF90BF90AF9059
:101DD0009F908F907F906F905F904F903F902F904B
:101DE0000895CF93DF9300D0CDB7DEB7E7EAF4E3F1
:101DF0008181898387818A83CE0101960E94E65979
:101E00000F900F90DF91CF910895CF93DF93EC0166
:101E10002091A7343091A8344091A9345091AA342C
:101E20006091AB347091AC348091AD349091AE340C
:101E3000AFEF0E944996E1F427E04AE250E06BE2FE
:101E400070E089E290E00E94546480E090E00E949B
:101E5000520DC15BD54F888349E050E06EE070E0E1
:101E600087EA94E30E94009EDF91CF910C94F10EDB
:101E7000DF91CF9108951F920F920FB60F92112408
:101E80000BB60F92FF920F931F932F933F934F9395
:101E90005F936F937F938F939F93AF93BF93CF93F2
:101EA000DF93EF93FF938091B23482608093B234DA
:101EB0008091620286FD2B9A8091620287FD2B9AA7
:101EC00080918E0290918F021816190614F4749A5C
:101ED000739A8091550A9091560AA091570AB09131
:101EE000580A85FF02C074987398809102029091FD
:101EF000030201979093030280930202892B09F059
:101F00004CC18091650A9091660A01969093660A89
:101F10008093650A8091E42F9091E52FA091E62FA0
:101F2000B091E72F0196A11DB11D8093E42F9093EE
:101F3000E52FA093E62FB093E72F80E190E09093F8
:101F40000302809302028091620280FD02C01D9B09
:101F500005C01092530A1092520A06C081E090E028
:101F60009093530A8093520A8091550A9091560A91
:101F7000A091570AB091580A97FF08C08091520A61
:101F80009091530A892B49F0749A739801EC1BE1E4
:101F9000C9EFDFE2FF24F39421C0739A7498F6CF5F
:101FA0008091650A9091660A01960E94E693892BBA
:101FB000E1F0F8016085718561157105A1F5F80101
:101FC000608571856115710509F03FC0065F1F4F7F
:101FD0002596F0E3CD30DF0709F44CC0F8016085A9
:101FE00071856115710529F3DBCF4281417020E0D5
:101FF00030E050E060E070E080E090E0A0E00E941F
:102000004996B9F277988091550A9091560AA09115
:10201000570AB091580A92FFCCCF749810928F0251
:1020200010928E02C6CF8091650A9091660A019641
:102030000E94E693892B19F61C821B82AE0162E195
:1020400080E292E00E94F75BBACF8091650A90919E
:10205000660A0E94E693892B09F0B8CFF8821A83AA
:1020600009831C821B82AE0162E18EE392E00E9432
:10207000F75BACCF609168027091690261157105E0
:10208000A1F18091650A9091660A0E94E693892BDE
:1020900061F580918D3490918E34A0918F34B09100
:1020A00090344091D6275091D7276091D8277091CE
:1020B000D927841B950BA60BB70B8093E91B909334
:1020C000EA1BA093EB1BB093EC1B80918D34909195
:1020D0008E34A0918F34B09190348093D627909312
:1020E000D727A093D827B093D92760916602709123
:1020F000670261157105A1F18091650A9091660AE8
:102100000E94E693892B61F58091913490919234ED
:10211000A0919334B09194344091DA275091DB2709
:102120006091DC277091DD27841B950BA60BB70B04
:102130008093ED1B9093EE1BA093EF1BB093F01BCD
:102140008091913490919234A0919334B0919434D1
:102150008093DA279093DB27A093DC27B093DD27C9
:102160008091620286FD2B988091620290916302B9
:10217000A0916402B091650291FF0FC00E94BB70F4
:102180008A3119F0C1E0C80F01C0CBE00E94716F25
:102190008C2F0E94D3700E94B96F40E050E060E045
:1021A00080E992E00E94F75BFF91EF91DF91CF9180
:1021B000BF91AF919F918F917F916F915F914F915F
:1021C0003F912F911F910F91FF900F900BBE0F9099
:1021D0000FBE0F901F9018958091111C9091F82FB1
:1021E000891B08950E94EC10882371F0E091F82F6C
:1021F000EF73F0E0EE59F34E808190E02091F82FDC
:102200002F5F2093F82F08958FEF9FEF0895CF93BE
:10221000DF93EC0110928A0A1092890A88819981D1
:102220000097C1F0863E934021F01982188283E026
:10223000BDC0613109F0B9C00E94F2109927909396
:10224000850A8093840A8D30910509F444C08F3F3C
:10225000910549F40E94EC108111EECF86EE93E0D7
:1022600099838883A2C08231910509F45AC08F37BF
:10227000910509F052C08091820A9091830A181644
:1022800019060CF560916E3D70916F3D88E090E00D
:102290000E94B09A60916E3D70916F3D80E290E037
:1022A0000E94B09A60916E3D70916F3D88E090E021
:1022B0000E94B09A8091820A9091830A019790932C
:1022C000830A8093820A8091820A9091830A8F37D1
:1022D000910509F0BFCF1092F82F1092111C809138
:1022E000820A9091830AFC01E35FFF4C1082909375
:1022F0008A0A8093890A1092830A1092820A809136
:10230000B0349091B134009709F4A4CF40E050E08C
:10231000609198120E94F75B9DCF8830910571F50E
:10232000AACF60916E3D70916F3D8DE090E00E946C
:10233000B09A1092810A1092800A2091800A3091FE
:10234000810A8091820A9091830A281739070CF03C
:10235000BACFF901E35FFF4C808160916E3D7091CF
:102360006F3D90E00E94B09A8091800A9091810A1E
:1023700001969093810A8093800ADFCF60916E3D31
:1023800070916F3D0E94B09A2091820A3091830A29
:102390008091840AF901E35FFF4C80832F5F3F4FF8
:1023A0003093830A2093820A8ECF81E0DF91CF9110
:1023B00008958091520A9091530A892BD1F080910F
:1023C000620290916302A0916402B091650293FD54
:1023D00010C00E94716F83B7817F866083BFF894BD
:1023E00083B7816083BF7894889583B78E7F83BFDE
:1023F00078940895CF93DF93FC01208131812115DA
:10240000310519F022333241A1F4EC010E942E6E05
:102410000E94D91140E050E065E880919C129091B3
:102420009D120E94F75B82E392E19983888381E0A9
:1024300004C0FC011182108283E0DF91CF910895E6
:10244000CF93DF9300D0CDB7DEB7892B81F05F93B8
:102450004F9382EE9FE09F938F9369837A830E94CC
:10246000FC9A0F900F900F900F907A8169817F9363
:102470006F938FED9FE09F938F930E94FC9A0F9034
:102480000F900F900F900F900F90DF91CF910895C4
:10249000EF92FF920F931F93CF93DF930E942E6EC4
:1024A00080EB0E944D6781111CC00E94AA67809139
:1024B000DE2B9091DF2B81609093DF2B8093DE2BBE
:1024C00089EA93E09F938F938FED9FE09F938F9383
:1024D0000E94FC9A0F900F900F900F90C1E0D0E0F7
:1024E00002C0C0E0D0E01EB11470729A0E942E6E3D
:1024F0008EE40E944D67811117C00E94AA678091E7
:10250000DE2B9091DF2B82609093DF2B8093DE2B6C
:102510007E018FEFE81AF80A40EB59E061EB73E0B7
:10252000CE010E942012E701111101C072980E9491
:102530002E6E8EEE0E944D67811116C00E94AA6712
:102540008091DE2B9091DF2B84609093DF2B809322
:10255000DE2B8E010F5F1F4F40EB59E069EB73E0FC
:10256000CE010E942012E8010E942E6E86EA0E948F
:102570004D67811116C00E94AA678091DE2B909151
:10258000DF2B88609093DF2B8093DE2B8E010F5F13
:102590001F4F40EB59E060EC73E0CE010E94201227
:1025A000E8010E942E6E8CE30E944D6781111EC0CF
:1025B0000E94AA678091DE2B9091DF2B806190931F
:1025C000DF2B8093DE2B8E010F5F1F4F40EB59E016
:1025D00068EC73E0CE010E94201287ED9FE09F938C
:1025E0008F930E94FC9A0F900F90E8010E942E6E2C
:1025F00082ED0E944D67811116C00E94AA678091EA
:10260000DE2B9091DF2B80629093DF2B8093DE2B6B
:102610008E010F5F1F4F40EB59E060ED73E0CE017C
:102620000E942012E8010E942E6E80E80E944D67F1
:10263000811116C00E94AA678091DE2B9091DF2B3A
:1026400091609093DF2B8093DE2B8E010F5F1F4FE5
:1026500040EB59E069ED73E0CE010E942012E801E1
:102660000E942E6E80ED0E944D67811116C00E945F
:10267000AA678091DE2B9091DF2B80689093DF2BEF
:102680008093DE2B8E010F5F1F4F40EB59E06FED03
:1026900073E0CE010E942012E8010E942E6E8CEEA3
:1026A0000E944D67811116C00E94AA678091DE2B9F
:1026B0009091DF2B92609093DF2B8093DE2B8E0125
:1026C0000F5F1F4F40EB59E067EE73E0CE010E94B1
:1026D0002012E80107E010E00E942E6E8CE70E94B5
:1026E0004D67811113C00E94AA678091DE2B9091E3
:1026F000DF2B80649093DF2B8093DE2B40EB59E03F
:102700006EEE73E0CE010E94201203C00150110949
:1027100019F70E94AA67DF91CF911F910F91FF9047
:10272000EF900C94BA0DCF93DF9300D0CDB7DEB706
:102730004A8369830E9481676981862F0E94B267FC
:102740004A81842F0E94B2670F900F90DF91CF9142
:102750000C94AA67AF92BF92CF92DF92EF92FF9252
:102760000F931F93CF93DF9300D01F92CDB7DEB7A7
:10277000182F022F4A835B8369830E9481676981D6
:10278000862F0E94B267812F81600E94A8674A81CC
:10279000A42E5B81B52E10E0E12CF12C680181E0C4
:1027A000C81AD108E016F10689F0EC14FD0419F4FA
:1027B0000E94CD6702C00E94C367F5018083FFEFCE
:1027C000EF1AFF0A8FEFA81AB80AECCF0F900F90FC
:1027D0000F90DF91CF911F910F91FF90EF90DF90BD
:1027E000CF90BF90AF900C94AA67BF92CF92DF9228
:1027F000EF92FF920F931F93CF93DF93CDB7DEB786
:1028000060970FB6F894DEBF0FBECDBFF82EE42E52
:102810006623D9F18E010F5F1F4F80E1F8011192FD
:102820008A95E9F728E0A80168E980EB0E94AA13DD
:10283000FF2041F087EF93E09F938F930E94E89AE7
:102840000F900F902EEFC22E23E0D22E37E0B32E42
:10285000B00EF80181918F011F928F93DF92CF927A
:102860000E94E89A0F900F900F900F90B012F1CF46
:1028700088851F928F9383E594E09F938F930E94A6
:10288000E89A0F900F900F900F90EE20D9F18E01E3
:102890000F5F1F4F80E1F80111928A95E9F720E15F
:1028A000A80160E880EB0E94AA13FF2041F083E0BA
:1028B00094E09F938F930E94E89A0F900F908EEF71
:1028C000E82E83E0F82E9FE0D92ED00EF8018191FA
:1028D0008F011F928F93FF92EF920E94E89A0F90C0
:1028E0000F900F900F90D012F1CF88891F928F9385
:1028F00083E594E09F938F930E94E89A0F900F9046
:102900000F900F9060960FB6F894DEBF0FBECDBF4C
:10291000DF91CF911F910F91FF90EF90DF90CF90BB
:10292000BF9008950F931F93CF93DF9300D0CDB73F
:10293000DEB71A82198222E0AE014F5F5F4F6AEA6A
:102940008EEE0E94AA1302EA1CE1898190E0982F82
:1029500088272A81822BF8019183808322E0AE01AF
:102960004F5F5F4F6CEA8EEE0E94AA13898190E060
:10297000982F88272A81822BF8019383828322E073
:10298000AE014F5F5F4F6EEA8EEE0E94AA138981FF
:1029900090E0982F88272A81822BF80195838483E1
:1029A00022E0AE014F5F5F4F60EB8EEE0E94AA13F4
:1029B000898190E0982F88272A81822BF801938BB8
:1029C000828B22E0AE014F5F5F4F62EB8EEE0E9482
:1029D000AA13898190E0982F88272A81822BF801F9
:1029E000958B848B22E0AE014F5F5F4F64EB8EEEE0
:1029F0000E94AA13898190E0982F88272A81822B30
:102A0000F801978B868B22E0AE014F5F5F4F66EB3C
:102A10008EEE0E94AA13898190E0982F88272A8140
:102A2000822BF8019783868322E0AE014F5F5F4FD0
:102A300068EB8EEE0E94AA13898190E0982F882778
:102A40002A81822BF8019187808722E0AE014F5FB7
:102A50005F4F6AEB8EEE0E94AA13898190E0982F57
:102A600088272A81822BF8019587848722E0AE018E
:102A70004F5F5F4F6CEB8EEE0E94AA13898190E04E
:102A8000982F88272A81822BF8019787868722E052
:102A9000AE014F5F5F4F6EEB8EEE0E94AA138981ED
:102AA00090E0982F88272A81822BF801918B808BC8
:102AB0000F900F90DF91CF911F910F9108952F925A
:102AC0003F924F925F926F927F928F929F92AF92BE
:102AD000BF92CF92DF92EF92FF920F931F93CF930B
:102AE000DF93CDB7DEB76C970FB6F894DEBF0FBE9D
:102AF000CDBF182F042F2D8B19821A821B82809133
:102B0000C61C811107C06C8F0E94921481E08093D3
:102B1000C61C6C8D662309F472C04EE264EF8EEE23
:102B20000E94931369E07AE180E090E00E942A67B6
:102B300022E0AE014F5F5F4F66EF8EEE0E94AA1358
:102B40002981822F90E0A0E0B0E04427582F692F20
:102B50007A2F8A81482B8091B81C9091B91C9A01D8
:102B6000AB01281B390B41095109A091B61CB0914A
:102B7000B71C0E947D946B017C013FE0F594E794C3
:102B8000D794C7943A95D1F76091B01C7091B11C5D
:102B9000CB01770FAA0BBB0BBC01CD014BE0660F3D
:102BA000771F881F991F4A95D1F72091B21C309149
:102BB000B31C4901330FAA08BB08A7019601280DD1
:102BC000391D4A1D5B1D0E943094C20ED31ED09247
:102BD000AD1CC092AC1C28E0C20ED11C54E0D594B0
:102BE000C7945A95E1F70D2C000CEE08FF08C0922F
:102BF000BA1CD092BB1CE092BC1CF092BD1C812F71
:102C00008295880F880F807C8C5C8887212E312CE0
:102C1000A3E0B0E0012E02C0AA0FBB1F0A94E2F7A6
:102C200025E335E00E9476949B01AC012E5F3F4F77
:102C30004F4F5F4F29873A874B875C8780E593EC3E
:102C4000A0E0B0E09C01AD0104C0559547953795D3
:102C500027951A95D2F7298B3A8B4B8B5C8B10E01A
:102C6000412C512C320188E090E0AC01421953090B
:102C70005B8F4A8F101709F43EC1488564EF8EEED2
:102C80000E94931369857A858B859C850E942A67AB
:102C900023E0AE014F5F5F4F66EF8EEE0E94AA13F6
:102CA000E091AC1CF091AD1CE05AFF409F01DF01A8
:102CB0000E945F946C837D838E839F838091A41C8C
:102CC0009091A51C9E878D872091A21C3091A31CFA
:102CD000388B2F872091A61C3091A71C0E945F94EF
:102CE0006B017C01ADE0F594E794D794C794AA9565
:102CF000D1F7A091A81CB091A91C2C813D814E81D7
:102D00005F818CE055954795379527958A95D1F742
:102D10000E948894BB2797FDB095AB2F8C0D9D1D0D
:102D2000AE1DBF1D0296A11DB11D32E0B595A79540
:102D3000979587953A95D1F79C01AD0130584F4F43
:102D40005F4FA091B41CB091B51C0E947D944B01C3
:102D50005C014FE0B694A794979487944A95D1F775
:102D600039818A8190E0A0E0B0E0BA2FA92F982F96
:102D70008827A32B2B81822B9C01AD010A8C04C0D8
:102D800055954795379527950A94D2F72E8B3F8B0B
:102D9000488F598F4F8558896A01550FEE08FF08F3
:102DA00062E0CC0CDD1CEE1CFF1C6A95D1F7A091F3
:102DB000AA1CB091AB1C2C813D814E815F810E9489
:102DC00088949B01AC0177E15595479537952795F8
:102DD0007A95D1F72C833D834E835F832D853E8585
:102DE000DF010E945F94DC01CB01EBE0B595A79574
:102DF00097958795EA95D1F72C813D814E815F812A
:102E0000820F931FA41FB51FC80ED91EEA1EFB1EFA
:102E1000022C04C0CC0CDD1CEE1CFF1C0A94D2F763
:102E200032E0C30ED11CE11CF11CF2E0F594E794F2
:102E3000D794C794FA95D1F72E893F89488D598D3B
:102E40002C193D094E095F0969897A898B899C890A
:102E50000E94CA9397FD0BC0660F771F881F991FAA
:102E6000A50194010E940E9469017A010AC0A5018E
:102E700094010E940E9469017A01CC0CDD1CEE1CB9
:102E8000FF1C9927F7FC9A958F2D7E2D6D2D9B01A8
:102E9000AC010E94CA939B01AC01AEEDBBE00E9465
:102EA0007D944C01BB2497FCB094AB2CA3E4B3EE0F
:102EB000A70196010E948B94BB2797FDB095AB2F7D
:102EC000880E991EAA1EBB1E4FEC840E4EE0941E67
:102ED000A11CB11C44E0B594A794979487944A959B
:102EE000D1F7C80CD91CEA1CFB1C4C0C5D1C6E1CD9
:102EF0007F1C1F5FBFCE112381F0212F30E040E007
:102F000050E0C301B2010E940E942093BE1C309386
:102F1000BF1C4093C01C5093C11C5D89552389F18F
:102F20006091BE1C7091BF1C8091C01C9091C11C0F
:102F3000611571058105910521F10E94039120E839
:102F400036EE45EC57E40E944F9021E03EED42E41E
:102F50005EE30E9468939B01AC0160E070E080E852
:102F60009FE30E946B8F2BE43AE34DEB57E30E9403
:102F70004F906093C21C7093C31C8093C41C9093A9
:102F8000C51C6C960FB6F894DEBF0FBECDBFDF91A7
:102F9000CF911F910F91FF90EF90DF90CF90BF9056
:102FA000AF909F908F907F906F905F904F903F90E9
:102FB0002F9008950F931F93CF93DF9300D000D0ED
:102FC00000D0CDB7DEB78E010F5F1F4F86E0F8014E
:102FD00011928A95E9F78091B81B811113C040E0E6
:102FE00061E386EA0E9493134AE06CE286EA0E945B
:102FF000931381E08093B81B6CE77EE380E090E060
:103000000E942A6748E06DE286EA0E9493136CE70B
:103010007EE380E090E00E942A6726E0A80162E358
:1030200086EA0E94AA1347E06DE286EA0E949313A3
:103030008A8190E0982F88272981822B9093B31B57
:103040008093B21B2C8130E0322F22274B81242B1E
:103050003093B51B2093B41B4E8150E0542F44276E
:103060006D81462B5093B71B4093B61B5F934F93D4
:103070003F932F939F938F9387E094E09F938F9339
:103080000E94E89A0FB6F894DEBF0FBECDBF269619
:103090000FB6F894DEBF0FBECDBFDF91CF911F9169
:1030A0000F910895CF92DF92EF92FF920F931F93AB
:1030B000CF93DF93CDB7DEB72A970FB6F894DEBF74
:1030C0000FBECDBF8E010F5F1F4F86E0F80111923A
:1030D0008A95E9F741E062E08CE30E94931348E5AA
:1030E00060E08CE30E94931362E174E380E090E07F
:1030F0000E942A6726E0A80163E08CE30E94AA13DD
:1031000043E062E08CE30E949313098110E0102FEA
:1031100000278A81082BE2E9FBE111830083EB8021
:10312000F12CFE2CEE248C81E82AF382E282CD8001
:10313000D12CDC2CCC248E81C82AD582C482B80143
:10314000012E000C880B990B0E9403919B01AC018E
:10315000B7010F2C000C880B990B2F8338874987F8
:103160005A870E9403912F81388549855A850E948C
:10317000EB8F20EE3EE245E652E40E94FB9220E017
:1031800030E044E353E40E946C8F9F938F937F93CE
:103190006F93DF92CF92FF92EF921F930F9385E18F
:1031A00094E09F938F930E94E89A0FB6F894DEBF45
:1031B0000FBECDBF2A960FB6F894DEBF0FBECDBFAF
:1031C000DF91CF911F910F91FF90EF90DF90CF9003
:1031D0000895CF93DF93EC0188819981009759F18D
:1031E0008B31924121F01982188283E06FC08FE603
:1031F0009AE00E94A35E892B41F18091550A90913B
:10320000560AA091570AB091580A93FD20C08091A8
:10321000550A9091560AA091570AB091580A94FD08
:1032200047C08091550A9091560AA091570AB091D3
:10323000580A95FD44C060E870E08FE69AE00E946D
:103240007C5E8BE192E19983888381E03FC080912D
:10325000DE2B82FFDCCF21E048E061E083E00E94CA
:103260005F158091C51C8F938091C41C8F938091B2
:10327000C31C8F938091C21C8F938091C11C8F932C
:103280008091C01C8F938091BF1C8F938091BE1C36
:103290008F938BE990E19F938F930E94FC9A8DB757
:1032A0009EB70A960FB6F8949EBF0FBE8DBFAFCFE4
:1032B0008091DE2B83FFB5CF0E94DA17B2CF8091C9
:1032C000DE2B84FFB8CF0E945218B5CFDF91CF918B
:1032D0000895CF93C82F8CEE0E94A8678C2F0E9470
:1032E000B26765E375E080E090E00E942A678DEEAA
:1032F0000E94A8670E94C367C82F0E94CD672C2F29
:1033000030E0322F2227A901482BCA01CF9108951E
:103310000F931F93CF93DF93C82F8CEE0E94A86763
:103320008C2F0E94B26762E174E380E090E00E941B
:103330002A678CEE0E94A86780E00E94B26765E36E
:1033400075E080E090E00E942A678DEE0E94A867F9
:103350000E94C367C82F0E94C367D82F0E94CD6701
:103360004D2F50E060E070E0762F652F542F4427FA
:103370006C2B8A019B01082BC901B801DF91CF9109
:103380001F910F9108952F923F924F925F926F92EB
:103390007F928F929F92AF92BF92CF92DF92EF92E5
:1033A000FF920F931F93CF93DF93CDB7DEB7CB542C
:1033B000D1090FB6F894DEBF0FBECDBF80910002D9
:1033C00090910102892BD1F110920102109200021A
:1033D0008CEE0E94A8678EE10E94B2676BE17EE4EA
:1033E00080E090E00E942A6782EA0E946919909327
:1033F000640A8093630A84EA0E9469199093620ABE
:103400008093610A86EA0E9469199093600A80930A
:103410005F0A88EA0E94691990935E0A80935D0AA8
:103420008AEA0E94691990935C0A80935B0A8CEA8D
:103430000E94691990935A0A8093590A88E40E945D
:1034400088196DAB7EAB8FAB98AF88E50E94881969
:103450004B015C0180915B0A90915C0A8C0120E039
:1034600030E040E050E0BA0122968FAF22972396D9
:103470001FAF239724962FAF249725963FAF25970C
:1034800026964FAF269727965FAF279728966FAF60
:10349000289729967FAF29979C0140E050E060E093
:1034A00070E080E090E008E00E94EB950E94A49517
:1034B0003901B42FA52FF62FE72F8C019401A50118
:1034C00060E070E080E090E05301CB2EDA2EEF2E2A
:1034D000FE2E0E9422962CA33BA34B83252E362E34
:1034E000472E582E792E632D742D852D972D315012
:1034F00041095F4F6F4F7F4F8F4F9F4F88248394B9
:10350000912C21153F4F4F4F5140610571058105A9
:10351000910509F010F4812C912C9A8289820091F6
:10352000590A10915A0A5801C12CD12CE12CF12CC6
:1035300000E010E02CA13BA14B81522D632D742D96
:10354000852D972D0E949094F22E032F142FB52FC6
:10355000F62FE72FD82EE92EA0E00E94499684F49A
:103560002150310940485F4F6F4F7F4F8F4F9F4F22
:10357000F22E032F142FB52FF62FE72FD82EE92E7A
:103580002F2D302F412F5B2F6F2F7E2F8D2D9E2DB6
:1035900007E10E9404962B8F3C8F4D8F5E8F6F8FBB
:1035A00078A389A39AA32053384F4F4F5F4F6F4F93
:1035B0007F4F8F4F9F4F2B8B3C8B4D8B5E8B6F8B39
:1035C000788F898F9A8F2056304F4F4F5F4F6F4FB4
:1035D0007F4F8F4F9F4F243D30434105510561057B
:1035E00071058105910529F020F0F4013196FA83E7
:1035F000E9838090610A9090620A940140E050E073
:1036000060E070E080E090E000E10E94EB952C83A8
:103610003D834E835F83662E78874C0140915D0A1F
:1036200050915E0AACA0BBA0CB80D22CE32CF42C32
:10363000052D172D9A0140E050E060E070E080E039
:1036400090E00E949094F22E032F142FB52FF62FA6
:10365000E72FD82EE92EA0E00E9449965CF4AFE750
:103660000E942B96F22E032F142FB52FF62FE72F43
:10367000D82EE92E2F2D302F412F5B2F6F2F7E2F2D
:103680008D2D9E2D07E00E94049659016A017B0151
:103690008C012C813D814E815F81662D7885C4012E
:1036A0000E9422962C833D834E835F8368877E87AA
:1036B0008F87988B2E5F3F4F434051096E4F7F4F4E
:1036C0008F4F9F4F22303105494F5F4F6440710546
:1036D0008105910539F030F009811A810F5F1F4F84
:1036E0001A8309836091630A7091640A80E090E014
:1036F00020E030E840E050E00E94E99429873A87D2
:103700004B875C87662E7D874C0140915F0A509104
:10371000600AACA0BBA0CB80D22CE32CF42C052DEE
:10372000172D9A0140E050E060E070E080E090E00A
:103730000E949094F22E032F142FB52FF62FE72F0F
:10374000D82EE92EA0E00E94499684F421503F4FE4
:103750004F4F5F4F6F4F7F4F8F4F9F4FF22E032F73
:10376000142FB52FF62FE72FD82EE92E2F2D302F1F
:10377000412F5B2F6F2F7E2F8D2D9E2D08E00E94F5
:10378000049659016A017B018C0129853A854B8594
:103790005C85662D7D85C4010E94229629873A8723
:1037A0004B875C876D87798B8A8B692E2F5F3F4FA4
:1037B000414051096109710981099109213030485D
:1037C0004C4F5F47614071058105910539F030F03C
:1037D00029813A812F5F3F4F3A8329832B893C8986
:1037E0004D895E896F89788D898D9A8D2F3C374000
:1037F00041055105610571058105910511F00CF038
:10380000A4C1ACA0BBA0CB80D22CE32CF42C052D02
:10381000172D95014C2D522D632D742D852D972D2F
:103820000E949094A12CB12CC12CE0E8DE2EE12C5A
:10383000F12C00E010E00E94169529AF3AAF4BAF93
:103840005CAF6DAF7EAF8FAF21969FAF2197AB8CF2
:10385000BC8CCD8CDE8CEF8CF8A009A11AA195014F
:10386000A601B701C8010E94909459016A017B0129
:10387000E82F192F02E00E94EB950E2F0E9422964E
:103880007901142F552EF62FE72F6C01922EAF2CB5
:10389000B42E052F462EB72F782E8D2CA0E00E9437
:1038A00049965CF4A1E00E942B96922EA32EB42E92
:1038B000052F462EB72F782E892E292D3A2D4B2DE8
:1038C000502F642D7B2F872D982D01E00E940496A8
:1038D0002AA7732E4A012C966FAF2C972B967FAF99
:1038E0002B978BA79CA72B833BA34CA39DA26EA3D6
:1038F0007FA388A799A7B52D9701412F552D6F2F2D
:103900007E2FC601A0E00E9449964CF4A3E00E94DD
:103910002B967901142FB52FF62FE72F6C01970105
:10392000412F5B2F6F2F7E2FC60102E00E9404966D
:103930002DA73EA74FA758AB69AB7AAB8BAB9CAB1F
:103940002901B42FA52F22966FAF2297F72F1C01C4
:103950002B893C894D895E896F89788D898D9A8DF7
:1039600024323A4F4F4F5F4F6F4F7F4F8F4F9F4FD4
:103970000CF08BC02B8D3C8D4D8D5E8D6F8D78A1A5
:1039800089A19AA12455324F4F4F5F4F6F4F7F4F00
:103990008F4F9F4F59016A017B018C010E949094C7
:1039A00019012A01B62FA72FFC0103E00E94EB9515
:1039B00051016201EB2EFA2E8F010E9437965901B8
:1039C0006A017B018C012AA5372DA4012C966FADCD
:1039D0002C972B967FAD2B978BA59CA50E942296AA
:1039E0002B833BA34CA35DA36EA37FA388A799A7BA
:1039F0009101A2016B2F7A2FCF0102E00E94EB957B
:103A000051016201EB2EFA2E8F010E94379602E0DF
:103A10000E94EB950E2F0E943796122FD32EE42E84
:103A2000B52FF62FE72FF82E092FA0E00E94499618
:103A30005CF4A1E00E942B96122FD32EE42EB52F1A
:103A4000F62FE72FF82E092F212F3D2D4E2D5B2F1E
:103A50006F2F7E2F8F2D902F01E00E940496590129
:103A60006A017B018C012DA53EA54FA558A969A926
:103A70007AA98BA99CA90E9422962901B42FA52F6F
:103A800022966FAF2297F72F1C012C813D814E812A
:103A90005F8168857E858F859889AB80BBA0CCA02F
:103AA000DDA0EEA0FFA008A519A50E9437962C83E3
:103AB0003D834E835F8368877E878F87988B2985B8
:103AC0003A854B855C856D8579898A89962D520169
:103AD000CB2EDA2E2296EFAC2297FF2E81010E9488
:103AE000379629873A874B875C876D87798B8A8BD6
:103AF000692E2B893C894D895E896F89788D898DE6
:103B00009A8DA9ACBAACCBACDCACEDACFEAC0FADD5
:103B100021961FAD21970E9437962056304F4F4F68
:103B20005F4F6F4F7F4F8F4F9F4F243D3043410575
:103B30005105610571058105910539F030F0098164
:103B40001A810F5F1F4F1A8309834DA95EA96FA9C0
:103B500078AD9A01AB0160E070E0CB0122962FAF07
:103B6000229723963FAF239724964FAF249725960D
:103B70005FAF259726966FAF269727967FAF27973B
:103B800028968FAF289729969FAF2997A984BA8442
:103B9000CB84DC84ED84F9880A89162D60E070E01E
:103BA00080E090E00E949094122FD32EE42EB52F47
:103BB000F62FE72FF82E092FA0E00E94499684F4F3
:103BC00021503109404E5F4F6F4F7F4F8F4F9F4FB6
:103BD000122FD32EE42EB52FF62FE72FF82E092F14
:103BE000212F3D2D4E2D5B2F6F2F7E2F8F2D902F50
:103BF00005E10E940496AC80BD80CE80DF80E88421
:103C0000FE840F8518890E943796122FD32EE42E3A
:103C1000B52FF62FE72FF82E092FA0E00E94499626
:103C200084F4215030484F4F5F4F6F4F7F4F8F4F7D
:103C30009F4F122FD32EE42EB52FF62FE72FF82EFD
:103C4000092F212F3D2D4E2D5B2F6F2F7E2F8F2D76
:103C5000902F0FE00E94049639014A015B016C012C
:103C600079018A011B012C01285E33404109510969
:103C70006109710981099109283D304D4140510583
:103C8000610571058105910531F028F0E981FA811E
:103C90003196FA83E9830E94AA6729813A81232B0E
:103CA00051F09301A401B501C6010E94A4957901C8
:103CB0008A011B012C019701A801B101C2010E94D8
:103CC000FB9020E030E048EC52E40E944F90C55B4E
:103CD000DF4F0FB6F894DEBF0FBECDBFDF91CF919F
:103CE0001F910F91FF90EF90DF90CF90BF90AF901A
:103CF0009F908F907F906F905F904F903F902F900C
:103D000008954F925F926F927F928F929F92AF929F
:103D1000BF92CF92DF92EF92FF922B013C0169019B
:103D20007A0123EC35EF4CE851E4C701B6010E945B
:103D3000FB924B015C0128EB3EE143E753E4C701F2
:103D4000B6010E946C8F9B01AC01C501B4010E94B9
:103D50004F900E94C9904B015C0120E030E048EC9C
:103D600052E4C301B2010E944F9021E835E943ECCF
:103D700050E40E94FB92A50194010E94FB924B012A
:103D80005C0123E333E948E853E4C701B6010E942C
:103D90006C8F9B01AC01C501B4010E944F9023E3DD
:103DA00033EB48E553E40E94FB92FF90EF90DF90E5
:103DB000CF90BF90AF909F908F907F906F905F90CB
:103DC0004F9008954F925F926F927F928F929F9241
:103DD000AF92BF92CF92DF92EF92FF9269017A0188
:103DE0000E946F9220E030E040E050E40E946B8F30
:103DF00022E93CE54EED5EE30E944F904B015C01F1
:103E000023EC35EF4CE851E4C701B6010E94FB9268
:103E10002B013C0128EB3EE143E753E4C701B60127
:103E20000E946C8F9B01AC01C301B2010E944F90B4
:103E30009B01AC01C501B4010E946C8F6B017C0138
:103E400028EB3EE143E753E40E94FB924B015C0107
:103E5000A701960163EC75EF8CE891E40E946B8FEB
:103E60009B01AC01C501B4010E944F90FF90EF90FF
:103E7000DF90CF90BF90AF909F908F907F906F908A
:103E80005F904F9008954F925F926F927F928F92C2
:103E90009F92AF92BF92CF92DF92EF92FF922B014F
:103EA0003C0169017A0123EC35EF4CE851E4C7018C
:103EB000B6010E94FB924B015C0128EB3EE143E717
:103EC00053E4C701B6010E946C8F9B01AC01C50190
:103ED000B4010E944F900E94C9904B015C0120E008
:103EE00030E048EC52E4C301B2010E944F90A501BA
:103EF00094010E94FB9220E030E040E251E40E94F5
:103F00006B8F24EE38E34EE05FE30E94FB929B014F
:103F1000AC01C701B6010E946C8FFF90EF90DF905B
:103F2000CF90BF90AF909F908F907F906F905F9059
:103F30004F90089580E80E94A86781110DC08EEF10
:103F40000E94B267811108C06BE17EE480E090E0DE
:103F50000E942A670C94AA670E94AA678091F02F9A
:103F60009091F12FA091F22FB091F32F0196A11D06
:103F7000B11D8093F02F9093F12FA093F22FB09367
:103F8000F32F0895FC01DC01AC014E5F5F4F90E020
:103F900031E38D91982788E0292F220F97FF03C0E6
:103FA000922F932701C0922F8150B1F7A417B50724
:103FB00081F721E030E08281981711F020E030E0B5
:103FC000C9010895DF92EF92FF920F931F93CF9351
:103FD000DF930E949A1F80E80E94A86781116DC03C
:103FE0008AEF0E94B267811168C08FE00E94B267B9
:103FF000811163C065E375E080E090E00E942A676C
:1040000081E80E94A867811158C00E94C367D82F19
:104010000E94C3670E94C367182F0E94C3670E9453
:10402000C367082F0E94C3670E94CD67F82E80E8FF
:104030000E94A867811141C08CEF0E94B267811174
:104040003CC089EC0E94B267811137C065E375E01E
:1040500080E090E00E942A6781E80E94A8670E94A1
:10406000C367E82E0E94C367D82E0E94C3670E94D0
:10407000C367C82F0E94CD671F92DF921F92EF92F5
:104080001F92FF921F920F931F921F931F92DF9315
:104090001F928F931F92CF938AE294E09F938F9306
:1040A0000E94E89A0E94AA678DB79EB742960FB603
:1040B000F8949EBF0FBE8DBF17C00E94AA67809163
:1040C000F02F9091F12FA091F22FB091F32F019644
:1040D000A11DB11D8093F02F9093F12FA093F22F8B
:1040E000B093F32F0E949A1F20E030E040E050E0B0
:1040F00060E070E080E090E0DF91CF911F910F9140
:10410000FF90EF90DF900895EF92FF920F931F932F
:10411000CF93DF9300D01F92CDB7DEB78C0180E83C
:104120000E94A867811154C00115110551F085EE58
:104130000E94B26781114CC061E077E980E090E0B5
:1041400009C083EE0E94B267811142C069E97AEB2F
:1041500081E090E00E942A6781E80E94A8678111AF
:1041600037C00E94C367E82E89830E94C367F82E78
:104170008A830E94CD678B830E94AA67CE01019635
:104180000E94C21F892B21F16F2D70E07E296C7F68
:1041900080E090E0012B69F00E94019120E030E086
:1041A0004AEF5AE30E94FB9220E030E040EC50E4FA
:1041B0000CC00E94019122E538EB4FE25BE30E94C4
:1041C000FB9226E636E64BE352E40E946B8F1BC05F
:1041D0000E94AA678091F02F9091F12FA091F22F69
:1041E000B091F32F0196A11DB11D8093F02F9093F4
:1041F000F12FA093F22FB093F32F0E949A1F60EF3C
:104200007FEF89E794E40F900F900F90DF91CF91AB
:104210001F910F91FF90EF9008950F931F93CF93ED
:10422000DF93729A8091620283FF08C08EE40E943D
:104230004D67811165C0C0E5D0E009C0C0E5D0E0A0
:1042400087EE93E00E942D0A2197D1F7EFCF87EEFA
:1042500093E00E942D0A2197D1F78FE40E944D67C9
:104260000E94C367D82FDF730E94C367082F0E9484
:10427000C367C82F0E94CD67182F0E94AA6780913C
:10428000620283FF72986D2F70E0762F6627600FB1
:10429000711D80E090E00E94019120E134E048EC43
:1042A0005BE30E94FB926093D2277093D3278093A5
:1042B000D4279093D5276C2F70E0762F6627610F57
:1042C000711D769567957695679580E090E00E94E0
:1042D000019124EA3CEF44E25CE30E94FB9220E07F
:1042E00030E040E252E40E946B8F6093B3347093ED
:1042F000B4348093B5349093B63480E090E002C03B
:1043000081E090E0DF91CF911F910F910895729815
:10431000729A8EE40E944D6780EA0E94B26780E044
:104320000E94B26780E00E94B2678FE40E944D67EE
:104330000E94C3678EE40E944D6780E80E94B267C6
:1043400080E00E94B26780E00E94B2670E94AA6784
:1043500080E090E008958AEC9FE09F938F930E9405
:10436000FC9A80917D020F900F90882361F01F923C
:104370008F9387EC9FE09F938F930E94FC9A0F90FE
:104380000F900F900F90089582EA9FE09F938F9374
:104390000E94FC9A8AE79FE09F938F930E94FC9A69
:1043A00083E59FE09F938F930E94FC9A88E19FE0B2
:1043B0009F938F930E94FC9A8CED9EE09F938F9326
:1043C0000E94FC9A8AEA9EE09F938F930E94FC9A37
:1043D0008EE69EE09F938F930E94FC9A88E49EE075
:1043E0009F938F930E94FC9A82E19EE09F938F930C
:1043F0000E94FC9A8091DE2B9091DF2B827091704D
:104400002DB73EB72E5E3F4F0FB6F8943EBF0FBE9E
:104410002DBF892B41F082EE9DE09F938F930E94E8
:10442000FC9A0F900F9086EB9DE09F938F930E94D4
:10443000FC9A8AE79DE09F938F930E94FC9A81E506
:104440009DE09F938F930E94FC9A85E29DE09F934D
:104450008F930E94FC9A86EF9CE09F938F930E941B
:10446000FC9A84EC9CE09F938F930E94FC9A83E9D2
:104470009CE09F938F930E94FC9A89E59CE09F9318
:104480008F930E94FC9A83E29CE09F938F930E94FB
:10449000FC9A83EF9BE09F938F930E94FC9A87EC9A
:1044A0009BE09F938F930E94FC9A88E99BE09F93E7
:1044B0008F930E94FC9A8FE59BE09F938F930E94BD
:1044C000FC9A86E29BE09F938F930E94FC9A8FEE6A
:1044D0009AE09F938F930E94FC9A81EC9AE09F93BD
:1044E0008F930E94FC9A8DB79EB780960FB6F89472
:1044F0009EBF0FBE8DBF8DE89AE09F938F930E9461
:10450000FC9A8CE59AE09F938F930E94FC9A8DE22F
:104510009AE09F938F930E94FC9A8EEF99E09F936D
:104520008F930E94FC9A87ED99E09F938F930E944E
:10453000FC9A81EA99E09F938F930E94FC9A8BE604
:1045400099E09F938F930E94FC9A85E399E09F9353
:104550008F930E94FC9A8CE099E09F938F930E9426
:10456000FC9A84ED98E09F938F930E94FC9A89EACD
:1045700098E09F938F930E94FC9A2DB73EB72A5ED6
:104580003F4F0FB6F8943EBF0FBE2DBF089589E58B
:1045900094E00C94249B4F925F926F927F928F9243
:1045A0009F92AF92BF92CF92DF92EF92FF92CF9302
:1045B000DF93CDB7DEB728970FB6F894DEBF0FBEF6
:1045C000CDBF8091E42F9091E52FA091E62FB0917F
:1045D000E72F89839A83AB83BC834090E42F50906C
:1045E000E52F6090E62F7090E72F8091E42F909157
:1045F000E52FA091E62FB091E72F8D839E83AF83A7
:10460000B8876091E42F7091E52F8091E62F90910B
:10461000E72F2CE3822E912CA12CB12CA501940123
:104620000E940E947F936F9330E1C32E3EE0D32E11
:10463000E12CF12C6D817E818F819885A7019601F7
:104640000E940E94A50194010E940E943F932F9313
:1046500040E8842E41E5942EAA24A394B12CC301F2
:10466000B201A50194010E940E94A70196010E9437
:104670000E943F932F9369817A818B819C81A50150
:1046800094010E940E943F932F9383E898E09F93A8
:104690008F930E94FC9A0FB6F894DEBF0FBECDBF79
:1046A00028960FB6F894DEBF0FBECDBFDF91CF9135
:1046B000FF90EF90DF90CF90BF90AF909F908F9042
:1046C0007F906F905F904F900895E4E7FDE38081C5
:1046D00091818234924479F0E457FD43FF93EF9344
:1046E00085E698E09F938F930E94FC9A0F900F901D
:1046F0000F900F9008953A96E53F81E4F80738F35C
:104700000895CF93DF93EC018C9A0E94A90C9F939C
:104710008F937F936F9389E598E09F938F930E9487
:10472000FC9A0F900F900F900F900F900F90209782
:1047300019F00E94BA0D08C087E598E09F938F9307
:104740000E94FC9A0F900F9081E00E945B0C2091D8
:1047500082023091830240918402509185020E942E
:10476000FB929F938F937F936F938BE498E09F933B
:104770008F930E94FC9A0F900F900F900F900F90C4
:104780000F90209719F00E94BA0D08C089E498E0B4
:104790009F938F930E94FC9A0F900F9082E00E944B
:1047A0005B0C20917E0230917F02409180025091FB
:1047B00081020E94FB929F938F937F936F938DE36F
:1047C00098E09F938F930E94FC9A0F900F900F9008
:1047D0000F900F900F90209719F00E94BA0D08C00B
:1047E0008BE398E09F938F930E94FC9A0F900F9019
:1047F00083E00E945B0C9F938F937F936F938CE277
:1048000098E09F938F930E94FC9A8C980F900F9042
:104810000F900F900F900F90209719F00E94BA0DF3
:1048200008C08AE298E09F938F930E94FC9A0F90B1
:104830000F908091DE2B87FF83C021E042E161E091
:1048400080ED0E9414699F938F937F936F938DE106
:1048500098E09F938F930E94FC9A0F900F900F9077
:104860000F900F900F90209719F00E94BA0D08C07A
:104870008BE198E09F938F930E94FC9A0F900F908A
:1048800021E042E162E080ED0E9414699F938F93E2
:104890007F936F938EE098E09F938F930E94FC9A92
:1048A0000F900F900F900F900F900F90209719F08E
:1048B0000E94BA0D08C08CE098E09F938F930E94ED
:1048C000FC9A0F900F9021E042E163E080ED0E949E
:1048D00014699F938F937F936F938FEF97E09F93CC
:1048E0008F930E94FC9A0F900F900F900F900F9053
:1048F0000F90CD2B19F00E94BA0D08C08DEF97E0F4
:104900009F938F930E94FC9A0F900F9021E042E1B9
:1049100064E080ED0E9414699F938F937F936F935F
:1049200080EF97E09F938F930E94FC9A0F900F90D7
:104930000F900F900F900F90DF91CF910C94BA0DC4
:10494000CD2BD1F3DF91CF9108950F931F93CF9388
:10495000DF93882389F049E050E06FEF70E087EA49
:1049600094E30E94369A49E050E06EE070E087EAF6
:1049700094E30E94009E13C0C7EAD4E30BEE17E055
:1049800089911F928F931F930F930E94FC9A0F900F
:104990000F900F900F9084E3CF3AD80789F7DF91FB
:1049A000CF911F910F910C94BA0D882311F0299A81
:1049B000089529980895882311F02A9A08952A982D
:1049C0000895882311F02B9A08952B980895CF927B
:1049D000DF92EF92FF92CF93DF936B017C0160FF38
:1049E00011C086E994E09F938F938FED9FE09F9392
:1049F0008F930E94FC9A0F900F900F900F9081E080
:104A000090E002C080E090E0C1FE09C0EC01219678
:104A100040EB59E06BE974E00E942012CE01C2FE27
:104A200009C0EC01219640EB59E063EA74E00E9472
:104A30002012CE01C3FE09C0EC01219640EB59E0E3
:104A40006BEA74E00E942012CE01C4FE09C0EC01A2
:104A5000219640EB59E06BE176E00E942012CE01F6
:104A6000C5FE09C0EC01219640EB59E06FEA74E005
:104A70000E942012CE01C6FE09C0EC01219640EB37
:104A800059E063EB74E00E942012CE01C7FE09C01A
:104A9000EC01219640EB59E069EB74E00E94201292
:104AA000CE01D0FE09C0EC01219640EB59E061EC4B
:104AB00074E00E942012CE01D1FE09C0EC012196C3
:104AC00040EB59E069EC74E00E942012CE01D2FE66
:104AD00009C0EC01219640EB59E06DEC74E00E94B6
:104AE0002012CE012091DE2B3091DF2B247032700A
:104AF000232B59F0D3FE09C0EC01219640EB59E07D
:104B000063ED74E00E942012CE012091DE2B23FF82
:104B10000BC0D4FE09C0EC01219640EB59E068EDD2
:104B200074E00E942012CE012091DE2B24FF0BC0E6
:104B3000D5FE09C0EC01219640EB59E06EED74E022
:104B40000E942012CE01D6FE09C0EC01219640EB56
:104B500059E066EE74E00E942012CE01D7FE09C033
:104B6000EC01219640EB59E061EF74E00E942012C5
:104B7000CE01E0FE0CC040EB59E062E075E0DF9151
:104B8000CF91FF90EF90DF90CF900C942012CD2822
:104B9000CE28CF2841F486EE97E09F938F930E9412
:104BA000FC9A0F900F90DF91CF91FF90EF90DF90E4
:104BB000CF900895CF92DF92EF92FF92CF93DF9341
:104BC000EC01C12CD12C7601209709F4A3C061EE31
:104BD00077E0CE010E94159A892B11F46894C0F8F1
:104BE00069ED77E0CE010E94159A892B11F4689443
:104BF000C1F861ED77E0CE010E94159A892B11F47E
:104C00006894C2F86DEC77E0CE010E94159A892B6A
:104C100011F46894C3F86AEC77E0CE010E94159A0B
:104C2000892B11F46894C4F866EC77E0CE010E94F9
:104C3000159A892B11F46894C5F860EC77E0CE01E1
:104C40000E94159A892B11F46894C6F868EB77E0F6
:104C5000CE010E94159A892B11F46894C7F860EB75
:104C600077E0CE010E94159A892B11F46894D0F850
:104C70006CEA77E0CE010E94159A892B11F46894B2
:104C8000D1F866EA77E0CE010E94159A892B11F4DB
:104C90006894D2F861EA77E0CE010E94159A892BD8
:104CA00011F46894D3F86BE977E0CE010E94159A6D
:104CB000892B11F46894D4F863E977E0CE010E945F
:104CC000159A892B11F46894D5F868E877E0CE013D
:104CD0000E94159A892B11F46894D6F867E777E05B
:104CE000CE010E94159A892B11F46894D7F862E7D7
:104CF00077E0CE010E94159A892B11F46894E0F8B0
:104D000060917B0270917C0280E090E00E94299A81
:104D1000EC015ACFC701B601DF91CF91FF90EF9020
:104D2000DF90CF900895AF92BF92CF92DF92EF9233
:104D3000FF920F931F93CF93DF93D22FC32F8A013C
:104D4000F62EC72ED82EE92E217030E040E050E03C
:104D500060E070E080E090E0A0E00E94499689F079
:104D600087E095E09F938F938FED9FE09F938F93C4
:104D70000E94FC9A0F900F900F900F90E1E0F0E0EE
:104D800002C0E0E0F0E08091DE2B80FF19C02D2F03
:104D9000247030E040E050E060E070E080E090E0BF
:104DA000A0E00E94499661F05F018FEFA81AB80A4F
:104DB00040EB59E06BE075E0CF010E942012F50155
:104DC0002D2F227030E040E050E060E070E080E0A5
:104DD00090E0A0E00E94499661F05F018FEFA81A71
:104DE000B80A40EB59E06FE075E0CF010E94201255
:104DF000F5012D2F287030E040E050E060E070E0D9
:104E000080E090E0A0E00E94499661F05F018FEFA2
:104E1000A81AB80A40EB59E067E275E0CF010E949A
:104E20002012F5012D2F207130E040E050E060E0CD
:104E300070E080E090E0A0E00E94499661F05F01A0
:104E40008FEFA81AB80A40EB59E062E175E0CF0194
:104E50000E942012F5012D2F207230E040E050E03A
:104E600060E070E080E090E0A0E00E94499661F090
:104E70005F018FEFA81AB80A40EB59E065E175E0D1
:104E8000CF010E942012F5012D2F207430E040E068
:104E900050E060E070E080E090E0A0E00E94499681
:104EA00061F05F018FEFA81AB80A40EB59E06BE19F
:104EB00075E0CF010E942012F5012D2F207830E0FF
:104EC00040E050E060E070E080E090E0A0E00E9410
:104ED000499661F05F018FEFA81AB80A40EB59E0DC
:104EE00061E275E0CF010E942012F50120E03C2F25
:104EF000317040E050E060E070E080E090E0A0E0E1
:104F00000E94499661F05F018FEFA81AB80A40EB42
:104F100059E064E275E0CF010E942012F50120E023
:104F20003C2F327040E050E060E070E080E090E0C4
:104F3000A0E00E94499661F05F018FEFA81AB80ABD
:104F400040EB59E069E275E0CF010E942012F501C3
:104F500020E03C2F347040E050E060E070E080E002
:104F600090E0A0E00E94499661F05F018FEFA81ADF
:104F7000B80A40EB59E060E375E0CF010E942012CF
:104F8000F50120E03C2F387040E050E060E070E038
:104F900080E090E0A0E00E94499661F05F018FEF11
:104FA000A81AB80A40EB59E063E375E0CF010E940C
:104FB0002012F50120E03C2F307140E050E060E02D
:104FC00070E080E090E0A0E00E94499661F05F010F
:104FD0008FEFA81AB80A40EB59E068E375E0CF01FB
:104FE0000E942012F50120E03C2F307240E050E09A
:104FF00060E070E080E090E0A0E00E94499661F0FF
:105000005F018FEFA81AB80A40EB59E06FE375E033
:10501000CF010E942012F50120E030E040E050E096
:105020006F2D647070E080E090E0A0E00E944996EF
:1050300061F05F018FEFA81AB80A40EB59E066E40F
:1050400075E0CF010E942012F5018091DE2B81FFD7
:1050500019C020E03C2F307440E050E060E070E088
:1050600080E090E0A0E00E94499661F05F018FEF40
:10507000A81AB80A40EB59E06AE475E0CF010E9433
:105080002012F5018091DE2B9091DF2B90FF19C04B
:1050900020E030E040E0512F507160E070E080E0AF
:1050A00090E0A0E00E94499661F05F018FEFA81A9E
:1050B000B80A40EB59E06DE475E0CF010E94201280
:1050C000F5018091DE2B9091DF2B90FF19C020E03D
:1050D00030E040E0512F507260E070E080E090E0FE
:1050E000A0E00E94499661F05F018FEFA81AB80A0C
:1050F00040EB59E060E575E0CF010E942012F50118
:105100008091DE2B9091DF2B90FF19C020E030E0E2
:1051100040E0512F507460E070E080E090E0A0E04B
:105120000E94499661F05F018FEFA81AB80A40EB20
:1051300059E066E575E0CF010E942012F50120E0FC
:105140003C2F307840E050E060E070E080E090E09C
:10515000A0E00E94499661F05F018FEFA81AB80A9B
:1051600040EB59E061E675E0CF010E942012F501A5
:1051700020E030E0402F417050E060E070E080E0DF
:1051800090E0A0E00E94499661F05F018FEFA81ABD
:10519000B80A40EB59E066E675E0CF010E942012A4
:1051A000F50120E030E0402F427050E060E070E018
:1051B00080E090E0A0E00E94499661F05F018FEFEF
:1051C000A81AB80A40EB59E069E675E0CF010E94E1
:1051D0002012F50120E030E040E050E06F2D6870D3
:1051E00070E080E090E0A0E00E94499661F05F01ED
:1051F0008FEFA81AB80A40EB59E06CE675E0CF01D2
:105200000E942012F50120E030E040E050E06F2DD8
:10521000607170E080E090E0A0E00E94499661F04B
:105220005F018FEFA81AB80A40EB59E060E775E01C
:10523000CF010E942012F5018091DE2B87FF19C05B
:1052400020E030E0402F487050E060E070E080E007
:1052500090E0A0E00E94499661F05F018FEFA81AEC
:10526000B80A40EB59E064E775E0CF010E942012D4
:10527000F5018091DE2B87FF19C020E030E0402F40
:10528000407150E060E070E080E090E0A0E00E94BB
:10529000499661F05F018FEFA81AB80A40EB59E018
:1052A00068E775E0CF010E942012F5018091DE2BA6
:1052B00087FF19C020E030E0402F407250E060E0EE
:1052C00070E080E090E0A0E00E94499661F05F010C
:1052D0008FEFA81AB80A40EB59E06CE775E0CF01F0
:1052E0000E942012F5018091DE2B87FF19C020E07B
:1052F00030E0402F407450E060E070E080E090E0EB
:10530000A0E00E94499661F05F018FEFA81AB80AE9
:1053100040EB59E060E875E0CF010E942012F501F2
:105320008091DE2B82FF19C020E030E0402F4078D2
:1053300050E060E070E080E090E0A0E00E944996DC
:1053400061F05F018FEFA81AB80A40EB59E06EEAEE
:1053500076E0CF010E942012F5018091DE2B82FFC2
:1053600019C020E030E040E0512F517060E070E063
:1053700080E090E0A0E00E94499661F05F018FEF2D
:10538000A81AB80A40EB59E064E875E0CF010E9422
:105390002012F5018091DE2B9091DF2B90FF19C038
:1053A00020E030E040E0512F527060E070E080E09B
:1053B00090E0A0E00E94499661F05F018FEFA81A8B
:1053C000B80A40EB59E067E875E0CF010E9420126F
:1053D000F5018091DE2B9091DF2B90FF19C020E02A
:1053E00030E040E0512F547060E070E080E090E0E9
:1053F000A0E00E94499661F05F018FEFA81AB80AF9
:1054000040EB59E06FE875E0CF010E942012F501F2
:105410008091DE2B9091DF2B91FF1EC020E030E0C9
:1054200040E0512F587060E070E080E090E0A0E034
:105430000E94499689F040EB59E068E975E0CF0198
:10544000DF91CF911F910F91FF90EF90DF90CF9060
:10545000BF90AF900C9420122D2F3C2FA8016F2DE0
:105460007C2D8D2D9E2DA0E00E94499641F48DE665
:1054700097E09F938F930E94FC9A0F900F90DF917B
:10548000CF911F910F91FF90EF90DF90CF90BF9041
:10549000AF900895AF92BF92DF92EF92FF920F9379
:1054A0001F93CF93DF93EC015B01FB01108268E651
:1054B00077E00E94159A892B59F58091DE2B3DE407
:1054C000F32E00E882FF03C024E8E22E02C094E03D
:1054D000E92E10E0D12C81FD00EC26E04AE250E0FC
:1054E0006BE270E089E290E00E94546481E090E019
:1054F0000E94520D882311F08DE5F82E8091DE2B4D
:105500009091DF2B90FD16E091FF07C0186005C059
:10551000F12C00E0E12C10E0D12C66E677E0CE0122
:105520000E94159A892B61F481E0F50180836091D6
:105530007B0270917C0280E090E00E94299AEC014D
:1055400064E677E0CE010E94159A892B61F48FEF13
:10555000F501808360917B0270917C0280E090E095
:105560000E94299AEC01209709F438C160E677E09F
:10557000CE010E94159A892B19F4FF2DF160FF2EA0
:105580006CE577E0CE010E94159A892B19F48F2DD6
:105590008460F82E69E577E0CE010E94159A892B88
:1055A00019F4EF2DE260FE2E67E577E0CE010E9450
:1055B000159A892B19F4FF2DF860FF2E64E577E02A
:1055C000CE010E94159A892B19F48F2D8061F82E37
:1055D0006EE477E0CE010E94159A892B19F4EF2D25
:1055E000E062FE2E68E477E0CE010E94159A892BD6
:1055F00019F4FF2DF064FF2E65E477E0CE010E94E0
:10560000159A892B19F48F2D8068F82E60E477E0C5
:10561000CE010E94159A892B09F4016069E377E0B5
:10562000CE010E94159A892B09F4026066E377E0A7
:10563000CE010E94159A892B09F4046061E377E09A
:10564000CE010E94159A892B09F408606AE277E07E
:10565000CE010E94159A892B09F4006163E277E07C
:10566000CE010E94159A892B09F400626FE177E060
:10567000CE010E94159A892B19F4ED2DE460DE2EDF
:105680006CE177E0CE010E94159A892B09F4006441
:1056900067E177E0CE010E94159A892B09F4006832
:1056A00064E177E0CE010E94159A892B19F4FE2D52
:1056B000F160EF2E61E177E0CE010E94159A892B0F
:1056C00019F48E2D8260E82E6EE077E0CE010E9404
:1056D000159A892B19F4EE2DE460EE2E6AE077E03E
:1056E000CE010E94159A892B19F4FE2DF860EF2E39
:1056F00066E077E0CE010E94159A892B19F48E2D71
:105700008061E82E62E077E0CE010E94159A892B35
:1057100019F4EE2DE062EE2E6EEF76E0CE010E94DF
:10572000159A892B19F4FE2DF064EF2E6CEF76E0BC
:10573000CE010E94159A892B19F48E2D8068E82ECF
:1057400069EF76E0CE010E94159A892B09F4116069
:1057500061EF76E0CE010E94159A892B09F4126060
:1057600068EE76E0CE010E94159A892B09F4146048
:105770006FED76E0CE010E94159A892B09F418602E
:105780006CED76E0CE010E94159A892B09F4106128
:1057900066ED76E0CE010E94159A892B09F410621D
:1057A0006BEC76E0CE010E94159A892B09F4106407
:1057B00067EC76E0CE010E94159A892B19F4ED2D45
:1057C000E860DE2E63EC76E0CE010E94159A892B0C
:1057D00009F0C0CEFD2DF061DF2EBCCE2F2D302F75
:1057E0004E2D512F6D2D70E080E090E0DF91CF9134
:1057F0001F910F91FF90EF90DF90BF90AF900895B1
:105800005F926F927F928F929F92AF92BF92CF9250
:10581000DF92EF92FF920F931F93CF93DF93782E37
:10582000C1ECDBE100E010E08DEBE82E86E0F82E25
:10583000872D8170582E872D8270682E98EAC92E88
:1058400096E0D92E20EBA22E26E0B22E3EEA832E41
:1058500036E0932E772051F01F930F93FF92EF9233
:105860000E94FC9A0F900F900F900F905520A1F07E
:1058700089858F9388858F93BF92AF920E94FC9AFF
:105880000F900F900F900F906620C1F09F928F9213
:105890000E94FC9A0F900F90662081F0DF92CF92C9
:1058A0000E94FC9A288139814A815B816C817D81CB
:1058B0008E819F810E9493260F900F900E94BA0DB7
:1058C0000F5F1F4F2A960430110521F6DF91CF910B
:1058D0001F910F91FF90EF90DF90CF90BF90AF900E
:1058E0009F908F907F906F905F90089583EA96E0ED
:1058F0009F938F930E94FC9A8091CE279091CF27FF
:10590000A091D027B091D1270F900F90813027EA36
:1059100092072EE1A207B10519F485E996E01DC0B2
:10592000823026EA92072EE1A207B10519F488E831
:1059300096E013C0823027EA92072EE1A207B10554
:1059400019F48AE796E009C0823028EA92072EE12E
:10595000A207B10549F48CE696E09F938F930E94CD
:10596000FC9A0F900F900895BF93AF939F938F93DE
:1059700086E696E09F938F930E94FC9A0F900F907B
:105980000F900F900F900F90089586E596E09F93EB
:105990008F930E94FC9A0E94C7220E94762C0E943C
:1059A000BA0D88EA9BE19F938F938EE496E09F93D4
:1059B0008F930E94FC9A60915C0270915D028091CD
:1059C0005E0290915F0228EE33E040E050E00E94DA
:1059D0000E945F934F933F932F938EE396E09F93A4
:1059E0008F930E94FC9A85E396E09F938F930E9489
:1059F000FC9A0E9448128091DE2B2DB73EB7225FA1
:105A00003F4F0FB6F8943EBF0FBE2DBF80FF05C0BD
:105A100041E061E081E00E94F51381E396E09F930D
:105A20008F930E94FC9A80E00E94A5240E94CB22C2
:105A3000809161021F928F9388E296E09F938F93EB
:105A40000E94FC9A8091510A1F928F938FE196E0F9
:105A50009F938F930E94FC9A80918D028F938091E7
:105A60008C028F9380918B028F9380918A028F9307
:105A700081E196E09F938F930E94FC9A1F9280E4AD
:105A80008F9389EF95E09F938F930E94FC9A80916A
:105A9000B8341F928F938091B7341F928F9386EE04
:105AA00095E09F938F930E94FC9A809160021F92D1
:105AB0008F938DED95E09F938F930E94FC9A809138
:105AC000620290916302A0916402B09165022DB7C9
:105AD0003EB7225E3F4F0FB6F8943EBF0FBE2DBFBC
:105AE00096FD03C084EA95E002C081EA95E09F93A9
:105AF0008F9383ED95E09F938F930E94FC9A83E0B0
:105B00000E94002C0F900F900F900F901D9903C0D2
:105B100084EA95E002C081EA95E09F938F9387EC39
:105B200095E09F938F930E94FC9A8DEB95E09F9355
:105B30008F930E94FC9A809162020F900F900F90B9
:105B40000F900F900F9081FF09C087EB95E09F9316
:105B50008F930E94FC9A0F900F9013C080FD03C09A
:105B600084EA95E002C081EA95E09F938F9383EBEE
:105B700095E09F938F930E94FC9A0F900F900F9047
:105B80000F908091620290916302A0916402B091A3
:105B9000650297FD03C084EA95E002C081EA95E0C2
:105BA0009F938F938AEA95E09F938F930E94FC9A2C
:105BB00083EA95E09F938F930E94FC9A6091550A27
:105BC0007091560A8091570A9091580A0E94E724D2
:105BD0000E94BA0D0F900F900F900F900F900F90A2
:105BE000779B03C084EA95E002C081EA95E09F9329
:105BF0008F938AE995E09F938F930E94FC9A0E946D
:105C0000330A0E940E0D9F938F937F936F938CE8BE
:105C100095E09F938F930E94FC9A0E94BD0C9F93E6
:105C20008F937F936F938EE795E09F938F930E945E
:105C3000FC9A81E090E00E94812380918D349091C4
:105C40008E34A0918F34B0919034BF93AF939F93D3
:105C50008F9380E795E09F938F930E94FC9A8091A9
:105C6000A2348F938091A1348F938091A0348F932D
:105C700080919F348F938CE595E09F938F930E9442
:105C8000FC9A8091913490919234A0919334B09188
:105C90009434BF93AF939F938F938EE495E09F933B
:105CA0008F930E94FC9A8DB79EB782960FB6F89498
:105CB0009EBF0FBE8DBF8091A6348F938091A53477
:105CC0008F938091A4348F938091A3348F938AE330
:105CD00095E09F938F930E94FC9A61E070E080E0D2
:105CE00090E00E94C30D61E070E081E090E00E94CE
:105CF000C30D0F900F900F900F900F900F90299958
:105D000003C084EA95E002C081EA95E09F938F93F7
:105D100082E395E09F938F930E94FC9A0F900F90DF
:105D20000F900F902A9903C084EA95E002C081EA9F
:105D300095E09F938F938AE295E09F938F930E94C3
:105D4000FC9A0F900F900F900F900895F89491E2A5
:105D5000E0E0F0E0909357008491E2E0F0E090936F
:105D600057002491E4E0F0E090935700E49190E034
:105D7000A0E0B0E0BC0155274427822F90E0A0E0CE
:105D8000B0E0BA2FA92F982F8827840F951FA61F40
:105D9000B71F8E0F911DA11DB11D8093CE2790932B
:105DA000CF27A093D027B093D12778940895CF938D
:105DB000DF93CDB7DEB761970FB6F894DEBF0FBEA5
:105DC000CDBF48E250E062E270E081EC9BE10E94CE
:105DD000E29D2091C11B3091C21B4091C31B509189
:105DE000C41B6091C51B7091C61B8091C71B90910D
:105DF000C81BAFEF0E94499609F05DC08DE4809307
:105E0000C11B80E88093C21B84E08093C31B109267
:105E1000C41B1092C51B1092C61B1092C71B109278
:105E2000C81B8CE390E09093CA1B8093C91B10920F
:105E3000CB1B1092CC1B1092CD1B1092CE1B10923C
:105E4000CF1B1092D01B1092D11B1092D21B10921C
:105E5000D41B1092D31B1092D51B1092D61B1092FC
:105E6000D71B1092D81B1092D91B1092DA1B1092DC
:105E7000DB1B1092DC1B1092DE1B1092DD1B1092BC
:105E8000DF1B1092E01B1092E11B1092E21B10929C
:105E9000E31B1092E41B1092E51B1092E61B10927C
:105EA000E81B1092E71B48E250E062E270E081ECF0
:105EB0009BE10E94009E44E050E06EE170E0CE0164
:105EC0000B960E94E29D8B859C85AD85BE858F3F9C
:105ED0002FEF9207A207B207A9F48AE090E4A0E0AE
:105EE000B0E08093620290936302A0936402B09347
:105EF000650244E050E06EE170E082E692E00E94CC
:105F0000009E08C08093620290936302A093640293
:105F1000B09365028091620290916302A091640245
:105F2000B0916502A2FF02C02A9A03C080E00E94DD
:105F3000DB2444E050E06AE570E0CE010B960E945D
:105F4000E29D8B859C85AD85BE858F3F2FEF9207A7
:105F5000A207B20789F41092550A1092560A1092BD
:105F6000570A1092580A44E050E06AE570E085E56F
:105F70009AE00E94009E08C08093550A9093560AAA
:105F8000A093570AB093580A49E050E06EE070E0E1
:105F900087EA94E30E94E29D0E94F10E44E050E003
:105FA0006EE470E0CE010B960E94E29D8B859C858D
:105FB000AD85BE8544E050E06EE470E08F3F9F4FBA
:105FC000AF4FBF4F29F482E892E00E94009E04C0C8
:105FD00082E892E00E94E29D44E050E06AE470E0D2
:105FE000CE010B960E94E29D8B859C85AD85BE857A
:105FF00044E050E06AE470E08F3F9F4FAF4FBF4FE7
:1060000029F48EE792E00E94009E04C08EE792E0A1
:106010000E94E29D44E050E062E570E0CE010B9604
:106020000E94E29D8B859C85AD85BE8544E050E055
:1060300062E570E08F3F9F4FAF4FBF4F29F486E876
:1060400092E00E94009E04C086E892E00E94E29DD9
:1060500041E050E06DE170E0CE0141960E94E29D8A
:10606000898941E050E06DE170E08F3F29F481E5DE
:106070009AE00E94009E04C081E59AE00E94E29DA1
:1060800041E050E06CE170E0CE0141960E94E29D5B
:10609000898941E050E06CE170E08F3F29F481E6AE
:1060A00092E00E94009E04C081E692E00E94E29D80
:1060B00041E050E06BE170E0CE0141960E94E29D2C
:1060C000898941E050E06BE170E08F3F29F480E680
:1060D00092E00E94009E04C080E692E00E94E29D51
:1060E0004AE050E064E070E0CE0101960E94E29D3B
:1060F00089814AE050E064E070E08F3F29F488EA4B
:106100009BE10E94009E04C088EA9BE10E94E29D00
:1061100044E050E066E570E0CE010B960E94E29DFF
:106120008B859C85AD85BE8544E050E066E570E0DA
:106130008F3F9F4FAF4FBF4F29F48AE892E00E94F4
:10614000009E04C08AE892E00E94E29D44E050E094
:1061500067E170E0CE010B960E94E29D8B859C85E5
:10616000AD85BE8544E050E067E170E08F3F9F4F12
:10617000AF4FBF4F29F48CE592E00E94009E04C00F
:106180008CE592E00E94E29D42E050E062E070E027
:10619000CE010F960E94E29D8F85988942E050E0E3
:1061A00062E070E08F3F910529F48CE49AE00E9450
:1061B000009E04C08CE49AE00E94E29D42E050E020
:1061C00060E070E0CE010F960E94E29D8F85988975
:1061D00042E050E060E070E08F3F910529F48AE4EE
:1061E0009AE00E94009E04C08AE49AE00E94E29D28
:1061F00061960FB6F894DEBF0FBECDBFDF91CF9191
:106200000895CF92DF92EF92FF9260917B0270919E
:106210007C0280E090E00E94299A68EA75E00E9482
:106220003D9A892B09F03BC18DE48093C11B80E826
:106230008093C21B84E08093C31B1092C41B1092F6
:10624000C51B1092C61B1092C71B1092C81B8CE373
:1062500090E09093CA1B8093C91B1092CB1B1092A5
:10626000CC1B1092CD1B1092CE1B1092CF1B109204
:10627000D01B1092D11B1092D21B1092D41B1092E3
:10628000D31B1092D51B1092D61B1092D71B1092C5
:10629000D81B1092D91B1092DA1B1092DB1B1092A4
:1062A000DC1B1092DE1B1092DD1B1092DF1B109284
:1062B000E01B1092E11B1092E21B1092E31B109264
:1062C000E41B1092E51B1092E61B1092E81B109243
:1062D000E71B48E250E062E270E081EC9BE10E9443
:1062E000009E8AE090E4A0E0B0E080936202909388
:1062F0006302A0936402B093650244E050E06EE153
:1063000070E082E692E00E94009E1092550A109280
:10631000560A1092570A1092580A44E050E06AE573
:1063200070E085E59AE00E94009E82E2C82EDD249E
:10633000DA948CECE82E8BE3F82EC0928202D09295
:106340008302E0928402F092850244E050E06EE421
:1063500070E082E892E00E94009EC0927E02D0929D
:106360007F02E0928002F092810244E050E06AE411
:1063700070E08EE792E00E94009E87ED94E3AFEE1E
:10638000BCE38093860290938702A0938802B09327
:10639000890244E050E062E570E086E892E00E9405
:1063A000009E8AE999E9A9E1B0E480938A0290937A
:1063B0008B02A0938C02B0938D0244E050E066E51E
:1063C00070E08AE892E00E94009E1092510A80E0FC
:1063D0000E94167241E050E06DE170E081E59AE0C4
:1063E0000E94009E8AE1809361020E94BE7041E09B
:1063F00050E06CE170E081E692E00E94009E8FE048
:106400008093600241E050E06BE170E080E692E052
:106410000E94009E8AE0E8EAFBE1DF011D928A9576
:10642000E9F74AE050E064E070E0CF010E94009E8E
:1064300080EA96E8A1E0B0E080935C0290935D0270
:10644000A0935E02B0935F0244E050E067E170E029
:106450008CE592E00E94009E10924D0A10924C0A28
:1064600042E050E062E070E08CE49AE00E94009E1E
:1064700010924B0A10924A0A42E050E060E070E04D
:106480008AE49AE00E94009E81E00E94A52480E0B8
:1064900090E0FF90EF90DF90CF900C94050FFF906D
:1064A000EF90DF90CF9008950E94146E6C9A6B9AD3
:1064B0006A9A6F9A729A749A739A779A809880B34C
:1064C000897F80BB8398849887E080937E00549A6C
:1064D0000E94A62E0E94D72E0E94A10A80E090E082
:1064E0000E94050F60915C0270915D0280915E02D6
:1064F00090915F020E9437670E94BD0C6093E02F6D
:106500007093E12F8093E22F9093E32F80916202AA
:1065100086FD239A219A229A239A0E94B60A1D9BED
:1065200005C01092530A1092520A089581E090E03B
:106530009093530A8093520A0895CF93DF9390E08B
:106540004091550A5091560A6091570A7091580A25
:1065500041FD08C02091620220FD04C021FF8CC0D3
:106560001D9B8AC02DE8289FE001299FD00D112492
:10657000CE018253934E9F938F938FEA95E09F9322
:106580008F930E94E89AFE01E953F34EDF01AA5768
:10659000BF4F2C910F900F900F900F90438154811B
:1065A000658176818091E42F9091E52FA091E62F6F
:1065B000B091E72F841B950BA60BB70B2223D1F1CB
:1065C000BF93AF939F938F93DF01A257BF4F119655
:1065D0008C9111978F938C918F93129711968C9128
:1065E00011978F938C918F9313978C911F928F9308
:1065F00011978C911F928F9313968C911F928F936A
:1066000011978C911F928F93E957FF4F80811F92B2
:106610008F931F922F9385EB95E09F938F930E940A
:10662000E89A8DB79EB746960FB6F8949EBF0FBEF8
:106630008DBF10C0BF93AF939F938F938CEF95E066
:106640009F938F930E94E89A0F900F900F900F9056
:106650000F900F900E94BA0D80917D02882361F007
:106660001F928F9383EE91E09F938F930E94FC9AE9
:106670000F900F900F900F90DF91CF910895809120
:10668000C71C882341F08091C81C90E00E949D3275
:106690000E94A70BF4CF0895CF93DF93EC0188817C
:1066A0009981883E2EE09207E9F018F4892BB9F021
:1066B00048C0803F2EE0920709F449C0843F9E40C5
:1066C00009F03FC087E69AE00E94A35E892BE9F1BA
:1066D00087E69AE00E94865E80E00E94D52488EEDC
:1066E0009EE02CC0623189F5299A60914A0A709126
:1066F0004B0A7695762F66277795679587E69AE019
:106700000E947C5E8091550A9091560AA091570A8A
:10671000B091580AA0FF10C080914B0A8F938091CE
:106720004A0A8F9384E890E19F938F930E94FC9A8A
:106730000F900F900F900F9080EF9EE099838883C9
:1067400004C01982188283E017C081E015C087E673
:106750009AE00E94A35E892BC1F387E69AE00E942B
:10676000865E0E943F3360E270E087E69AE00E9416
:106770007C5E84EF9EE0E2CFDF91CF9108952F926F
:106780003F924F925F926F927F928F929F92AF92C1
:10679000BF92CF92DF92EF92FF920F931F93CF930E
:1067A000DF93CDB7DEB72B970FB6F894DEBF0FBEE1
:1067B000CDBF9B878A873A01FC0180819181892B1B
:1067C00011F00C94F94760917B0270917C02CA0130
:1067D0000E94299A60E870E0C3010E945C9A0097C9
:1067E00059F460916E3D70916F3D8AE090E00E9497
:1067F000B09A81E00C94FE478130910561F4F30179
:106800001081912E990C9908892C092D292C392C4D
:10681000492C592CB9C082309105B9F4F30180811B
:10682000082E000C990B982F88272181820F911D2B
:1068300027FD9A95182F992E892E880C8808082DE7
:10684000282C382C482C582C9FC083309105B1F54A
:10685000F3012081922F990F990B392F492F592F2E
:10686000692F792F892F00E10E94EB9519012A01E8
:106870004B01B82FA92F2181922F990F990B392FF6
:10688000492F592F692F792F892F08E00E94EB9506
:1068900059016A017B018C019101A201B4018B2F86
:1068A0009A2F0E942296A2801A2D110F110BB12E41
:1068B000C12ED12EE12EF12E012F55C004970CF4DC
:1068C0005BC0F3012081922F990F990B392F492F2B
:1068D000592F692F792F892F08E10E94EB95190113
:1068E0002A014B01B82FA92F2181922F990F990BC3
:1068F000392F492F592F692F792F892F00E10E94B5
:10690000EB9559016A017B018C019101A201B4014F
:106910008B2F9A2F0E942296A3801A2D110F110BF4
:10692000B12EC12ED12EE12EF12E012F0E942296E2
:1069300019012A014B01B82FA92F2281922F990FFB
:10694000990B392F492F592F692F792F892F08E05B
:106950000E94EB9559016A017B018C019101A20112
:10696000B4018B2F9A2F0E942296122F932E842EE1
:10697000052F1B012C0108C01AE0912C812C00E08E
:10698000212C312C412C512C0E94BA0D212F392D54
:10699000482D502FB101C2012537F3E63F07FDE630
:1069A0004F075105610571058105910511F40C949E
:1069B000DE422537E3E63E07EDE64E075105610569
:1069C00071058105910511F008F0B2C12337F2E796
:1069D0003F0741055105610571058105910511F4D8
:1069E0000C9477452337E2E73E07410551056105E1
:1069F00071058105910511F008F0B9C02536F4E65E
:106A00003F0741055105610571058105910509F4AF
:106A1000DBC72536E4E63E074105510561057105F2
:106A20008105910511F008F041C0A6E70E94499642
:106A300011F40C94663F0E94499609F070F4A8E6A0
:106A40000E94499611F40C94353DA5E70E944996A1
:106A500011F40C94503F0C94F747212F392D482DF9
:106A6000502FB101C2012436F1E63F07410551051F
:106A7000610571058105910511F40C949F45253739
:106A8000E2E63E0741055105610571058105910565
:106A900009F431C52A3336424105510561057105B6
:106AA0008105910509F430C30C94F747212F392D46
:106AB000482D502FB101C2012737EFE63E074105AF
:106AC0005105610571058105910511F40C9444434C
:106AD0002737FFE63F07410551056105710581052F
:106AE000910509F0C8F42436E9E63E074105510551
:106AF000610571058105910511F40C94293F253636
:106B00003E4641055105610571058105910511F468
:106B10000C9478430C94F747212F392D482D502F92
:106B2000B101C2012536E2E73E0741055105610585
:106B300071058105910511F40C9444442936F2E75E
:106B40003F0741055105610571058105910511F466
:106B50000C942645233331474105510561057105E4
:106B60008105910511F00C94F7470C949F45212F56
:106B7000392D482D502FB101C2012236F5E63F07CD
:106B8000F4E64F075105610571058105910509F48A
:106B90001BC72236E5E63E07E4E64E0751056105D0
:106BA00071058105910511F008F05BC02133F4E611
:106BB0003F07F1E64F075105610571058105910514
:106BC00009F4B6C22133E4E63E07E1E64E0751057B
:106BD000610571058105910509F0C0F42337F3E7DC
:106BE0003F0741055105610571058105910511F4C6
:106BF0000C948B45283734474105510561057105D3
:106C00008105910509F480C20C94F747212F392D95
:106C1000482D502FB101C2012837F4E63F07F1E6B5
:106C20004F075105610571058105910509F47CC285
:106C30002C36E5E73E07E2E64E0751056105710592
:106C40008105910509F457C4233634464146510560
:106C5000610571058105910511F00C94F7470C94BD
:106C60009F45212F392D482D502FB101C2012D36BE
:106C7000E5E73E07E8E64E07510561057105810528
:106C8000910511F40C94B5452D36F5E73F07F8E66C
:106C90004F075105610571058105910509F0E0F483
:106CA0002237E2E73E07E5E64E075105610571052B
:106CB0008105910511F40C948F4223363D464846D8
:106CC0005105610571058105910511F00C94F74797
:106CD0000E9452180C94F947212F392D482D502F1E
:106CE000B101C2012436E3E63E07ECE64E0751054A
:106CF000610571058105910511F40C94F241273667
:106D0000FFE63F07FCE64F07510561057105810568
:106D1000910511F40C94F54123363243494651054F
:106D2000610571058105910511F00C94F74720C2AA
:106D3000212F392D482D502FB101C2012037FCE6FB
:106D40003F07F5E64F07F8E65F0761057105810526
:106D5000910509F48AC62037ECE63E07E5E64E07C2
:106D6000E8E65E07610571058105910511F008F0FF
:106D7000E0C02437F8E73F07F4E74F075105610506
:106D800071058105910511F40C94D23F2437E8E791
:106D90003E07E4E74E075105610571058105910540
:106DA00011F008F05DC02033F1E33F07F1E74F0732
:106DB0005105610571058105910511F40C948F420F
:106DC0002033E1E33E07E1E74E0751056105710518
:106DD0008105910509F0C0F42133F2E63F07F0E7A1
:106DE0004F075105610571058105910509F498C2A8
:106DF00022333246404751056105710581059105F1
:106E000009F4E3C20C94F747212F392D482D502F58
:106E1000B101C2012037F5E63F07F2E74F07510500
:106E2000610571058105910511F40C9444442C36DB
:106E3000E4E73E074E07510561057105810591059F
:106E400011F40C941D47213331434147510561052D
:106E500071058105910511F00C94F7470C94DE4201
:106E6000212F392D482D502FB101C2012B36ECE6D0
:106E70003E07E5E74E07E2E65E076105710581051D
:106E8000910509F438C32B36FCE63F07F5E74F07B9
:106E9000F2E65F07610571058105910509F0E0F4EF
:106EA0002437E4E63E07E7E74E0751056105710523
:106EB0008105910511F40C946B4724373F464F46EA
:106EC0005246610571058105910511F00C94F74753
:106ED0000C9400000C94F947212F392D482D502F88
:106EE000B101C2012E36E1E63E07E8E64E07E3E6D1
:106EF0005E07610571058105910511F40C94A63FAB
:106F00002633F9E63F07F5E74F07F5E65F0761052A
:106F100071058105910509F4ACC529363C46414609
:106F20005346610571058105910511F00C94F747F1
:106F300089C3212F392D482D502FB101C20124378B
:106F4000F3E73F07F5E64F07F2E75F0761057105D5
:106F50008105910511F40C94F4432437E3E73E07CF
:106F6000E5E64E07E2E75E076105710581059105DB
:106F700011F008F062C02337F5E63F07F2E74F074C
:106F8000F0E75F07610571058105910511F40C9427
:106F900065462337E5E63E07E2E74E07E0E75E0792
:106FA000610571058105910509F0D0F42136FDE6F2
:106FB0003F07F5E74F07F8E65F07610571058105B3
:106FC000910511F40C9462432237374740475047EC
:106FD000610571058105910509F45CC20C94F747C0
:106FE000212F392D482D502FB101C2012436FDE645
:106FF0003F07F3E64F07F2E75F076105710581057B
:10700000910509F441C62136ECE63E07E5E64E0758
:10701000E2E75E07610571058105910509F446C542
:107020002337324747475047610571058105910570
:1070300011F00C94F7470C94F743212F392D482D6C
:10704000502FB101C2012437E2E73E07E1E64E07C7
:10705000E5E75E07610571058105910509F46FC6D5
:107060002437F2E73F07F1E64F07F5E75F076105D1
:1070700071058105910509F0C8F42437E3E73E075F
:10708000E5E64E07E4E75E076105710581059105B8
:1070900009F4B3C72737304748475447610571059E
:1070A0008105910509F428C70C94F747212F392D44
:1070B000482D502FB101C2012F36ECE63E07EFE517
:1070C0004E07E6E75E07610571058105910509F444
:1070D00086C52C36F1E63F07F4E74F07F8E75F0770
:1070E000610571058105910511F40C94E74622377D
:1070F000374640475547610571058105910511F0F7
:107100000C94F7470C94CE4183E080939534109211
:1071100097341092963445E954E362E18EE392E0AD
:107120000E94F75B0C94F9470E94DA170C94F94718
:1071300021E042E161E080ED0E94146921E042E13A
:1071400061E080ED0E94146921E042E161E080EDA0
:107150000E94146921E042E161E080ED0E9414691F
:1071600021E042E161E080ED0E9414690C94F9474E
:1071700060917B0270917C0280E090E00E94299AED
:1071800068E076E00E943D9A892B09F0C5C06091C5
:107190007B0270917C0280E090E00E94299A8C0131
:1071A000009709F497C06CEE73E00E943D9A892B1A
:1071B000E1F488EE93E0A0E0B0E080935C0290936D
:1071C0005D02A0935E02B0935F0268EE73E080E020
:1071D00090E00E94376744E050E067E170E08CE5A2
:1071E00092E00E94009E0C94F9476EE076E0C801A0
:1071F0000E943D9A892BE1F480E197E2A0E0B0E0A3
:1072000080935C0290935D02A0935E02B0935F0254
:1072100060E177E280E090E00E94376744E050E070
:1072200067E170E08CE592E00E94009E0C94F947C3
:1072300061E176E0C8010E943D9A892BE1F480EA81
:1072400096E8A1E0B0E080935C0290935D02A09389
:107250005E02B0935F0260EA76E881E090E00E940F
:10726000376744E050E067E170E08CE592E00E940F
:10727000009E0C94F94765E176E0C8010E943D9AB2
:10728000892BE1F480E89AE1A6E0B0E080935C020B
:1072900090935D02A0935E02B0935F0260E87AE192
:1072A00086E090E00E94376744E050E067E170E0DC
:1072B0008CE592E00E94009E0C94F94782E693E0F0
:1072C0009F938F930E94FC9A0E94BA0D0F900F908B
:1072D0000C94F94760915C0270915D0280915E02AE
:1072E00090915F0228EE33E040E050E00E940E945F
:1072F0005F934F933F932F938EE593E09F938F93EC
:107300000E94FC9A0E94BA0D0F900F900F900F9060
:107310000F900F900C94F9470E9448120C94F94773
:1073200060917B0270917C0280E090E00E94299A3B
:107330008C0161EA75E00E943D9A892BA1F480914D
:10734000620290916302A0916402B0916502A26012
:107350008093620290936302A0936402B0936502EB
:10736000299A0C94F94764EA75E0C8010E943D9A95
:10737000892BB1F48091620290916302A091640222
:10738000B0916502AD7F8093620290936302A093F7
:107390006402B093650280E00E94D5240C94F94702
:1073A000299903C084EA95E002C081EA95E09F93A1
:1073B0008F9386E593E09F938F930E94FC9A0F90A2
:1073C0000F900F900F900C94F94760917B02709191
:1073D0007C0280E090E00E94299A8C0161EA75E0CD
:1073E0000E943D9A892BE1F48091620290916302A0
:1073F000A0916402B0916502A460809362029093B0
:107400006302A0936402B09365022A9A44E050E0BC
:107410006EE170E082E692E00E94009E0C94F947D3
:1074200064EA75E0C8010E943D9A892BF1F48091CD
:10743000620290916302A0916402B0916502AB7FF9
:107440008093620290936302A0936402B0936502FA
:1074500080E00E94DB2444E050E06EE170E082E6D0
:1074600092E00E94009E0C94F9472A9903C084EA96
:1074700095E002C081EA95E09F938F938EE493E0BC
:107480009F938F930E94FC9A0F900F900F900F90F4
:107490000C94F94760917B0270917C0280E090E04F
:1074A0000E94299A8C0161EA75E00E943D9A892B1D
:1074B00019F477980C94F94764EA75E0C8010E94C2
:1074C0003D9A892B19F4779A0C94F947779B03C05E
:1074D00084EA95E002C081EA95E09F938F9384E16E
:1074E00095E09F938F930E94FC9A0F900F900F90BE
:1074F0000F900C94F94760917B0270917C0280E0C0
:1075000090E00E94299A8C0169E176E00E943D9A00
:10751000892BD1F48091C71C1F928F938091C91C35
:107520001F928F938091C81C1F928F931F9284E1AA
:107530008F9384E293E09F938F930E94FC9A0FB6FF
:10754000F894DEBF0FBECDBF6EE176E0C8010E94A9
:107550003D9A892B19F40E943F3370C066E276E0B1
:10756000C8010E943D9A892B09F047C060917B02B7
:1075700070917C0280E090E00E94299A009709F4C3
:107580005DC00E9416998531910570F590934D0A62
:1075900080934C0A42E050E062E070E08CE49AE0B4
:1075A0000E94009E60917B0270917C0280E090E0DE
:1075B0000E94299A009709F441C00E94169990935D
:1075C0004B0A80934A0A42E050E060E070E08AE4AF
:1075D0009AE00E94009E60917B0270917C0280E0A4
:1075E00090E00E94299A2AC082E193E09F938F93B2
:1075F0000E94FC9A0F900F9021C080914D0A8F93AA
:1076000080914C0A8F9389E093E09F938F930E941F
:10761000FC9A0E94BA0D80914B0A8F9380914A0A7E
:107620008F938AEF92E09F938F930E94FC9A0E941F
:10763000BA0D0FB6F894DEBF0FBECDBF0E94BA0DD3
:107640000C94F94760917B0270917C0280E090E09D
:107650000E94299A8C0166E675E00E943D9A892B6A
:1076600009F077C060917B0270917C0280E090E02D
:107670000E94299A8C01009711F40C94F94764E256
:1076800076E00E943D9A892BB1F482E29FEFACEC48
:10769000BBE38093820290938302A0938402B09311
:1076A000850244E050E06EE470E082E892E00E94DF
:1076B000009E0C94F9476AE276E0C8010E943D9A68
:1076C000892BB1F482E29FEFACECBAE380938202A3
:1076D00090938302A0938402B093850244E050E02B
:1076E0006EE470E082E892E00E94009E0C94F947FC
:1076F000C8010E9412992B013C0120E030E0A90151
:107700000E944A908823D9F081E00E945B0C9B0183
:10771000AC01C301B2010E944F906093820270934A
:107720008302809384029093850244E050E06EE4EB
:1077300070E082E892E00E94009E0C94F9478DEE82
:1077400092E09F938F930E94FC9A0F900F900C945D
:10775000F94769E675E0C8010E943D9A892B09F056
:1077600077C060917B0270917C0280E090E00E9483
:10777000299A8C01009711F40C94F94764E276E0A1
:107780000E943D9A892BB1F482E29FEFACECBBE3FF
:1077900080937E0290937F02A0938002B093810237
:1077A00044E050E06AE470E08EE792E00E94009EC0
:1077B0000C94F9476AE276E0C8010E943D9A892B51
:1077C000B1F482E29FEFACECBAE380937E02909337
:1077D0007F02A0938002B093810244E050E06AE40B
:1077E00070E08EE792E00E94009E0C94F947C80179
:1077F0000E9412992B013C0120E030E0A9010E9477
:107800004A908823D9F082E00E945B0C9B01AC0176
:10781000C301B2010E944F9060937E0270937F0279
:10782000809380029093810244E050E06AE470E02B
:107830008EE792E00E94009E0C94F94780EE92E061
:107840009F938F930E94FC9A0F900F900C94F9478E
:1078500061E675E0C8010E943D9A892B09F073C06A
:1078600060917B0270917C0280E090E00E94299AF6
:107870008C01009711F40C94F94764E276E00E94C1
:107880003D9A892BB1F487ED94E3AFEEBCE380938E
:10789000860290938702A0938802B093890244E005
:1078A00050E062E570E086E892E00E94009E0C9451
:1078B000F9476AE276E0C8010E943D9A892B51F4AB
:1078C00081ED92E09F938F930E94FC9A0F900F900E
:1078D0000C94F947C8010E9412992B013C0120E049
:1078E00030E0A9010E944A90882319F180E00E94AB
:1078F0005B0C4B015C0121EE3AE744E95EE3C30116
:10790000B2010E946B8FA50194010E944F90609379
:10791000860270938702809388029093890244E0E4
:1079200050E062E570E086E892E00E94009E0C94D0
:10793000F94784EC92E09F938F930E94FC9A0F90FA
:107940000F900C94F9470E94A90C9F938F937F93FB
:107950006F938DEB92E09F938F930E94FC9A82E04D
:107960000E945B0C20917E0230917F024091800248
:10797000509181020E94FB92162F072FF82EE92EBC
:1079800081E00E945B0CEF92FF920F931F93209176
:1079900082023091830240918402509185020E94BC
:1079A000FB929F938F937F936F9381EB92E09F93D2
:1079B0008F930E94FC9A0E94BA0D0FB6F894DEBF16
:1079C0000FBECDBF0C94F94760917B0270917C0291
:1079D00080E090E00E94299A009711F10E94DA2538
:1079E0000091550A1091560A2091570A3091580A71
:1079F000601771078207930739F16093550A7093F6
:107A0000560A8093570A9093580A44E050E06AE57A
:107A100070E085E59AE00E94009E8DE095E002C04E
:107A200086E095E09F938F930E94FC9A6091550A9F
:107A30007091560A8091570A9091580A0E94E72443
:107A40000E94BA0D0F900F908BEF94E09F938F934D
:107A50000E94FC9A6FEF7FEFCB010E94E7240E9407
:107A6000BA0D0F900F900C94F9470E94C4210C940A
:107A7000F947F3018481843329F440E061E080E038
:107A80000E94F51380917D02882311F40C94F9472C
:107A90001F928F9388EF94E09F938F930E94FC9A9C
:107AA0000F900F900F900F900C94F947F301848181
:107AB000893709F080C060917B0270917C0280E080
:107AC00090E00E94299A8C0161EA75E00E943D9A3B
:107AD000892B51F48091620290916302A09164021B
:107AE000B0916502906410C064EA75E0C8010E941C
:107AF0003D9A892BD1F48091620290916302A0910A
:107B00006402B09165029F7B80936202909363024E
:107B1000A0936402B093650244E050E06EE170E02F
:107B200082E692E00E94009E46C06FE276E0C801C5
:107B30000E943D9A892B21F58091C01B8F938091E3
:107B4000BF1B8F938091BE1B8F938091BD1B8F9322
:107B50008091BC1B8F938091BB1B8F938091BA1B2C
:107B60008F938091B91B8F9386E892E09F938F93B8
:107B70000E94FC9A0FB6F894DEBF0FBECDBF1BC0AB
:107B80008091620290916302A0916402B0916502BB
:107B900096FD03C084EA95E002C081EA95E09F93D8
:107BA0008F9382E892E09F938F930E94FC9A0F90AC
:107BB0000F900F900F9080917D02882311F40C9408
:107BC000F9471F928F9385EF94E09F938F930E94C4
:107BD000FC9A0F900F900F900F900C94F947F301BF
:107BE00084818737E9F560917B0270917C0280E0A7
:107BF00090E00E94299A0097D9F00E9412992B01D7
:107C00003C0120E030E0A9010E944A90882381F0E5
:107C100040928A0250928B0260928C0270928D0286
:107C200044E050E066E570E08AE892E00E94009E41
:107C300080918D028F9380918C028F9380918B0223
:107C40008F9380918A028F9384E792E09F938F9322
:107C50000E94FC9A0F900F900F900F900F900F9032
:107C600080917D02882311F40C94F9471F928F9321
:107C700082EF94E09F938F930E94FC9A0F900F9055
:107C80000F900F900C94F94760917B0270917C02E9
:107C900080E090E00E94299A8C0161EA75E00E94E0
:107CA0003D9A40906202509063026090640270902E
:107CB0006502892B19F4689457F809C064EA75E0E5
:107CC000C8010E943D9A892B99F4E89457F8409294
:107CD000620250926302609264027092650244E014
:107CE00050E06EE170E082E692E00E94009E13C0D8
:107CF00057FC03C084EA95E002C081EA95E09F93B7
:107D00008F9380E792E09F938F930E94FC9A0F904D
:107D10000F900F900F9080917D02882311F40C94A6
:107D2000F9471F928F938FEE94E09F938F930E9459
:107D3000FC9A0F900F900F900F900C94F947609160
:107D40007B0270917C0280E090E00E94299A8C0175
:107D500065E376E00E943D9A892B11F489E108C021
:107D600069E376E0C8010E943D9A892B49F480E1DD
:107D70008093C4001092C50082E08093C00055C07B
:107D80006DE376E0C8010E943D9A892B11F488E0EA
:107D9000EFCF62E476E0C8010E943D9A892B39F06A
:107DA00067E476E0C8010E943D9A892B11F483E0D4
:107DB000DFCF8091C400893141F48BE692E09F933C
:107DC0008F930E94FC9A0F900F908091C400803195
:107DD00041F486E692E09F938F930E94FC9A0F9065
:107DE0000F908091C400883041F480E692E09F9328
:107DF0008F930E94FC9A0F900F908091C400833063
:107E000041F48AE592E09F938F930E94FC9A0F9031
:107E10000F908091C400883041F484E592E09F93F4
:107E20008F930E94FC9A0F900F9080917D0288237F
:107E300011F40C94F9471F928F938CEE94E09F936A
:107E40008F930E94FC9A0F900F900F900F900C94BC
:107E5000F94760917B0270917C0280E090E00E9483
:107E6000299A64E276E00E943D9A892B11F481E020
:107E700001C080E00E94A52480917D02882311F436
:107E80000C94F9471F928F9389EE94E09F938F9300
:107E90000E94FC9A0F900F900F900F900C94F9474E
:107EA0000E94CB2280917D02882311F40C94F94723
:107EB0001F928F9386EE94E09F938F930E94FC9A7B
:107EC0000F900F900F900F900C94F9470E94C722CB
:107ED00080917D02882311F40C94F9471F928F93AF
:107EE00083EE94E09F938F930E94FC9A0F900F90E3
:107EF0000F900F900C94F94760917B0270917C0277
:107F000080E090E00E94299A0E941699803170F4D6
:107F10008093510A0E94167241E050E06DE170E0DA
:107F200081E59AE00E94009E0C94F9478091510AE5
:107F30001F928F938AE492E09F938F930E94FC9A02
:107F40000F900F900F900F900C94F94760917B0267
:107F500070917C0280E090E00E94299A0E9416991C
:107F600095EF980F903170F4809361020E94BE707B
:107F700041E050E06CE170E081E692E00E94009EFA
:107F80000C94F947809161021F928F9381E492E0F3
:107F90009F938F930E94FC9A0F900F900F900F90D9
:107FA0000C94F94760917B0270917C0280E090E034
:107FB0000E94299A009789F04AE050E0BC0188EAC3
:107FC0009BE10E944D9A4AE050E064E070E088EA4C
:107FD0009BE10E94009E0C94F94788EA9BE19F93E5
:107FE0008F938CE496E09F938F930E94E89A0F9072
:107FF0000F900F900F900C94F94760917B02709155
:108000007C0280E090E00E94299A8C016CEE73E083
:108010000E943D9A892BD9F4219A80916202909115
:108020006302A0916402B091650280618093620254
:1080300090936302A0936402B093650244E050E021
:108040006EE170E082E692E00E94009ED2C76AE68E
:1080500075E0C8010E943D9A892BD9F4229A80913B
:10806000620290916302A0916402B0916502806205
:108070008093620290936302A0936402B0936502BE
:1080800044E050E06EE170E082E692E00E94009EE3
:10809000B0C76EEC73E0C8010E943D9A892BD9F4F9
:1080A000239A8091620290916302A0916402B09140
:1080B000650280648093620290936302A0936402DD
:1080C000B093650244E050E06EE170E082E692E039
:1080D0000E94009E8EC76DE075E0C8010E943D9A27
:1080E000892BD9F4239A8091620290916302A09126
:1080F0006402B0916502806880936202909363028B
:10810000A0936402B093650244E050E06EE170E039
:1081100082E692E00E94009E6CC769EF79E0C80198
:108120000E943D9A892B71F581E08093F92F81ECB3
:108130009BE19093FB2F8093FA2F1092FD2F1092CA
:10814000FC2F8091620290916302A0916402B09131
:10815000650291608093620290936302A09364022F
:10816000B093650244E050E06EE170E082E692E098
:108170000E94009E49EF5FE262E18EE392E00E947E
:10818000F75B37C765EF73E0C8010E943D9A892B02
:1081900011F5E1EFFBE1119211922CE1E131F207CF
:1081A000D1F78091620290916302A0916402B09134
:1081B000650292608093620290936302A0936402CE
:1081C000B093650244E050E06EE170E082E692E038
:1081D0000E94009E0EC764EA75E0C8010E943D9AA5
:1081E0004091620250916302609164027091650255
:1081F000892BC1F44F705C7F4093620250936302FD
:1082000060936402709365022B9A44E050E06EE143
:1082100070E082E692E00E94009E80919E340E946F
:10822000D370E7C644FD03C084EA95E002C081EA4A
:1082300095E09F938F9386E392E09F938F930E94A4
:10824000FC9A809162020F900F900F900F9085FD25
:1082500003C084EA95E002C081EA95E09F938F9382
:108260008BE292E09F938F930E94FC9A809162022E
:108270000F900F900F900F9086FD03C084EA95E059
:1082800002C081EA95E09F938F9380E292E09F93F2
:108290008F930E94FC9A809162020F900F900F9032
:1082A0000F9087FD03C084EA95E002C081EA95E063
:1082B0009F938F9385E192E09F938F930E94FC9A06
:1082C0008091620290916302A0916402B091650274
:1082D0000F900F900F900F9090FD03C084EA95E0EF
:1082E00002C081EA95E09F938F938AE092E09F938A
:1082F0008F930E94FC9A8091620290916302A091F8
:108300006402B09165020F900F900F900F9091FD55
:1083100003C084EA95E002C081EA95E09F938F93C1
:108320008FEF91E09F938F930E94FC9A809162025D
:1083300090916302A0916402B09165020F900F903A
:108340000F900F9091FF55C684E596E00E94249B04
:1083500091EFE92E9BE1F92E00E010E02CE5822E52
:1083600026E0922EF70180819181F2E0EF0EF11C60
:108370009F938F93C8010B969F938F939F928F9299
:108380000E94E89A0F5F1F4F0F900F900F900F9071
:108390000F900F900031110529F72BC68FED94E057
:1083A0009F938F930E94FC9A80917D020F900F9073
:1083B000882361F01F928F938CED94E09F938F93AD
:1083C0000E94FC9A0F900F900F900F90F89498E0F5
:1083D00088E10FB6F894A895809360000FBE909343
:1083E0006000FFCF0E94C56804C660917B02709157
:1083F0007C0280E090E00E94299A8C0161EA75E09D
:108400000E943D9A892BE9F40E94B96F8091620223
:1084100090916302A0916402B09165028D7F8160AA
:108420008093620290936302A0936402B09365020A
:1084300044E050E06EE170E082E692E00E94009E2F
:10844000D8C564EA75E0C8010E943D9A892BE1F421
:108450000E94716F8091620290916302A091640208
:10846000B09165028C7F8093620290936302A09327
:108470006402B093650244E050E06EE170E082E691
:1084800092E00E94009EB5C567E676E0C8010E94B2
:108490003D9A892BE9F40E94716F8091620290915C
:1084A0006302A0916402B09165028E7F8260809326
:1084B000620290936302A0936402B093650244E069
:1084C00050E06EE170E082E692E00E94009E91C56D
:1084D0008091620281FF0FC087E696E09F938F93A1
:1084E0008BEF91E09F938F930E94FC9A0F900F90D7
:1084F0000F900F907EC580FD03C084EA95E002C016
:1085000081EA95E09F938F9387EF91E09F938F93FC
:108510000E94FC9A0F900F900F900F906AC5809167
:10852000F72F8F938091F62F8F938091F52F8F9354
:108530008091F42F8F938091F32F8F938091F22F5E
:108540008F938091F12F8F938091F02F8F93809153
:10855000EF2F8F938091EE2F8F938091ED2F8F933C
:108560008091EC2F8F938091EB2F8F938091EA2F46
:108570008F938091E92F8F938091E82F8F9380EBD9
:1085800094E09F938F930E94FC9A0E94BA0D809171
:108590007D020FB6F894DEBF0FBECDBF882309F46D
:1085A00028C51F928F938DEA94E09F938F930E942A
:1085B000FC9A0F900F900F900F901BC5F89489E0D4
:1085C00021E030E0F90180935700C895E02C20E0CD
:1085D00030E0F90180935700C895F02C7894F89416
:1085E00023E030E0F90180935700C895002D22E088
:1085F00030E0F90180935700C895102D7894809150
:10860000D1278F938091D0278F938091CF278F93FD
:108610008091CE278F9383EA94E09F938F930E945B
:10862000FC9A1F92EF921F92FF921F920F931F923C
:108630001F938CE794E09F938F930E94FC9A0E9473
:108640006523809166001F928F9380E794E09F934B
:108650008F930E94FC9A0E94BA0D80917D020FB602
:10866000F894DEBF0FBECDBF882309F4C2C41F92A9
:108670008F938DE694E09F938F930E94FC9A0F90C6
:108680000F900F900F90B5C460E070E080E090E034
:108690000E94C30D60E070E081E090E00E94C30D95
:1086A00080917D02882309F4A4C41F928F938AE6E7
:1086B00094E09F938F930E94FC9A0F900F900F90DD
:1086C0000F9097C40E9487210E94BA0D80917D026D
:1086D000882309F48EC41F928F9387E694E09F93BA
:1086E0008F930E94FC9A0F900F900F900F9081C46F
:1086F00060917B0270917C0280E090E00E94299A58
:108700006EE176E00E943D9A892B31F5F89486E976
:108710009AE00E94E65C8C01892B69F0C8010F96F3
:108720000E94EE5FB80184E092E00E949F5CC80165
:108730000E94925DF0CF86E99AE00E94775D892BD6
:1087400029F086E99AE00E941F5DF5CF86E99AE05C
:108750000E94E25C789436C086E99AE00E94E65C6A
:108760008C018CE6E82E86E0F82E0115110551F1FA
:10877000F80186811F928F9380851F928F93858148
:108780001F928F9381851F928F9387811F928F9362
:1087900084811F928F9383811F928F9382811F9276
:1087A0008F9382851F928F93FF92EF920E94E89A97
:1087B000C8010E94925D8C010FB6F894DEBF0FBE17
:1087C000CDBFD3CF80917D02882309F412C41F92BC
:1087D0008F9384E694E09F938F930E94FC9A0F906E
:1087E0000F900F900F9005C40E94013102C4609158
:1087F0007B0270917C0280E090E00E94299A8C01BB
:108800006BEA76E00E943D9A892BD1F48091620256
:1088100090916302A0916402B0916502977F80936A
:10882000620290936302A0936402B093650244E0F5
:1088300050E06EE170E082E692E00E94009ED9C3B3
:108840006AE276E0C8010E943D9A892BD1F48091BA
:10885000620290916302A0916402B09165029860F7
:108860008093620290936302A0936402B0936502C6
:1088700044E050E06EE170E082E692E00E94009EEB
:10888000B8C30E94330AB5C360917B0270917C0229
:1088900080E090E00E94299AFC0120812332C1F4FB
:1088A0004AE050E060E070E001960E94AF967B8362
:1088B0006A8360917B0270917C0280E090E00E946C
:1088C000299A2A813B81243031050CF096C002C0E0
:1088D0001B821A82009709F490C01982BE016F5F53
:1088E0007F4F0E944A2A19013A014B01B82FA92F44
:1088F0008AE02A813B81829FF001839FF00D112441
:10890000EF53F44E4080518032813C8383818D83CC
:1089100094819E8325812F8336813887878189873B
:108920009101A301B4018B2F9A2F5201CC80DD80DD
:10893000EE80FF80088519850E94409609F460C08A
:108940008981811103C0208231822AC0181684F4E3
:10895000422853289C81692A2D81722A3E81832ACC
:108960008F81982A9885B92B2985A22B408217C020
:10897000209430946094709480949094B095A095D5
:10898000242053203C8163228D8178229E8189227C
:108990002F8192223885B3238985A8232082518292
:1089A0006282738284829582B683A78348E250E014
:1089B00062E270E081EC9BE10E94009E8CE594E015
:1089C0009F938F930E94FC9A8AE02A813B81829F29
:1089D000F001839FF00D1124EF53F44E208131817B
:1089E0004281538164817581868197810E9493269B
:1089F0000E94BA0D0F900F9003C082E00E94002CDD
:108A000080E594E09F938F930E94FC9A2FEF3FEFB5
:108A10004FEF5FEF6FEF7FEF8FEF9FEF0E94932697
:108A20000E94BA0D80917D020F900F90882309F467
:108A3000E0C21F928F938DE494E09F938F930E94E6
:108A4000FC9A0F900F900F900F90D3C260917B0211
:108A500070917C0280E090E00E94299AFC012081C4
:108A60002332A1F44AE050E060E070E001960E94F9
:108A7000AF968B0160917B0270917C0280E090E068
:108A80000E94299A04301105ECF402C000E010E0C5
:108A90000097C1F04AE050E060E070E00E94DA9791
:108AA0002AE0209FF001219FF00D1124EF53F44E96
:108AB0007187608748E250E062E270E081EC9BE100
:108AC0000E94009E81E00E94002C80917D028823FC
:108AD00009F48FC21F928F938AE494E09F938F933F
:108AE0000E94FC9A0F900F900F900F9082C20E94EC
:108AF000266080917D02882309F47BC21F928F93A8
:108B000087E494E09F938F930E94FC9A0F900F90BC
:108B10000F900F906EC20E94C52C80917D02882319
:108B200009F467C21F928F9384E494E09F938F931C
:108B30000E94FC9A0F900F900F900F905AC280E005
:108B400090E00E94812380917D02882309F451C224
:108B50001F928F9381E494E09F938F930E94FC9ADD
:108B60000F900F900F900F9044C28091DE2B81FFE9
:108B70002DC00E940D21892B49F58091D5278F9317
:108B80008091D4278F938091D3278F938091D22780
:108B90008F9386E394E09F938F930E94FC9A809139
:108BA000B6348F938091B5348F938091B4348F9382
:108BB0008091B3348F9389E294E09F938F930E94C6
:108BC000FC9A0FB6F894DEBF0FBECDBF0E94BA0D5F
:108BD0008091DE2B9091DF2B90FF63C081E090E0CD
:108BE0000E9484207B011C0180E090E00E94842090
:108BF0004B018C010E94E21F3F922F92FF92EF9255
:108C000088E194E09F938F930E94FC9A1F930F93A7
:108C10009F928F9288E094E09F938F930E94FC9A9A
:108C2000240138019401A80147018101B701C10164
:108C30000E94811E9F938F937F936F938DEF93E09C
:108C40009F938F930E94FC9A242D352D462D572DEE
:108C50006E2D792D822D912F0E94E21E9F938F936E
:108C60007F936F938FEE93E09F938F930E94FC9A74
:108C7000242D352D462D572D6E2D792D822D912F9A
:108C80000E94431F9F938F937F936F938CED93E08C
:108C90009F938F930E94FC9A0FB6F894DEBF0FBE8D
:108CA000CDBF0E94BA0D80917D02882309F4A1C135
:108CB0001F928F9389ED93E09F938F930E94FC9A6C
:108CC0000F900F900F900F9094C18091DE2B82FF38
:108CD0002BC021E048E061E083E00E945F158091B5
:108CE000C51C8F938091C41C8F938091C31C8F935C
:108CF0008091C21C8F938091C11C8F938091C01C66
:108D00008F938091BF1C8F938091BE1C8F9382ECB8
:108D100093E09F938F930E94FC9A0E94BA0D0FB626
:108D2000F894DEBF0FBECDBF8091DE2B9091DF2B7C
:108D300091FF3BC00E94C31920E030E048EC52E4B0
:108D4000162F072FF82EE92E0E94FB9220E836EE10
:108D500045EC57E40E944F9021E03EED42E45EE393
:108D60000E9468939B01AC0160E070E080E89FE3A3
:108D70000E946B8F2BE43AE34DEB57E30E944F9038
:108D80009F938F937F936F93EF92FF920F931F9315
:108D900089EA93E09F938F930E94FC9A0E94BA0DF8
:108DA0000FB6F894DEBF0FBECDBF80917D02882341
:108DB00009F41FC11F928F9386EA93E09F938F93CC
:108DC0000E94FC9A0F900F900F900F9012C160912B
:108DD0007B0270917C0280E090E00E94299A60EB17
:108DE00076E00E943D9A892BB1F460917B027091EC
:108DF0007C0280E090E00E94299A009709F4F9C073
:108E00000E941699803108F0F4C090915201892B8C
:108E100080935201EEC0809152018F701F928F9308
:108E20008AEE91E09F938F930E94FC9A0E94BA0D64
:108E30000F900F900F900F90DCC060917B027091AB
:108E40007C0280E090E00E94299A009711F14AE0AC
:108E500050E060E070E00E94AF96603198F460935B
:108E600060021F926F9389E993E09F938F930E9412
:108E7000FC9A41E050E06BE170E080E692E00E94F5
:108E8000009E11C0809160021F928F9380E993E051
:108E900006C0809160021F928F9387E893E09F93B2
:108EA0008F930E94FC9A0F900F900F900F900E944A
:108EB000BA0D80917D02882309F49BC01F928F9385
:108EC00084E893E09F938F930E94FC9A0F900F90F9
:108ED0000F900F908EC060917B0270917C0280E0B9
:108EE00090E00E94299A8C0161EA75E00E943D9A07
:108EF000892BE1F40E94236E8091620290916302BB
:108F0000A0916402B0916502906180936202909397
:108F10006302A0936402B093650244E050E06EE106
:108F200070E082E692E00E94009E63C064EA75E011
:108F3000C8010E943D9A892B99F5F8940E94306EE1
:108F40000FB6F894A89580916000886180936000C6
:108F5000109260000FBE84B7877F84BF809160004D
:108F60008861809360001092600078948091620222
:108F700090916302A0916402B09165029F7E8093FC
:108F8000620290936302A0936402B093650244E08E
:108F900050E06EE170E082E692E00E94009E29C0FF
:108FA00065EB76E0C8010E943D9A409162025091C3
:108FB00063026091640270916502892B21F454FF71
:108FC00018C0F894FFCF54FD03C084EA95E002C0B6
:108FD00081EA95E09F938F9386EE91E09F938F9324
:108FE0000E94FC9A0F900F900F900F9002C00E9469
:108FF000AB21EA85FB851182108283E02B960FB6A8
:10900000F894DEBF0FBECDBFDF91CF911F910F91BE
:10901000FF90EF90DF90CF90BF90AF909F908F9098
:109020007F906F905F904F903F902F900895CF93D7
:10903000DF93EC0188819981009741F0843F914151
:1090400009F48CC01982188283E093C00E945432C4
:109050008091620280FD05C081FF01C01D9B0E94BE
:10906000716F809170008C7F809370008091B6004A
:1090700080628093B6001092B20082E08093B100CB
:109080008091B6008770E1F78091700081608093D5
:10909000700061E57AE080E090E00E94FD6D0E9442
:1090A000C72280E00E94A52480EB90E19F938F93DC
:1090B0000E94FC9A0E9448128091DE2B0F900F9024
:1090C00086FD0E9471688091DE2B9091DF2B90FDD0
:1090D0000E949A1F8091DE2B87FF06C021E04CE0A2
:1090E00061E080ED0E9414698091510A0E9416721D
:1090F000809161020E94BE700E94BB708093860ABC
:10910000809161020E94BE708091510A1F928F93DC
:109110008091860A1F928F938AEB96E09F938F939C
:109120000E94E89A1092880A1092870A0F900F9076
:109130000F900F900F900F9082E592E09093B134D2
:109140008093B03483E290E09093991280939812C8
:1091500084EF91E19983888381E00BC06332E1F76A
:109160004DE050E360E070E087E89AE00E94BF3392
:10917000E3CFDF91CF9108950F931F93CF93DF93A8
:10918000EC018A0188819981009711F1893092411F
:1091900021F01982188283E020C06231E9F4A8012D
:1091A00062E170E087E89AE00E94BF3384E0809338
:1091B000953410929734109296341093993400930A
:1091C000983445E954E362E18EE392E00E94F75B54
:1091D00089E092E19983888381E0DF91CF911F91AB
:1091E0000F910895AF92BF92CF92DF92EF92FF92CC
:1091F0000F931F93CF93DF93EC018091550A9091C9
:10920000560AA091570AB091580A81FD08C0909162
:10921000620290FD04C091FF57C01D9B55C05A01CA
:109220008B01FB01C384D484E584F684A4E6B0E01A
:10923000A70196010E947D94672F782F892F992787
:1092400024E630E040E050E00E940E947F936F935C
:10925000CD2CDE2CEF2CFF24DF92CF92F8018681FB
:109260001F928F9385811F928F9388818F701F9299
:109270008F9389811F928F93F50181811F928F9324
:1092800080811F928F932296DF93CF938CEC96E090
:109290009F938F930E94E89A80917D02EDB7FEB76D
:1092A00074960FB6F894FEBF0FBEEDBF882361F031
:1092B0001F928F9380EE91E09F938F930E94FC9A70
:1092C0000F900F900F900F90DF91CF911F910F9102
:1092D000FF90EF90DF90CF90BF90AF9008958436CD
:1092E000910514F19F938F9380E197E09F938F9363
:1092F0000E94E89A8091E82F9091E92FA091EA2F9F
:10930000B091EB2F0196A11DB11D8093E82F909392
:10931000E92FA093EA2FB093EB2F0F900F900F90AF
:109320000F9081E090E0089580E090E008952F9202
:109330003F924F925F926F927F928F929F92AF92E5
:10934000BF92CF92DF92EF92FF920F931F93CF9332
:10935000DF93CDB7DEB7CC59D1090FB6F894DEBF95
:109360000FBECDBFCB56DF4F99838883C559D04000
:109370008A01633871F48BE89AE0C456DF4F688342
:10938000CC59D0400E94365AC456DF4F6881CC5920
:10939000D040CB56DF4FA881B981C559D0402D911F
:1093A0003C91213AB1E13B0709F414C440F4211582
:1093B000310581F0273C3F4009F456C44AC4233BA1
:1093C00041E1340709F426C42A3B314111F40C94DD
:1093D0005F573FC444EF52E061E870E08BE89AE0E9
:1093E0000E941B5A87EC9FE0ECC35A01E3E0F0E0D7
:1093F000EC0FFD1FE40FF51F1082CA010E946F4998
:10940000892B81F720E030E040E050E0CC56DF4F80
:109410006881C459D040627070E080E090E0A0E0C4
:109420000E94499609F0BBC6212F287030E040E029
:1094300050E060E070E080E090E0A0E00E9449969B
:1094400099F127E04AE250E06BE270E089E290E0B7
:109450000E94546487EA94E30E94C366BC01990F9A
:10946000880B990B0E94039120E030E048EC52E415
:109470000E944F909F938F937F936F9384E497E024
:109480009F938F931F9287E78F93CE018A0D9B1D29
:1094900003969F938F930E94549BA80EB91E0FB6FC
:1094A000F894DEBF0FBECDBF212F207130E040E029
:1094B00050E060E070E080E090E0A0E00E9449961B
:1094C000E9F126E04AE250E06BE270E089E290E0E8
:1094D0000E94546481E090E00E94520D8093500AF3
:1094E0008AE19CE10E94C366BC01990F880B990B2D
:1094F0000E94039120E030E048EC52E40E944F903B
:109500009F938F937F936F938EE497E09F938F93B6
:109510001F9287E78F93C501029621E030E02C0F60
:109520003D1F820F931F9F938F930E94549BA80E01
:10953000B91E0FB6F894DEBF0FBECDBFC257DF4FC6
:109540002881CE58D04030E040E050E060E070E04C
:1095500080E090E0A0E00E94499601F10E940E0D8B
:109560009F938F937F936F9389E597E09F938F935A
:109570001F9287E78F93C5010296A1E0B0E0AC0F80
:10958000BD1F8A0F9B1F9F938F930E94549BA80E11
:10959000B91E0FB6F894DEBF0FBECDBF212F2074C9
:1095A00030E040E050E060E070E080E090E0A0E07B
:1095B0000E94499631F18091E32F8F938091E22FA1
:1095C0008F938091E12F8F938091E02F8F9387E687
:1095D00097E09F938F931F9287E78F93C501029621
:1095E00021E030E02C0F3D1F820F931F9F938F933C
:1095F0000E94549BA80EB91E0FB6F894DEBF0FBE92
:10960000CDBF212F207830E040E050E060E070E0F6
:1096100080E090E0A0E00E94499641F1F8948091AA
:109620008D3490918E34A0918F34B0919034789491
:10963000BF93AF939F938F9385E797E09F938F930B
:109640001F9287E78F93C5010296A1E0B0E0AC0FAF
:10965000BD1F8A0F9B1F9F938F930E94549BA80E40
:10966000B91E0FB6F894DEBF0FBECDBF20E0302F7D
:10967000317040E050E060E070E080E090E0A0E019
:109680000E94499609F09DC520E0302F327040E0DD
:1096900050E060E070E080E090E0A0E00E94499639
:1096A00009F00DC620E0302F347040E050E060E05B
:1096B00070E080E090E0A0E00E94499609F030C69A
:1096C00020E0302F387040E050E060E070E080E053
:1096D00090E0A0E00E94499609F051C620E0302FAA
:1096E000307140E050E060E070E080E090E0A0E0A9
:1096F0000E94499609F0C1C620E0302F307240E048
:1097000050E060E070E080E090E0A0E00E944996C8
:1097100009F0E3C620E030E040E050E0CC56DF4FF7
:109720006881C459D040647070E080E090E0A0E0AF
:109730000E94499609F0FFC620E0C856DF4F3881E5
:10974000C859D04040E050E060E070E080E090E038
:10975000A0E00E94499609F05BC720E0C756DF4FA2
:109760003881C959D04040E050E060E070E080E0CE
:1097700090E0A0E00E94499609F078C7CE56DF4FEE
:109780005881C259D0405170952E20E030E0452FCD
:1097900050E060E070E080E090E0A0E00E94499638
:1097A00009F092C720E030E0CE56DF4F4881C25921
:1097B000D040427050E060E070E080E090E0A0E0D7
:1097C0000E94499609F0B3C720E030E0C657DF4F4A
:1097D0004881CA58D04050E060E070E080E090E0FE
:1097E000A0E00E94499609F0D5C720E030E040E0B3
:1097F00050E0CC56DF4F6881C459D040687070E0AB
:1098000080E090E0A0E00E94499609F0EEC720E0D9
:1098100030E040E050E0CC56DF4F6881C459D04082
:10982000607170E080E090E0A0E00E94499611F045
:109830000C94215420E030E0CE56DF4F4881C259CD
:10984000D040487050E060E070E080E090E0A0E040
:109850000E94499611F00C944D5420E030E0CE5611
:10986000DF4F4881C259D040407150E060E070E065
:1098700080E090E0A0E00E94499611F00C948054A2
:1098800020E030E0CE56DF4F4881C259D0404072D0
:1098900050E060E070E080E090E0A0E00E94499637
:1098A00011F00C94B35420E030E0CE56DF4F4881E5
:1098B000C259D040407450E060E070E080E090E039
:1098C000A0E00E94499611F00C94E654CE56DF4F6A
:1098D000F881C259D040F0787F2E20E030E04F2F41
:1098E00050E060E070E080E090E0A0E00E944996E7
:1098F00011F00C941955CD56DF4F2881C359D04033
:109900002170622E20E030E040E0562D60E070E0F3
:1099100080E090E0A0E00E94499611F40C94725708
:109920008091DE2B82FD02C00C94615521E046E05F
:1099300061E083E00E945F1520E030E0472D50E0B9
:1099400060E070E080E090E0A0E00E94499611F4B1
:109950000C9461558091DE2B82FF02C00C94265539
:1099600020E030E040E0CD56DF4F5881C359D04071
:10997000527060E070E080E090E0A0E00E944996C4
:1099800011F00C94965520E030E040E0CD56DF4FCA
:109990005881C359D040547060E070E080E090E09E
:1099A000A0E00E94499611F00C94C95520E030E0E7
:1099B00040E0CD56DF4F5881C359D040507160E030
:1099C00070E080E090E0A0E00E94499611F00C94D5
:1099D000FC5520E030E040E0CD56DF4F5881C359C0
:1099E000D040507260E070E080E090E0A0E00E9423
:1099F000499611F00C943B5620E030E040E0CD5603
:109A0000DF4F5881C359D040507460E070E080E06F
:109A100090E0A0E00E94499611F00C947A5620E064
:109A200030E040E0CD56DF4F5881C359D0405870E8
:109A300060E070E080E090E0A0E00E94499611F0C4
:109A40000C94B95620E030E040E0C656DF4F588114
:109A5000CA59D04060E070E080E090E0A0E00E9451
:109A6000499611F00C94EA5620E030E0492D50E080
:109A700060E070E080E090E0A0E00E94499611F084
:109A80000C942157212F302FCE56DF4F4881C259D9
:109A9000D040CD56DF4F5881C359D040CC56DF4F10
:109AA0006881C459D0407D2DC956DF4F8881C75980
:109AB000D0409C2DA0E00E94499611F00C942C57A8
:109AC000809160028061898380917F0A8A83FE0190
:109AD000EA0DFB1D13828091550A9091560AA091C0
:109AE000570AB091580A85010D5F1F4F80FF0CC0C7
:109AF0001F930F9385E199E09F938F930E94E89ABB
:109B00000F900F900F900F90B801CE0101960E9418
:109B10004B638091620282FF0AC02DE830E3A80106
:109B2000BE016F5F7F4F8BE692E00E94D767809106
:109B3000550A9091560AA091570AB091580A82FD91
:109B400073980E94B96F8BE89AE00E94385A80910E
:109B5000620290916302A0916402B091650290FF4D
:109B600040C03FEFA31AB30A0E94BB70F82E89E1F0
:109B70000E94D3708091620290916302A09164026E
:109B8000B091650290FF29C0739880917F0A8F5F22
:109B900080937F0A8A83B5016F5F7F4FCE01019664
:109BA0000E944B638BE89AE00E94385A40E050E0F4
:109BB00065E880919C1290919D120E94F75B81EA6A
:109BC00091E1CB56DF4FA881B981C559D0408D9323
:109BD0009C933CC0A12CB12CCDCF8F2D0E94D37073
:109BE000739A8091520A9091530A892B11F00E9426
:109BF000716F80917F0A8F5F80937F0A8091550AF1
:109C00009091560AA091570AB091580A82FFEACB68
:109C1000739AE8CB87E79AE00E94A35E892BB1F0A4
:109C20000E94B96F8091620287FD2B9860E470E01A
:109C300087E79AE00E947C5E8AEB91E1CB56DF4F8A
:109C4000E881F981C559D0409183808381E00C94EB
:109C50008257CB56DF4FA881B981C559D0401D929C
:109C60001C9283E00C948257623181F780906202EB
:109C700090906302A0906402B090650291FCB2CB18
:109C8000F8018081813021F50180F281E02D108181
:109C900001812281CE56DF4F2883C259D0403381C3
:109CA000CD56DF4F3883C359D0404481CC56DF4F67
:109CB0004883C459D040D5805681C956DF4F588358
:109CC000C759D040C780E084F184212C312C52C088
:109CD0008230B9F423803480E12CF12C11E000E0D3
:109CE000CE56DF4F1882C259D040B0E8CD56DF4F74
:109CF000B883C359D040CC56DF4F1882C459D040E6
:109D000032C08330D1F0843009F06CCBE12CF12CDF
:109D1000212C312C15E000E0CE56DF4F1882C259BD
:109D2000D040CD56DF4F1882C359D040E2E0CC5628
:109D3000DF4FE883C459D04016C0E12CF12C212C10
:109D4000312C15E000E0CE56DF4F1882C259D040CA
:109D5000CD56DF4F1882C359D040F1E0CC56DF4FCB
:109D6000F883C459D040D12CC956DF4F1882C75947
:109D7000D040C12C4090E02F5090E12F6090E22F16
:109D80007090E32F20918A0230918B0240918C02D7
:109D900050918D02C657DF4F288339834A835B83F6
:109DA000CA58D0402DEC3CEC4CE45EE3C657DF4F84
:109DB000688179818A819B81CA58D0400E946C8FCA
:109DC0009B01AC01C301B2010E94289287FD0BC028
:109DD000E894A0F88092620290926302A0926402DA
:109DE000B092650246C0C657DF4F288139814A814B
:109DF0005B81CA58D040C301B2010E944A9087FFDC
:109E000038C08091EC2F9091ED2FA091EE2FB09162
:109E1000EF2F0196A11DB11D8093EC2F9093ED2F94
:109E2000A093EE2FB093EF2FA0FCDCCA6894A0F8AB
:109E30008092620290926302A0926402B0926502E4
:109E400015E400E2CE56DF4F1882C259D040CD56FD
:109E5000DF4F1882C359D04034E0CC56DF4F3883EF
:109E6000C459D040D12CC956DF4F1882C759D040B1
:109E7000C12CCE56DF4F4881C259D0404470C657DE
:109E8000DF4F4883CA58D04020E030E050E060E027
:109E900070E080E090E0A0E00E94499609F08C9A82
:109EA000512F5072C257DF4F5883CE58D040252FC4
:109EB00030E040E050E060E070E080E090E0A0E062
:109EC0000E94499611F00E940E0D802F8074C85692
:109ED000DF4F8883C859D04020E0382F40E050E061
:109EE00060E070E080E090E0A0E00E94499611F010
:109EF0000E940D21902F9078C756DF4F9883C95943
:109F0000D04020E0392F40E050E060E070E080E099
:109F100090E0A0E00E94499651F00E94A90C609345
:109F20009A3470939B3480939C3490939D34212F6A
:109F3000217030E040E050E060E070E080E090E0D0
:109F4000A0E00E944996F1F088EA9BE19F938F93ED
:109F500084E297E09F938F931F9287E78F93CE01C0
:109F600003969F938F930E94549B4C010E946F49CC
:109F70000FB6F894DEBF0FBECDBF892B09F032CAF1
:109F8000540102C0A12CB12C212F227030E040E0FE
:109F900050E060E070E080E090E0A0E00E94499630
:109FA000D1F1C50102966CE277E0E1E0F0E0EC0F60
:109FB000FD1F8E0F9F1F0E94469AF3E0AF0EB11C4B
:109FC00027EA622E24E3722E3EEF832E33E0932E97
:109FD00047E7542ED3018D913D011F928F939F929D
:109FE0008F921F925F92C5010296E1E0F0E0EC0FC4
:109FF000FD1F8E0F9F1F9F938F930E94549BA80E4F
:10A00000B91E0FB6F894DEBF0FBECDBF3FEA631690
:10A0100034E37306F9F6212F247030E040E050E07D
:10A0200060E070E080E090E0A0E00E94499609F4D2
:10A0300050C0C501029660E377E041E050E04C0F6C
:10A040005D1F840F951F0E94469A54E0A50EB11C17
:10A050002E018AE7480E511C80E1D2011D928A959B
:10A06000E9F728E0A20168E980EB0E94AA13320117
:10A07000B8E06B0E711C9EEF892E93E0992E27E7B6
:10A08000F20181912F011F928F939F928F921F92C5
:10A090002F93C501029641E050E04C0F5D1F840FE5
:10A0A000951F9F938F93C556DF4F2883CB59D04080
:10A0B0000E94549BA80EB91E0FB6F894DEBF0FBEC7
:10A0C000CDBFC556DF4F2881CB59D0404614570429
:10A0D000B9F6CD56DF4F9881C359D0409078C65617
:10A0E000DF4F9883CA59D04020E030E040E0592F3C
:10A0F00060E070E080E090E0A0E00E944996E1F42A
:10A100008091520A9091530A9F938F9385E397E031
:10A110009F938F931F9287E78F93CE018A0D9B1D8C
:10A1200003969F938F930E94549BA80EB91E0FB65F
:10A13000F894DEBF0FBECDBF20E030E040E050E03D
:10A14000CC56DF4F6881C459D040617070E080E028
:10A1500090E0A0E00E94499609F454C9E3E0F0E0E1
:10A16000EC0FFD1FEA0DFB1D80E28083A50183E05B
:10A1700090E08A199B09FC01E40FF51FE35FFF4C97
:10A1800020814F5F5F4F222309F42FC92081E1E036
:10A19000F0E0EC0FFD1FE40FF51F2283ECCFCE01A2
:10A1A0008A0D9B1D6CE377E003960E94469AB7E008
:10A1B000AB0EB11CC5010E946F49892B09F012C971
:10A1C00033C9E114F10409F45FCAF89440908D3466
:10A1D00050908E3460908F34709090347894809149
:10A1E000121C9091131CA091141CB091151CA3017A
:10A1F0009201281B390B4A0B5B0BCA01B9010E9463
:10A200000191C257DF4F688379838A839B83CE583D
:10A21000D040B70180E090E00E9401919B01AC0129
:10A22000C257DF4F688179818A819B81CE58D040A7
:10A230000E944F904C019F928F937F936F9380E881
:10A2400097E09F938F931F9287E78F939E012A0D2C
:10A250003B1D2D5F3F4F3F932F93C456DF4F6883C5
:10A26000CC59D040C556DF4F7883CB59D0400E949F
:10A27000549BA80EB91EC456DF4F6881CC59D040FC
:10A28000C556DF4F7881CB59D040862F972FA82D08
:10A29000B92D80939F349093A034A093A134B093B0
:10A2A000A2344092121C5092131C6092141C7092A3
:10A2B000151C0FB6F894DEBF0FBECDBFE5C9E11483
:10A2C000F10409F4EFC9F8948091E91B9091EA1B1D
:10A2D000A091EB1BB091EC1B78949F938F9380918E
:10A2E00069028F93809168028F938DE897E09F9326
:10A2F0008F931F9287E78F93C5010296A1E0B0E08C
:10A30000AC0FBD1F8A0F9B1F9F938F930E94549B7E
:10A31000A80EB91E0FB6F894DEBF0FBECDBFC2C9DE
:10A32000F8948091913490919234A0919334B091AB
:10A3300094347894BF93AF939F938F938DE997E074
:10A340009F938F931F9287E78F93C501029621E019
:10A3500030E02C0F3D1F820F931F9F938F930E941D
:10A36000549BA80EB91EC5010E946F490FB6F89400
:10A37000DEBF0FBECDBF892B09F034C8A1C9E114DF
:10A38000F10409F4ABC9F8944090913450909234A0
:10A39000609093347090943478948091161C9091CE
:10A3A000171CA091181CB091191CA3019201281B25
:10A3B000390B4A0B5B0BCA01B9010E940191C257CC
:10A3C000DF4F688379838A839B83CE58D040B7015F
:10A3D00080E090E00E9401919B01AC01C257DF4FE9
:10A3E000688179818A819B81CE58D0400E944F90AC
:10A3F0004C019F928F937F936F9388EA97E09F938E
:10A400008F931F9287E78F939E012A0D3B1D2D5F2F
:10A410003F4F3F932F93C456DF4F6883CC59D040B2
:10A42000C556DF4F7883CB59D0400E94549BA80E6D
:10A43000B91EC456DF4F6881CC59D040C556DF4F96
:10A440007881CB59D040862F972FA82DB92D809396
:10A45000A3349093A434A093A534B093A63440922F
:10A46000161C5092171C6092181C7092191C0FB683
:10A47000F894DEBF0FBECDBF31C9EF2809F43CC947
:10A48000F8948091ED1B9091EE1BA091EF1BB09181
:10A49000F01B78949F938F93809167028F938091A4
:10A4A00066028F9385EB97E09F938F931F9287E7C8
:10A4B0008F93C5010296A1E0B0E0AC0FBD1F8A0FDB
:10A4C0009B1F9F938F930E94549BA80EB91E0FB69B
:10A4D000F894DEBF0FBECDBF0FC98091E42F9091DD
:10A4E000E52FA091E62FB091E72FBF93AF939F93F5
:10A4F0008F9385EC97E09F938F931F9287E78F93BD
:10A50000C501029621E030E02C0F3D1F820F931F02
:10A510009F938F930E94549BA80EB91EC5010E9461
:10A520006F490FB6F894DEBF0FBECDBF892B11F077
:10A530000C94F249EFC88091EF2F8F938091EE2F0A
:10A540008F938091ED2F8F938091EC2F8F9380913B
:10A55000EB2F8F938091EA2F8F938091E92F8F9328
:10A560008091E82F8F9380ED97E09F938F931F92B8
:10A5700087E7982E9F92C5010296A1E0B0E0AC0F4C
:10A58000BD1F8A0F9B1F9F938F930E94549BA80E01
:10A59000B91EC5010E946F490FB6F894DEBF0FBE09
:10A5A000CDBF892B11F00C94F2498091DE2B909154
:10A5B000DF2B90FFC1C88091F32F8F938091F22FF2
:10A5C0008F938091F12F8F938091F02F8F9384EF51
:10A5D00097E09F938F931F929F92C501029621E06F
:10A5E00030E02C0F3D1F820F931F9F938F930E948B
:10A5F000549BA80EB91EC5010E946F490FB6F8946E
:10A60000DEBF0FBECDBF892B11F00C94F24994C868
:10A610008091D5278F938091D4278F938091D327D2
:10A620008F938091D2278F9386E098E09F938F93AA
:10A630001F9287E78F93C5010296A1E0B0E0AC0FAF
:10A64000BD1F8A0F9B1F9F938F930E94549BA80E40
:10A65000B91EC5010E946F490FB6F894DEBF0FBE48
:10A66000CDBF892B11F00C94F24977C880919D34AD
:10A670008F9380919C348F9380919B348F938091A2
:10A680009A348F9381E198E09F938F931F9287E78D
:10A690008F93C501029621E030E02C0F3D1F820F01
:10A6A000931F9F938F930E94549BA80EB91EC501C0
:10A6B0000E946F490FB6F894DEBF0FBECDBF892B45
:10A6C00011F00C94F2495AC881E00E945B0C209171
:10A6D00082023091830240918402509185020E944F
:10A6E000FB929F938F937F936F938EE198E09F935C
:10A6F0008F931F9287E78F93C5010296A1E0B0E088
:10A70000AC0FBD1F8A0F9B1F9F938F930E94549B7A
:10A71000A80EB91EC5010E946F490FB6F894DEBF9E
:10A720000FBECDBF892B11F00C94F2493BC882E0DB
:10A730000E945B0C20917E0230917F02409180024A
:10A74000509181020E94FB929F938F937F936F930E
:10A750008BE298E09F938F931F9287E78F93C501B9
:10A76000029621E030E02C0F3D1F820F931F9F9334
:10A770008F930E94549BA80EB91EC5010E946F4979
:10A780000FB6F894DEBF0FBECDBF892B11F00C942D
:10A79000F2491AC883E00E945B0C9F938F937F93CA
:10A7A0006F9388E398E09F938F931F9287E78F932F
:10A7B000C5010296A1E0B0E0AC0FBD1F8A0F9B1F40
:10A7C0009F938F930E94549BA80EB91E8C98C5012D
:10A7D0000E946F490FB6F894DEBF0FBECDBF892B24
:10A7E00011F00C94F2490C94F54B299903C084EABA
:10A7F00095E002C081EA95E09F938F9385E498E00D
:10A800009F938F931F9287E78F93C501029621E054
:10A8100030E02C0F3D1F820F931F9F938F930E9458
:10A82000549BA80EB91EC5010E946F490FB6F8943B
:10A83000DEBF0FBECDBF892B11F00C94F2490C94F2
:10A84000074C2A9903C084EA95E002C081EA95E0AA
:10A850009F938F938DE498E09F938F931F9287E748
:10A860008F93C5010296A1E0B0E0AC0FBD1F8A0F27
:10A870009B1F9F938F930E94549BA80EB91EC501E6
:10A880000E946F490FB6F894DEBF0FBECDBF892B73
:10A8900011F00C94F2490C941A4C8091DE2B87FD38
:10A8A00002C00C942D4C21E042E161E080ED0E9459
:10A8B00014699F938F937F936F9385E598E09F939F
:10A8C0008F931F9287E78F93C501029621E030E0B6
:10A8D0002C0F3D1F820F931F9F938F930E94549BB9
:10A8E000A80EB91EC5010E946F490FB6F894DEBFCD
:10A8F0000FBECDBF892B11F00C94F2490C942D4C56
:10A900008091DE2B87FD02C00C94404C21E042E197
:10A9100062E080ED0E9414699F938F937F936F9301
:10A9200083E698E09F938F931F9287E78F93C501EB
:10A930000296A1E0B0E0AC0FBD1F8A0F9B1F9F9352
:10A940008F930E94549BA80EB91EC5010E946F49A7
:10A950000FB6F894DEBF0FBECDBF892B11F00C945B
:10A96000F2490C94404C8091DE2B87FD02C00C9480
:10A97000534C21E042E163E080ED0E9414699F9313
:10A980008F937F936F9381E798E09F938F931F92AC
:10A9900087E78F93C501029621E030E02C0F3D1F21
:10A9A000820F931F9F938F930E94549BA80EB91EF2
:10A9B000C5010E946F490FB6F894DEBF0FBECDBF30
:10A9C000892B11F00C94F2490C94534C8091DE2B9E
:10A9D00087FD02C00C94664C21E042E164E080ED0A
:10A9E0000E9414699F938F937F936F938FE798E0F2
:10A9F0009F938F931F9287E78F93C5010296A1E0E3
:10AA0000B0E0AC0FBD1F8A0F9B1F9F938F930E94D6
:10AA1000549BA80EB91EC5010E946F490FB6F89449
:10AA2000DEBF0FBECDBF892B11F00C94F2490C9400
:10AA3000664C8091DE2B82FD02C00C947B4C46E07C
:10AA400061E083E00E945F150C947B4C8091C11CF7
:10AA50008F938091C01C8F938091BF1C8F938091A6
:10AA6000BE1C8F938DE898E09F938F931F9287E78A
:10AA70008F93C501029641E050E04C0F5D1F840F9B
:10AA8000951F9F938F930E94549BA80EB91EC501DA
:10AA90000E946F490FB6F894DEBF0FBECDBF892B61
:10AAA00011F00C94F24920E030E040E0562D60E0D7
:10AAB00070E080E090E0A0E00E94499611F40C94D0
:10AAC000B04C8091DE2B82FD02C00C94B04C809182
:10AAD000C51C8F938091C41C8F938091C31C8F934E
:10AAE0008091C21C8F9385E998E09F938F931F926A
:10AAF00087E78F93C5010296E1E0F0E0EC0FFD1FC0
:10AB00008E0F9F1F9F938F930E94549BA80EB91E78
:10AB1000C5010E946F490FB6F894DEBF0FBECDBFCE
:10AB2000892B11F00C94F2490C94B04C8091DE2BDF
:10AB30009091DF2B90FD02C00C94C34C80E090E01C
:10AB40000E9484209F938F937F936F9380EA98E075
:10AB50009F938F931F9287E78F93C501029641E0E1
:10AB600050E04C0F5D1F840F951F9F938F930E94A1
:10AB7000549BA80EB91EC5010E946F490FB6F894E8
:10AB8000DEBF0FBECDBF892B11F00C94F2490C949F
:10AB9000C34C8091DE2B9091DF2B90FD02C00C9472
:10ABA000D64C81E090E00E9484209F938F937F9306
:10ABB0006F9380EB98E09F938F931F9287E78F931B
:10ABC000C5010296E1E0F0E0EC0FFD1F8E0F9F1F24
:10ABD0009F938F930E94549BA80EB91EC5010E949B
:10ABE0006F490FB6F894DEBF0FBECDBF892B11F0B1
:10ABF0000C94F2490C94D64C8091DE2B9091DF2B73
:10AC000090FD02C00C94E94C81E090E00E94842009
:10AC10002B013C0180E090E00E9484209B01AC016C
:10AC2000C301B2010E94811E9F938F937F936F9304
:10AC300081EC98E09F938F931F9287E78F93C501D4
:10AC4000029641E050E04C0F5D1F840F951F9F93CB
:10AC50008F930E94549BA80EB91EC5010E946F4994
:10AC60000FB6F894DEBF0FBECDBF892B11F00C9448
:10AC7000F2490C94E94C8091DE2B9091DF2B90FDF2
:10AC800002C00C94FC4C81E090E00E9484202B01D7
:10AC90003C0180E090E00E9484209B01AC01C30154
:10ACA000B2010E94E21E9F938F937F936F938CEC6F
:10ACB00098E09F938F931F9287E78F93C501029629
:10ACC000E1E0F0E0EC0FFD1F8E0F9F1F9F938F932D
:10ACD0000E94549BA80EB91EC5010E946F490FB671
:10ACE000F894DEBF0FBECDBF892B11F00C94F24952
:10ACF0000C94FC4C8091DE2B9091DF2B90FD02C0D8
:10AD00000C940F4D81E090E00E9484202B013C01C7
:10AD100080E090E00E9484209B01AC01C301B2015D
:10AD20000E94431F9F938F937F936F938AED98E0C8
:10AD30009F938F931F9287E78F93C501029641E0FF
:10AD400050E04C0F5D1F840F951F9F938F930E94BF
:10AD5000549BA80EB91EC5010E946F490FB6F89406
:10AD6000DEBF0FBECDBF892B11F00C94F2490C94BD
:10AD70000F4D8091DE2B9091DF2B91FD02C00C9442
:10AD8000224D0E94C3199F938F937F936F938DEEF3
:10AD900098E09F938F931F9287E78F93C501029648
:10ADA000E1E0F0E0EC0FFD1F8E0F9F1F9F938F934C
:10ADB0000E94549BA80EB91EC5010E946F490FB690
:10ADC000F894DEBF0FBECDBF892B11F00C94F24971
:10ADD0000C94224DD10116968C9116971F928F9349
:10ADE00015968C9115971F928F9313968C911397AC
:10ADF0001F928F9312968C911F928F938EEF98E0F3
:10AE00009F938F931F9287E78F93C5010296E1E08E
:10AE1000F0E0EC0FFD1F8E0F9F1F9F938F930E94FA
:10AE2000549BA80EB91EC5010E946F490FB6F89435
:10AE3000DEBF0FBECDBF892B11F00C94F2490C94EC
:10AE4000344D779A8091550A9091560AA091570AED
:10AE5000B091580A92FD749A8091550A9091560AC1
:10AE6000A091570AB091580A82FD0CC080916202ED
:10AE700080FD08C081FD02C00C94604D1D9902C088
:10AE80000C94604D40E050E060E070E0CE0101962F
:10AE90000E94BC0A8091C71C90E020914C0A30911E
:10AEA0004D0A8217930710F40C94604D40E050E077
:10AEB00062E18CE092E00E94F75B0C94604D87E7C2
:10AEC0009AE00E94A35E892B11F40C94264E0E94F6
:10AED000716F8091620287FD02C00C94F2492B9A37
:10AEE0000C94F24920E030E0472D50E060E070E043
:10AEF00080E090E0A0E00E94499611F00C94AA4CEA
:10AF00000C94B04CC456DF4F0FB6F894DEBF0FBEA2
:10AF1000CDBFDF91CF911F910F91FF90EF90DF9008
:10AF2000CF90BF90AF909F908F907F906F905F90E9
:10AF30004F903F902F9008950C94605A4F925F92DB
:10AF40006F927F92AF92BF92CF92DF92EF92FF9279
:10AF50000F931F93CF93DF93CDB7DEB760970FB6F4
:10AF6000F894DEBF0FBECDBF6B010E94BB70E82F0F
:10AF7000F0E0EE0FFF1FE552F44E808191810196C3
:10AF8000918380838091550A9091560AA091570A27
:10AF9000B091580A81FD749840906202509063020B
:10AFA00060906402709065020E949D627C01FC01C9
:10AFB0008081982F92959F70913099F48F7051F401
:10AFC0008091BF1B9091C01B01969093C01B8093F2
:10AFD000BF1B38C1B60187EB94E30E94D459892B7B
:10AFE00051F08091BD1B9091BE1B01969093BE1BAA
:10AFF0008093BD1B27C1D301C2013EE0B695A79542
:10B00000979587953A95D1F7F82FF170AF2E86E98D
:10B010009AE00E94E65C8C01892B09F448C0B601D5
:10B02000C80102960E94D459892BE9F198014BE698
:10B030005AE060E074E6C8010F960E946A5FF7016B
:10B040009181F8018481981321C082858F5F828766
:10B050008091BB1B9091BC1B01969093BC1B80936D
:10B06000BB1B84E00E94BC63F801208530E02817F8
:10B07000390708F077C184E00E94BC63F80180873B
:10B08000F70180818F70F8018187DCC0F80112869A
:10B0900084E00E94BC63F8018087F70180818F7093
:10B0A000F801818760C1C8010E94925DB4CF84E03D
:10B0B00092E00E947A5C8C01892B09F4C3C0B6012E
:10B0C000C80102960E94CB59F70181818150F80195
:10B0D000848380E091E0A0E0B0E083879487A58737
:10B0E000B687128684E00E94BC63F8018087F7016E
:10B0F00080818F70F8018187B80186E99AE00E940B
:10B100004A5D98014BE65AE060E074E6C8010F968C
:10B110000E946A5FBB24B394F7018181F8018483A4
:10B12000F70180818F70F801878384E00E94BC63FF
:10B13000F801858383E00E94BC63F80186838781E0
:10B140008F3009F0B12CF7014180F8018481481A51
:10B15000512C612C712C86E0440C551C661C771C0C
:10B160008A95D1F72385348545855685A0ECB0E0D6
:10B170000E947D94BB27A92F982F872F480E591E18
:10B180006A1E7B1E4386548665867686A601B801B4
:10B19000C7010E94BC0A8091C71C90E020914C0A14
:10B1A00030914D0A8217930738F040E050E062E199
:10B1B0008CE092E00E94F75B80914C0A90914D0ADE
:10B1C000029708F44BC08091DE2B86FF2AC00E94B4
:10B1D0006368C70105960E942F68F70181811F925D
:10B1E0008F93F80186811F928F9385811F928F9391
:10B1F00086E299E09F938F931F9280E18F93CE0117
:10B2000001966C019F938F930E94549B82E00E9451
:10B210004968C6010E942F680FB6F894DEBF0FBEC2
:10B22000CDBF8091620290916302A0916402B091BF
:10B23000650297FD4DC080914C0A90914D0A02978E
:10B2400008F47AC08091550A9091560AA091570A45
:10B25000B091580A81FF89C0749A87C080916202B8
:10B2600090916302A0916402B091650296FFABCF0A
:10B27000AA2009F4A8CFF7018081982F9F709230FF
:10B28000E8F09150807F892B80838BE89AE00E94C0
:10B290009C578091B91B9091BA1B01969093BA1B51
:10B2A0008093B91B8091550A9091560AA091570A34
:10B2B000B091580A96FF87CF739885CF8091BF1BB6
:10B2C0009091C01B01969093C01B8093BF1B7BCFB6
:10B2D00088EA9BE12091A81B222309F4ACCF9F931D
:10B2E0008F9389E399E09F938F93CE0101963C0160
:10B2F0009F938F930E94919B6C01B301C7010296AB
:10B300000E94679A0F900F900F900F900F900F90E0
:10B31000009709F490CFEFEFCE1ADE0A8C0D9D1D39
:10B32000AC010196FA0120812032D1F362E186E17D
:10B3300092E00E94F75B7FCFBB2009F483CF82E0CD
:10B340008093F92F1092FB2F1092FA2F1093FD2F5C
:10B350000093FC2F49EF5FE262E18EE392E00E94EE
:10B36000F75B70CFA12CB12CD7CE60960FB6F894B6
:10B37000DEBF0FBECDBFDF91CF911F910F91FF9028
:10B38000EF90DF90CF90BF90AF907F906F905F90E5
:10B390004F9008950895FB012081FC012083FB015B
:10B3A0002181FC0121830895FC019081DB018C91B6
:10B3B000981309C021E090E0318111968C913813E7
:10B3C00020E0822F089580E090E00895BC0187EB93
:10B3D00094E30C94CB59DC011996ED91FC911A97EA
:10B3E0000280F381E02D309709F0099408950F93BE
:10B3F0001F93CF93DF9300D0CDB7DEB78C0188E1E8
:10B400000E94CF63BC01CE0101960E94CB59D801A6
:10B410001996ED91FC911A970190F081E02DBE01F3
:10B420006F5F7F4FC80109950F900F90DF91CF910B
:10B430001F910F910895EF92FF920F931F93CF9357
:10B44000DF938C01EB017A014EE053E00E94455AF4
:10B45000F801F286E18662E173E0CE01DF91CF91DF
:10B460001F910F91FF90EF900C949F5A0C945E5A8D
:10B47000CF93DF93EC0167EB74E388E10E94C5632F
:10B48000CE01DF91CF910C94605AEF92FF920F930F
:10B490001F93CF93DF938C01EB017A010E947B5ABB
:10B4A000F801F086E78266E173E0CE01DF91CF918B
:10B4B0001F910F91FF90EF900C949F5A0C94835A18
:10B4C0000C943175DC011796ED91FC911897019061
:10B4D000F081E02D0994DC011796ED91FC9118970D
:10B4E0000280F381E02D309709F0099408958AE9EC
:10B4F00092E10C94E25CFC0173836283BC018AE9F3
:10B5000092E10C944A5DBC018AE992E10C942B5DB6
:10B51000CF93DF93EC018AE992E10E94E65C009709
:10B5200049F0FC01228133812C173D0729F00E944C
:10B53000925DF5CF80E090E0DF91CF9108950F9379
:10B540001F93CF93DF938B010E94885AEC01892BC4
:10B5500031F01D830C83C8010E945F778E83DF91D9
:10B56000CF911F910F9108951F93CF93DF93DC012B
:10B570001496ED91FC9115973097E1F0162FEC01A0
:10B5800090939D1280939C1282E08887CD0106964D
:10B590000995082E000C990B0297029710F01338AA
:10B5A00039F4BE01CE01DF91CF911F910C94E45A82
:10B5B00081E08887DF91CF911F910895FC0120855C
:10B5C00020FD0C94B45A0895CF92DF92EF92FF922F
:10B5D0000F931F93CF93DF93E0909C12F0909D12F6
:10B5E000C0909E12D0909F12F601E817F90739F02B
:10B5F000309709F44BC00190F081E02DF6CF009711
:10B6000009F444C08B01EC018885882309F1188670
:10B61000C114D10461F0CC15DD0529F0AE0167E855
:10B62000C6010E94DE5AF601C080D180F1CFEC81C4
:10B63000FD81309769F0C017D10751F0D0939D126A
:10B64000C0939C1240E050E063E8CE010696099555
:10B65000E0919E12F0919F12CE17DF0741F488818E
:10B66000998190939F1280939E120CC0FC01309799
:10B6700049F0808191818C179D07C1F7888199815C
:10B6800091838083F0929D12E0929C12DF91CF9182
:10B690001F910F91FF90EF90DF90CF9008951F932F
:10B6A000CF93DF931092A812C0919E12D0919F1257
:10B6B00011E0209779F08985882341F01887198651
:10B6C00040E050E062E8CE010E94B45A0990D8816F
:10B6D000C02DEFCFDF91CF911F91089580914B1333
:10B6E00091E0980F90934B13089560919C12709184
:10B6F0009D120C94E45A8AE880934B1310924913DC
:10B7000010924A1310929F1210929E1210929D1244
:10B7100010929C1208958091A81281110E944F5B93
:10B7200050914A13552309F452C0E09149132E2F2A
:10B7300030E085E0E89FF0011124E755FD4E60817F
:10B740006093A712A181B281B093A612A093A51213
:10B75000838194819093A4128093A3122F5F3F4F13
:10B760002F71332720934913515050934A13009758
:10B7700031F580919E1290919F129093A212809326
:10B78000A1128091A1129091A212892B01F18091B6
:10B79000A81281110E944F5B4091A5125091A612F0
:10B7A0006091A7128091A1129091A2120E94DE5A7C
:10B7B000E091A112F091A21280819181DECF6138D7
:10B7C00019F421E0FC012087AD010E94DE5A80912E
:10B7D000A81220914A1390E0820F911D0895809144
:10B7E000A81220914A1390E0820F911D08959C01A8
:10B7F00090914A139032B9F0E0914913E90FEF713B
:10B80000E093A01285E0E89FF0011124E755FD4E7A
:10B81000608352834183348323839F5F90934A13D1
:10B8200080E090E0089581E090E00895CF93DF9369
:10B83000C0919C12D0919D120E94DE5AD0939D120D
:10B84000C0939C12DF91CF910895AB0130919E126D
:10B8500020919F12E32FF22FE817F907B1F03097EC
:10B8600021F00190F081E02DF7CF009771F0FC01FD
:10B870003083218390939F1280939E1221E0208732
:10B880001782168261E80C94165C0895009749F0BF
:10B89000FC0120852150223020F421E021872093D3
:10B8A000A812089521E030E0FC018085811102C0DA
:10B8B00020E030E0C9010895CF93DF93EC014A8185
:10B8C0005B8160E070E08C819D810E94369A2A81C4
:10B8D0003B8188819981289FA001299F500D389F25
:10B8E000500D112460E070E08E819F81DF91CF9137
:10B8F0000C94369AFC018281938120E030E0281775
:10B900003907D1F0A481B581A20FB31F4C91411129
:10B9100010C081E08C9380819181289FA001299F94
:10B92000500D389F500D112486819781840F951FEB
:10B9300008952F5F3F4FE3CF80E090E00895FC0132
:10B94000868197814281538120E030E024173507BA
:10B95000D1F08617970781F4A481B581A20FB31F98
:10B960008C91181614F481508C9384819581FC017C
:10B97000E20FF31F80810895A081B1818A0F9B1F80
:10B980002F5F3F4FE3CF8FEF0895FC012681378172
:10B9900062177307A0F0A081B18142815381A49FF7
:10B9A000C001A59F900DB49F900D1124280F391F41
:10B9B00081E090E06217730720F080E0089580E056
:10B9C00090E00895FC01118210820895FC018081AD
:10B9D00091810895FB0120813181FC013183208315
:10B9E0000895DC01ED91FC91309741F080819181C7
:10B9F000009711F0FC01FACFCF01089580E090E0AC
:10BA00000895DC01ED91FC9111973097A9F0208108
:10BA10003181232B21F41D921C92CF010895A08126
:10BA2000B1818D919C911197892B11F0FD01F7CF78
:10BA300011821082CD01089580E090E00895DC012C
:10BA4000ED91FC911197309721F0208131812D9358
:10BA50003C93CF010895DC01ED91FC913097C9F042
:10BA6000A0E0B0E0E617F70761F4FB012081318127
:10BA7000109709F4DC012D933C93FB011182108295
:10BA8000089520813181DF012115310511F0F9017F
:10BA9000E9CF08950F931F93CF93DF938C01EB01B0
:10BAA0000E942B5D19821882C8010E94F15C0097E8
:10BAB00011F4F80101C0FC01D183C083DF91CF9163
:10BAC0001F910F9108950F931F93CF93DF93EC0174
:10BAD0008B010E942B5D88819981F801918380837D
:10BAE00019830883DF91CF911F910F910895DC0195
:10BAF000ED91FC9180E090E0309729F00196019063
:10BB0000F081E02DF9CF0895FB01309719F4BA01C7
:10BB10000C94635D80819181DA018D939C935183B4
:10BB200040830895009721F0FC0180819181089560
:10BB300080E090E0089580914E1390914F13892BEF
:10BB400029F410924D1310924C1308950E94B96C71
:10BB5000E0914E13F0914F13228133814081518146
:10BB6000240F351F281B390B0480F581E02D3097F9
:10BB700069F06281738140815181460F571F481BD4
:10BB8000590B4217530780F79A01EECF820F931F8C
:10BB900090934D1380934C13089580E992E00C9498
:10BBA000465CEF92FF920F931F93CF93DF938C012C
:10BBB000FC0180819181009799F08A359105D9F037
:10BBC000F8011182108283E068C086819781841712
:10BBD000950709F049C00480F581E02D3097A9F759
:10BBE00010924F1310924E138AE590E0F801918362
:10BBF000808381E052C0673891F16238A9F7C09123
:10BC00004E13D0914F13E12CF12C209769F3CE0104
:10BC10000E94287B892BF1F0AE0168E88E819F811C
:10BC20000E94F75B892BA1F41F821E828C819D816B
:10BC3000E114F10421F0F7019583848304C090930B
:10BC40004F1380934E131D821C820E949B5DD7CFA1
:10BC50000E94CD5D7E010C80DD81C02DD6CFE091AC
:10BC60004E13F0914F13BACFF0934F13E0934E134E
:10BC7000A481B581109709F4B7CF16968D919C9148
:10BC800017978417950739F414968D919C91159701
:10BC900095838483EDCFFD01EBCFDF91CF911F9191
:10BCA0000F91FF90EF900895CF93DF93EC010E94E6
:10BCB000CD5D2E813F8190914E1380914F13232BA8
:10BCC00059F0E92FF82F309739F0EC17FD0781F084
:10BCD0000480F581E02DF7CF20919C1230919D12C8
:10BCE0003F832E839C838D83D0934F13C0934E1339
:10BCF000DF91CF910C949B5DCF93DF93EC010E9479
:10BD0000087BCE01DF91CF910C94545ECF93DF93EB
:10BD1000EC010E94147BCE01DF91CF910C94545E14
:10BD2000CF93DF93EC010E941E7BCE01DF91CF9178
:10BD30000C94545EFC0120813181620F731F71836A
:10BD400060830C949B5D21E030E0FC01868197814B
:10BD5000892B11F020E030E0C9010895FC01228117
:10BD6000338180819181820F931F0895FC0180812E
:10BD70009181089581E090E020914E1330914F130E
:10BD8000232B11F480E090E0089580914E13909160
:10BD90004F13892B29F080914C1390914D130895E6
:10BDA00080E090E00895CF93DF93EC01E0914E1393
:10BDB000F0914F138E179F0769F48C819D819093AA
:10BDC0004F1380934E130DC0848195818C179D076E
:10BDD00021F0FC013097C1F706C08C819D819583CD
:10BDE00084830E949B5D1D821C821F821E82DF91C4
:10BDF000CF910895EF92FF920F931F93CF93DF930C
:10BE00008C017A01FC0180819181009741F08B3493
:10BE1000910501F1F8011182108283E048C081E5AB
:10BE200093E10E94E65CEC01209751F06C817D81EA
:10BE3000CE0102960E947C5E0990D881C02DF4CF7D
:10BE400081E0809350138BE490E0F801918380832C
:10BE500081E02DC06838E1F781E593E10E94E65C5E
:10BE6000EC01209781F3CE010296E816F906D9F489
:10BE7000BE0181E593E10E942B5DE0909C12F09061
:10BE80009D128A859B8590939D1280939C12EC85D0
:10BE9000FD85309719F08E859F850995F0929D124A
:10BEA000E0929C12D0CF0990D881C02DDACFDF91DB
:10BEB000CF911F910F91FF90EF9008951092501322
:10BEC00081E593E10E94E25C60E070E08AE992E043
:10BED0000C94255C0F931F93CF93DF93EC0100919B
:10BEE0009C1210919D121B870A875D874C873F87A4
:10BEF0002E8780915013882379F08AE992E09093FD
:10BF00009D1280939C12CE0102960E947C5E10933B
:10BF10009D1200939C1202C07D836C83BE0181E55B
:10BF200093E10E942B5DBE0181E593E1DF91CF910A
:10BF30001F910F910C944A5D0F931F93CF93DF9342
:10BF4000EC0180915013882391F000919C12109184
:10BF50009D128AE992E090939D1280939C12CE01EB
:10BF600002960E94865E10939D1200939C12BE0161
:10BF700081E593E10E942B5DBE0181E593E1DF91B4
:10BF8000CF911F910F910C944A5D0F931F93CF9304
:10BF9000DF93EC0180915013882391F000919C1263
:10BFA00010919D128AE992E090939D1280939C12C9
:10BFB000CE0102960E94905E10939D1200939C12F7
:10BFC000BE0181E593E10E942B5DBE0181E593E115
:10BFD000DF91CF911F910F910C944A5DCF93DF9326
:10BFE000EC0180915013882329F0CE0102960E9423
:10BFF000D35E04C01F821E8219861886BE0181E5A9
:10C0000093E1DF91CF910C942B5DCF93DF9320913F
:10C010005013222329F00296DF91CF910C94A35E56
:10C02000EC0181E593E10E94E65C009739F08C1702
:10C030009D0739F0FC0180819181F7CF81E090E08C
:10C0400002C080E090E0DF91CF9108952F923F925F
:10C050004F925F926F927F928F929F92AF92BF9218
:10C06000CF92DF92EF92FF920F931F93CF93DF93C4
:10C07000CDB7DEB7E8970FB6F894DEBF0FBECDBFE1
:10C08000E6EAF6E3AAEEB6E32C9111963C911197FD
:10C0900012964C91129713965C91A6EEB6E35C90C3
:10C0A00011964C90119712963C90129713962C90E3
:10C0B00094AC8090E3367090E4366090E53680ADC5
:10C0C000898391AD9A8382AD8B8393AD9C8384A940
:10C0D0008D8395A99E8386A98F8397A9988780A928
:10C0E000898791A99A8782A98B8793A99C8784A520
:10C0F0008D8795A59E8786A58F8797A5988B80A508
:10C10000898B91A59A8B82A58B8B93A59C8B84A1FF
:10C110008D8B95A19E8B86A18F8B97A1988F80A1E7
:10C12000898F91A19A8F82A18B8F93A19C8F848DEF
:10C130008D8F958D9E8F868D8F8F978D98A3808DF7
:10C1400089A3918D9AA3828D8BA3938D9CA38489BF
:10C150008DA395899EA386898FA3978998A78089A7
:10C1600089A791899AA782898BA793899CA784859F
:10C170008DA795859EA786858FA7978598AB808587
:10C1800089AB91859AABB284A384F480E580D68094
:10C19000C78080818FAB918198AF128103812BABD7
:10C1A0003CAB4DAB5EAB0E94E56C5EA95F934DA9C5
:10C1B0004F933CA93F932BA92F932F923F924F92DD
:10C1C0005F926F927F928F929F922C812F932B81FF
:10C1D0002F932A812F9329812F9328852F932F81A5
:10C1E0002F932E812F932D812F932C852F932B8589
:10C1F0002F932A852F9329852F9328892F932F8575
:10C200002F932E852F932D852F932C892F932B8958
:10C210002F932A892F9329892F93288D2F932F8944
:10C220002F932E892F932D892F932C8D2F932B8D28
:10C230002F932A8D2F93298D2F9328A12F932F8D04
:10C240002F932E8D2F932D8D2F932CA12F932BA1D8
:10C250002F932AA12F9329A12F9328A52F932FA1A4
:10C260002F932EA12F932DA12F932CA52F932BA588
:10C270002F932AA52F9329A52F9328A92F932FA574
:10C280002F932EA52F932DA52F93AF92BF922AA95E
:10C290002F9329A92F93CF92DF92EF92FF920F93C2
:10C2A0001F9328AD2F932FA92F939F938F937F9345
:10C2B0006F938091B8341F928F93E7EBF4E3808102
:10C2C0001F928F9385E291E19F938F930E94FC9A36
:10C2D000EEEEF6E324A535A546A557A550A441A446
:10C2E00032A423A4848D8983858C768C678C908D71
:10C2F0009A83818D8B83928D9C83838D8D8394898A
:10C300009E8385898F839689988787898987908975
:10C310009A8781898B8792899C8783898D87948569
:10C320009E8785858F879685988B8785898B908555
:10C330009A8B81858B8B92859C8B9384D480C580CE
:10C34000B680A78010810181F280E3800FB6F89457
:10C35000DEBF0FBECDBF2BAB3CAB4DAB5EAB0E9487
:10C36000E56C5EA95F934DA94F933CA93F932BA920
:10C370002F932F923F924F925F926F927F928F9264
:10C3800029812F932D812F932C812F932B812F93F4
:10C390002A812F9329852F9328852F932F812F93DF
:10C3A0002E812F932D852F932C852F932B852F93C3
:10C3B0002A852F9329892F9328892F932F852F93AF
:10C3C0002E852F939F922C892F932B892F932A8927
:10C3D0002F93AF92BF92CF92DF92EF92FF920F9383
:10C3E0001F939F938F937F936F938091B8341F9285
:10C3F0008F93E7EBF4E380811F928F9386EB90E1BC
:10C400009F938F930E94FC9A0FB6F894DEBF0FBEE5
:10C41000CDBFE8960FB6F894DEBF0FBECDBFDF915B
:10C42000CF911F910F91FF90EF90DF90CF90BF9031
:10C43000AF909F908F907F906F905F904F903F90C4
:10C440002F90089580E3809307140895CF93DF938E
:10C450006091071470E0C0E3D0E0C61BD70B6B5AA5
:10C460007C4EAE010E942D9ACE01DF91CF910895AE
:10C47000CF92DF92EF92FF920F931F93CF93DF93B0
:10C48000C0900A14D0900B146091071470E0E6017C
:10C49000E096C61BD70BC138D105E0F47C0100E360
:10C4A00010E0061B170B6B5A7C4EA8010E942D9AB8
:10C4B0006091531370915413809108149091091452
:10C4C000680F791FA601C701800F911F0E942D9A46
:10C4D000CE0102C080E090E0DF91CF911F910F91DB
:10C4E000FF90EF90DF90CF90089590910714890FFF
:10C4F00080930714089520910A1430910B14281783
:10C50000390798F04091081450910914480F591FA9
:10C510005093091440930814281B390B30930B14C3
:10C5200020930A1481E090E0089580E090E008955F
:10C5300090930B1480930A1408958091081490919D
:10C5400009148B579C4E08958091071490E08B5AE4
:10C550009C4E089581E090E0209153133091541344
:10C560002558334111F480E090E008950E94AA62BA
:10C57000892B61F0609153137091541340910A1408
:10C5800050910B1485E893E10C942D9A2091081496
:10C590003091091421153105B9F080910A14909158
:10C5A0000B14C096E5E8F3E1AF0145555341481738
:10C5B000590734F4DF01A20FB31F4C914193F4CF1C
:10C5C00010920914109208140895809153139091B9
:10C5D0005413089580910A1490910B14089590912A
:10C5E000071480E3891B08958091071490E3981B3A
:10C5F00020910A1430910B14A901490F511DCA0151
:10C6000008950F931F93CF938C01C09107148C2F23
:10C6100090E0801791076CF00E94F462800F911FE8
:10C620008138910530F4C01BC093071481E090E07D
:10C6300002C080E090E0CF911F910F910895CF93B9
:10C64000DF93E1ECF4E31192119284E3E13FF80708
:10C65000D1F7C9EBD4E36CE073E0CE010E94CB5973
:10C66000229684E3C13CD807B1F7DF91CF910895BA
:10C67000109209141092081410920B1410920A14BC
:10C6800080E38093071485E893E19093541380939B
:10C6900053130C941F63EF92FF920F931F93CF934A
:10C6A000DF9300D0CDB7DEB78C0169837A830E9417
:10C6B00038636981E62E7A81F72E81E8E816F10465
:10C6C00018F080E8E82EF12CA701B80180915313EF
:10C6D000909154130E942D9AF0920B14E0920A1438
:10C6E000C7010F900F90DF91CF911F910F91FF9095
:10C6F000EF9008950F931F93CF93DF938C01EB017D
:10C700000E9438631093541300935313D0930B1467
:10C71000C0930A14DF91CF911F910F910895DC010E
:10C7200090E3E1ECF4E301900D929A95E1F788E053
:10C73000E9EBF4E3DB0101900D928A95E1F70895AE
:10C74000FC0190E3A1ECB4E301900D929A95E1F71E
:10C7500088E0FB01A9EBB4E301900D928A95E1F723
:10C760000895E82FF0E0EE0FFF1FEF53FB4C7183AD
:10C77000608381E090E00895E82FF0E0EE0FFF1F66
:10C78000EF53FB4C80819181089590E0880F991FB1
:10C7900087579B4C0E94CB5981E090E0089590E030
:10C7A000880F991F87579B4C08958115910511F0AB
:10C7B0000197F1F70895E091F434F091F534908108
:10C7C0008091F33489230895E091F134F091F234AB
:10C7D00090818091F334892B8083E091F634F0913D
:10C7E000F73490818091F334892B80830895E09110
:10C7F000F134F091F23490818091F3348095892363
:10C800008083E091F634F091F73490818091F33495
:10C8100080958923808308951F93CF93DF93E091C0
:10C82000F134F091F23490818091F3348095892332
:10C830008083E091F634F091F73490818091F33465
:10C84000892B80838FEB93E00E94D5631FB7F89408
:10C85000E091F634F091F73490818091F334809533
:10C860008923808383E890E00E94D563E091F434CB
:10C87000F091F534D081C091F3341FBF78948BE3ED
:10C8800093E00E94D563E091F434F091F534808117
:10C890009091F334982319F08D2F8C2301C081E0FF
:10C8A000DF91CF911F9108955093F7344093F63460
:10C8B0007093F2346093F1349093F5348093F434B0
:10C8C00081E001C0880F2A95EAF78093F3340C9435
:10C8D0000C64CF93DF93C82FDFB7F894E091F63460
:10C8E000F091F73490818091F334892B808383E039
:10C8F00090E00E94D563CC2351F0E091F634F091A2
:10C90000F73490818091F33480958923808387E187
:10C9100090E00E94D563E091F434F091F534908179
:10C920008091F334892309F4C0E089E590E00E9406
:10C93000D563E091F634F091F73490818091F3342F
:10C94000809589238083DFBF8BE390E00E94D563CD
:10C950008C2FDF91CF910895CF93DF93C82FD8E02C
:10C960008C2F81700E946964C6958111C068D15076
:10C97000B9F78C2FDF91CF9108958FEF0C94AC64B1
:10C98000DF92EF92FF920F931F93CF93DF93E82EE6
:10C990008B010E940C64811135C080EF0E94AC6451
:10C9A000D0E0C0E488EFD82EDC0E81E00E946964FC
:10C9B000F82E81E00E946964882319F0FF2071F04D
:10C9C00023C0F1100BC0CE1530F0F801808180FF3C
:10C9D00005C0EC1619F0DC2FFF24F3948F2D0E9474
:10C9E0006964F80190819695FF2011F09068F80134
:10C9F0009083C150CD11D9CF0F5F1F4FC111D2CF3E
:10CA00008D2F03C08FEF01C08EEFDF91CF911F916B
:10CA10000F91FF90EF90DF900895EF92FF921F9398
:10CA2000CF93DF93182FEB010E940C64209771F0D5
:10CA300085E50E94AC647E0188E0E80EF11C8991D6
:10CA40000E94AC64CE15DF05D1F703C08CEC0E94C8
:10CA5000AC64812FDF91CF911F91FF90EF900C94E8
:10CA6000AC640F931F93CF93DF93DB01EC9111968E
:10CA70009C911197F0E0F92B803179F4EE7F63E01F
:10CA8000EE0FFF1F6A95E1F716969C9116976CE0E2
:10CA900070E0691B7109E60FF71FF7FF07C091E00F
:10CAA000EA019883F195E195F10902C0EA01188243
:10CAB000883279F414968C91982F9076903649F0BC
:10CAC00086FF02C0EE7F05C085FF02C0EC7F01C07B
:10CAD000E87FCF0144E0969587954A95E1F7D90123
:10CAE0008C93EF70E801E88380E0DF91CF911F9194
:10CAF0000F9108950F931F93CF93DF93EC018B0158
:10CB0000B80188810E94C06488839FEF980F9D3F81
:10CB100030F4F8019081983211F0903189F7DF916B
:10CB2000CF911F910F910895CF93DF93EC010E9455
:10CB30000C64BE0184EB0E940D6581E00E94696473
:10CB4000C82F0E940C6481E0C11101C080E0DF9118
:10CB5000CF9108951F93CF93DF9300D0CDB7DEB769
:10CB6000182F69837A830E940C640E94DB636981B9
:10CB70007A81882341F084E40E940D65113029F008
:10CB80000E94E46302C082E001C080E00F900F9039
:10CB9000DF91CF911F9108955F926F927F928F9254
:10CBA0009F92AF92BF92CF92DF92EF92FF920F933C
:10CBB0001F93CF93DF93CDB7DEB729970FB6F894C5
:10CBC000DEBF0FBECDBF5C014B013A0189010E945F
:10CBD0000C64B5018EEB0E940D65CE0101967C01BF
:10CBE0006C0199E0592E5E0C0E94BD64F6018193A0
:10CBF0006F015E12F9CF69E070E0C7010E94A27F69
:10CC0000D82E811108C09301A401B701F5018081DC
:10CC10000E94316502C083E0D82E8D2D29960FB673
:10CC2000F894DEBF0FBECDBFDF91CF911F910F9162
:10CC3000FF90EF90DF90CF90BF90AF909F908F903C
:10CC40007F906F905F9008956F927F928F929F92E6
:10CC5000AF92BF92CF92DF92EF92FF920F931F930A
:10CC6000CF93DF93CDB7DEB729970FB6F894DEBF29
:10CC70000FBECDBF782E5B014A01890160E070E0F4
:10CC80008EEB0E940D65CE0101967C016C0199E04E
:10CC9000692E6E0C0E94BD64F60181936F016E12C5
:10CCA000F9CF69E070E0C7010E94A27FD82E811100
:10CCB00007C09401A501B701872D0E94316502C00C
:10CCC00083E0D82E8D2D29960FB6F894DEBF0FBEC7
:10CCD000CDBFDF91CF911F910F91FF90EF90DF902B
:10CCE000CF90BF90AF909F908F907F906F9008955E
:10CCF0000F931F93CF93DF93CDB7DEB728970FB66F
:10CD0000F894DEBF0FBECDBF182F062F98E0E8E1E4
:10CD1000F3E0DE01119601900D929A95E1F7242F30
:10CD2000440F330B41E752E0249FC001259F900D33
:10CD3000349F900D112464E670E00E94FA9384E61B
:10CD4000089F600D711D1124FE01319688E08E0F41
:10CD5000419150E02417350719F46F5F7F4F02C0EF
:10CD60008E13F6CF112319F0719561957109CB01DE
:10CD700028960FB6F894DEBF0FBECDBFDF91CF91DE
:10CD80001F910F9108950F931F93CF93DF93CDB70A
:10CD9000DEB72B970FB6F894DEBF0FBECDBF182FAE
:10CDA000092F682F792F88E0810F0E94AA658823B8
:10CDB00019F084E391E243C066E471E48FE090E00F
:10CDC0000E942A679E01275F3F4FAE01465F5F4F7B
:10CDD000BE01655F7F4F812F902F0E94CC6581112E
:10CDE000E8CF88E0E8E1F3E0DE01119601900D92D2
:10CDF0008A95E1F7298541E752E0249FC001259FEC
:10CE0000900D112464E670E00E94FA938A8594E6FE
:10CE1000899F600D711D1124FE01319688E08E0FEF
:10CE20009191291303C06F5F7F4F02C08E13F8CF1B
:10CE30008B85882319F0719561957109CB012B962B
:10CE40000FB6F894DEBF0FBECDBFDF91CF911F911B
:10CE50000F910895DC01CB0181159105A105B10564
:10CE600029F081509040A040B040D9F708959B012F
:10CE7000AC011092B90060E072E18AE790E00E9494
:10CE80000E94DA01C9014097A109B109B695A79599
:10CE9000979587958093B800089594EA9093BC0085
:10CEA00040EA56E861E070E09091BC0097FD07C051
:10CEB0004150510961097109B9F781E008959091D4
:10CEC000B900987F983011F09031B9F78093BB008A
:10CED00084E88093BC0080EA96E8A1E0B0E020916D
:10CEE000BC0027FD05C00197A109B109C1F7E5CF35
:10CEF0008091B900887F883111F08034F1F680E0AC
:10CF0000089524EA34E844E92093BC009091BC00E1
:10CF100097FFFCCF9091B900987F983011F0903135
:10CF200099F78093BB003093BC009091BC0097FFB1
:10CF3000FCCF9091B900987F903211F0983539F478
:10CF40004093BC009091BC0094FDFCCFDDCF0895D0
:10CF50000C944D6784E98093BC008091BC0084FDF3
:10CF6000FCCF08958093BB0084E88093BC0080913F
:10CF7000BC0087FFFCCF9091B900987F81E0983288
:10CF800009F480E0089584EC8093BC008091BC009B
:10CF900087FFFCCF8091BB00089584E88093BC009C
:10CFA0008091BC0087FFFCCF8091BB000895CF9398
:10CFB000DF93FC017096EC01A991CE01A0933F0193
:10CFC000CE17DF07C1F780913C018F7D80933C0134
:10CFD00080913C01877F80933C01DB015096FB01EF
:10CFE000819180933E01EA17FB07D1F780913C01C4
:10CFF000806880933C0180913D0180FFFCCF4051CF
:10D00000510980913C01806280933C0180913C01F8
:10D01000877F80933C01141615069CF4FB018191D7
:10D0200080933E01EA17FB07D1F780913C018068AD
:10D0300080933C0180913D0180FFFCCF405151091C
:10D04000EACFF901C901409620913E012193E817EA
:10D05000F907D1F781E090E0DF91CF9108950F9328
:10D060001F93CF93DF93EC018CE70E9481678CE7DD
:10D070000E94B2678E01005F1F4F89910E94B267C4
:10D08000C017D107D1F7DF91CF911F910F910C9469
:10D09000AA67813019F440E050E002C040EC50E053
:10D0A00060E070E08CE790E00C949313813019F409
:10D0B0004EE050E002C048E050E060E070E08CE7F5
:10D0C00090E00C94931341E050E060E070E08CE756
:10D0D00090E00E9493136AE67AE080E090E00C947E
:10D0E0002A6748E350E060E070E08CE790E00E943F
:10D0F000931349E350E060E070E08CE790E00E9419
:10D10000931344E150E060E070E08CE790E00E940F
:10D11000931348E750E060E070E08CE790E00E94F5
:10D1200093134EE550E060E070E08CE790E00E94E1
:10D1300093134DE650E060E070E08CE790E00E94D1
:10D1400093136CE17AE186E090E00E942A674CE05C
:10D1500050E060E070E08CE790E00E94931341E0C3
:10D1600050E060E070E08CE790E00E94931346E0AE
:10D1700050E060E070E08CE790E00E9493136AE674
:10D180007AE080E090E00C942A67CF93DF93CDB7EC
:10D19000DEB7A2970FB6F894DEBF0FBECDBF81E118
:10D1A000EDECF9E0DE01529601900D928A95E1F7DF
:10D1B00081E1EEEDF9E0DE01119601900D928A9584
:10D1C000E1F70E947168CE0142960E942F6882E0CA
:10D1D0000E9449686AE67AE080E090E00E942A674F
:10D1E000CE0101960E942F6860E17EEA88E290E01D
:10D1F0000E942A6780E00E94566860E17EEA88E229
:10D2000090E00E942A674EE050E060E070E08CE71A
:10D2100090E00E949313A2960FB6F894DEBF0FBE63
:10D22000CDBFDF91CF910895CF92DF92EF92FF9221
:10D230000F931F93CF93DF9300D01F92CDB7DEB72C
:10D24000042F122F213061F0223031F0243031F0E0
:10D25000283031F493E005C091E003C092E001C0B2
:10D2600090E0E82FF0E08160F82E0C3009F4E0C087
:10D270000E3011F49460DCC0003111F49860D8C015
:10D28000023109F0D5C0613009F4B7C09C6062304A
:10D2900011F4906207C0633011F4906403C06430ED
:10D2A00009F490669068692F70E023E030E0AE01E9
:10D2B0004F5F5F4FCF010E94AA1369E07AE180E0DF
:10D2C00090E00E942A678F2D0E944D670E94C367DD
:10D2D00089830E94C3678A83023119F40E94C3675D
:10D2E0008B830E94C36787FDF1CF0E94CD670E94A8
:10D2F000AA6769E07AE180E090E00E942A678F2DBA
:10D300000E944D670E94C36789830E94C3678A8316
:10D31000023119F40E94CD678B830E94CD670E9471
:10D32000AA6769812A81023139F5862F90E0A0E051
:10D33000B0E04B81DC019927882730E0322F22278B
:10D34000820F931FA11DB11D61FF09C0840F911DA4
:10D35000A11DB11DBC01CD018C6F9F6F06C0BC012A
:10D36000CD01640F711D811D911D0E94039120E864
:10D370003FEF4FEF57E41FC070E0762F6627620F34
:10D38000711D072E000C880B990B0E9403910C3025
:10D3900029F420E030EE4FEF54E40DC00E3029F4B4
:10D3A00020E038EF4FEF55E406C0003131F420E0C3
:10D3B0003EEF4FEF56E40E944F902FE632E143E0FC
:10D3C00050E40E94FB926B017C01612F70E080E0D1
:10D3D00090E00E9403919B01AC01C701B6010E943D
:10D3E0004F900F900F900F90DF91CF911F910F9161
:10D3F000FF90EF90DF90CF9008959C68692F70E0C8
:10D4000023E030E0AE014F5F5F4FCF010E94AA13CF
:10D4100069E07AE180E090E00E942A678F2D0E9407
:10D420004D670E94C36789830E94C3678A8356CF72
:10D43000613009F02CCF9068692F70E023E030E074
:10D44000AE014F5F5F4FCF010E94AA1369E07AE1FE
:10D4500080E090E00E942A678F2D0E944D670E9415
:10D46000C36789830E94C3678A833BCFE6E4F1E008
:10D4700090812081308180819295969596959370C8
:10D4800022952F70922B892B232F22952F70822B80
:10D4900008950F931F93CF93DF9300D0CDB7DEB7DE
:10D4A00046E06CE080E00E947B6D89E18093C400DF
:10D4B0001092C50082E08093C00080E00E940B6E55
:10D4C0000E94A96C84B784B784B784B784B78FEE01
:10D4D00099E09F938F9382E792E19F938F930E94AD
:10D4E000FC9A0E94DC7B0E947B5B60E070E080E93C
:10D4F00092E00E94255C0E945E5FE0912003F09123
:10D50000210309950E94366A90E00E94187CCE01A2
:10D5100001960E94D76B0F900F900F900F90882369
:10D5200041F082E592E19F938F930E94FC9A0F90C5
:10D530000F90CE0101960E94E6590E94E56B8C0186
:10D540000E94E16BAE014F5F5F4FB8010E94DD703A
:10D550000E94476B0E94BE700E94E96B0E94167287
:10D5600085E492E19F938F930E94FC9A8A811F9297
:10D570008F9301E412E11F930F930E94FC9A89811B
:10D580001F928F931F930F930E94FC9A8FE392E157
:10D590009F938F930E94FC9A0E941C7CE0915D03F4
:10D5A000F0915E030995E0914F03F09150030995C6
:10D5B000E0913603F091370309950E941D72182FF0
:10D5C0000E94BB701F921F931F928F9380915C03E8
:10D5D0008F9380915B038F9380914E038F93809103
:10D5E0004D038F9384E292E19F938F930E94FC9A64
:10D5F000E0916703F09168030FB6F894DEBF0FBEA9
:10D60000CDBF309791F00995BC0180E890E00E9471
:10D61000E6937F936F9381E192E19F938F930E94B2
:10D62000FC9A0F900F900F900F908FE092E19F93D4
:10D630008F930E94FC9A60E070E086EE92E00E9478
:10D64000255C8AEF92E00E94EC7A87E092E19F935A
:10D650008F930E94FC9A0F900F900F900F900F9055
:10D660000F90DF91CF911F910F9108957F936F934A
:10D670009F938F9381E092E19F938F930E94FC9AF6
:10D680000F900F900F900F900F900F900895DF92D2
:10D69000EF92FF920F931F93CF93DF93CDB7DEB737
:10D6A000A0970FB6F894DEBF0FBECDBF83E690E023
:10D6B0000E94FA9D182F282F35EF380F303108F0CF
:10D6C000982F9095291709F463C08DE892E19F93F4
:10D6D0008F930E94FC9AE2EDF2E18E010F5F1F4FE3
:10D6E0000F900F90D801D02EE12EF02E88E0800F01
:10D6F00094919D9331968A13FBCFF89448E050E0C3
:10D700006FE770E0C8010E94009EE4ECF2E1D801EE
:10D710008EE08F0D94919D9331968A13FBCF4EE04E
:10D7200050E061E770E0C8010E94009EEAEBF2E180
:10D730002AE02F0D8491D8018D938D0131962A1303
:10D74000F9CF4AE050E067E670E08D2D9E2D0E94F3
:10D75000009E6DEC7BEA81E690E00E94189E60E0FE
:10D7600070E08FE590E00E94189E60E08EE590E00A
:10D770000E940A9E60E070E085E690E00E94189E9C
:10D780001AE16AE175EE83E690E00E94189E7894B3
:10D79000812FA0960FB6F894DEBF0FBECDBFDF91EC
:10D7A000CF911F910F91FF90EF90DF900895F89423
:10D7B00042E050E06FE770E00E94E29D789480E0E4
:10D7C000089581E690E00C94FA9D8FE590E00C942A
:10D7D000FA9D8EE590E00C94F29D0F931F930091BB
:10D7E0000235109103352091043530910535482FCD
:10D7F00050E060E070E0DB01CA01800F911FA21FC2
:10D80000B31F8093023590930335A0930435B093F2
:10D8100005358091FE349091FF34A0910035B09190
:10D820000135840F951FA61FB71F8093FE34909378
:10D83000FF34A0930035B09301358091A236882340
:10D84000A1F08091FA349091FB34A091FC34B09116
:10D85000FD34480F591F6A1F7B1F4093FA345093C1
:10D86000FB346093FC347093FD341F910F91089545
:10D870001F920F920FB60F9211240BB60F922F9397
:10D880003F934F935F936F937F938F939F93AF9348
:10D89000BF93EF93FF9380910E1490910F14019614
:10D8A00090930F1480930E1480910D148F5F8093CA
:10D8B0000D148038A9F410920D14809102359091C6
:10D8C0000335A0910435B09105350196A11DB11D18
:10D8D0008093023590930335A0930435B0930535BA
:10D8E0008091A2368823E1F080910C148F5F8093A1
:10D8F0000C148038A9F410920C148091FA34909191
:10D90000FB34A091FC34B091FD340196A11DB11DF2
:10D910008093FA349093FB34A093FC34B093FD349D
:10D920000E94BA5E892B11F00E94CD5DFF91EF91AC
:10D93000BF91AF919F918F917F916F915F914F9127
:10D940003F912F910F900BBE0F900FBE0F901F9025
:10D950001895F8941092B60016BC83EF87BD82E04C
:10D9600084BD94E095BD95B395BB80936E0078948B
:10D97000089580910E1490910F1420910E143091FF
:10D980000F1482179307A9F70895009741F022E337
:10D9900030E0000021503109E1F70197F6CF0895FA
:10D9A0000F931F93CF93DF93EC010E94B96C8C010E
:10D9B0000E94B96C801B910B8C179D07C8F3DF91F7
:10D9C000CF911F910F91089508950F931F93609128
:10D9D00002357091033580910435909105350091A1
:10D9E00002351091033520910435309105356017CB
:10D9F00071078207930759F71F910F9108951F929E
:10DA00000F920FB60F9211241092BC020F900FBE0E
:10DA10000F901F9018951F920F920FB60F9211241E
:10DA20000BB60F922F933F934F935F936F937F9318
:10DA30008F939F93AF93BF93EF93FF93E091B202C5
:10DA4000F091B3028081E091BD02F091BE02309767
:10DA500009F00995FF91EF91BF91AF919F918F913F
:10DA60007F916F915F914F913F912F910F900BBEDE
:10DA70000F900FBE0F901F9018951F920F920FB628
:10DA80000F9211241092C9020F900FBE0F901F9099
:10DA900018951F920F920FB60F9211240BB60F928A
:10DAA0002F933F934F935F936F937F938F939F93A6
:10DAB000AF93BF93EF93FF93E091BF02F091C00249
:10DAC0008081E091CA02F091CB02309709F009956C
:10DAD000FF91EF91BF91AF919F918F917F916F9146
:10DAE0005F914F913F912F910F900BBE0F900FBE02
:10DAF0000F901F9018952DE0829FC0011124FC010A
:10DB0000EE54FD4FA281B3811C92A481B5816C9328
:10DB1000A681B78188ED8C93A085B1854C93128640
:10DB20001486138608952DE0829FC0011124FC0104
:10DB3000EE54FD4F81E08287A081B1816C933A96CB
:10DB400080818111FDCF08951F93CF93DF93182F0C
:10DB5000EB01FE019491992339F0FE016491812F2C
:10DB60000E94936D2196F5CFDF91CF911F9108957B
:10DB70001F93CF93DF93182FEB019881992369F0BE
:10DB80009A3021F46DE0812F0E94936D69916D3080
:10DB9000A1F3812F0E94936DF0CFDF91CF911F9160
:10DBA0000895CF93DF93CDB7DEB79E01285F3F4F37
:10DBB0004E815F8160E470E080E194E10E94C19B4E
:10DBC00060E174E18D810E94B86DDF91CF9108957D
:10DBD000CF93C82F8A3031F46DE0809150140E94A9
:10DBE000936D02C08D3029F06C2F809150140E94EB
:10DBF000936D80E090E0CF9108952DE0829FC00169
:10DC00001124FC01EE54FD4F748763870895682F3B
:10DC100080E00C94936D8093501484EA92E090938A
:10DC20006F3D80936E3D089584B7877F84BF0FB6A4
:10DC3000F894A895809160008861809360001092AC
:10DC400060000FBE08959FE088E10FB6F894A89594
:10DC5000809360000FBE909360000895A89508958A
:10DC60000FB6F894A8958091600088618093600059
:10DC7000109260000FBE0895F89498E088E10FB606
:10DC8000F894A895809360000FBE90936000FFCF3A
:10DC900080910D3580910D3590E0089540E06FE161
:10DCA00081E491E00C94B173E9E3F1E0808180813B
:10DCB0008D7F80838DE090E00197F1F723E040E0D5
:10DCC0006FE182E491E00E94BC7383E090E00197F1
:10DCD000F1F708959091390191FD0AC0282F803104
:10DCE00008F02FE040E06FE085E491E00C94BC7315
:10DCF00008958091390181FD0EC040E06FE181E41B
:10DD000091E00E94B173282F2F7E81E090E02130B6
:10DD100021F080E0089580E090E00895809139013D
:10DD200081FF02C081E0089540E06FE181E491E06D
:10DD30000E94B1738F3121F08F7E8150823090F735
:10DD400080E008950E948E6E8823E1F30895CF93BA
:10DD5000DF93C82F0E94A26E0E944E6ED82FC81764
:10DD600071F1C83019F40E94546E25C0C93121F4F4
:10DD7000863189F429E005C0C63169F4893159F446
:10DD800026E040E06FE182E491E00E94BC7383E012
:10DD900090E00197F1F72C2F40E06FE182E491E0F1
:10DDA0000E94BC73D83019F489E691E002C083E088
:10DDB00090E00197F1F70E944E6E8C1303C080E44F
:10DDC00090E002C083E490E0DF91CF9108950E943B
:10DDD000A26E1092A2360E94546E80913901826028
:10DDE00080933901809125378823D9F1809194005F
:10DDF00090919500409136375091373784179507A9
:10DE0000A0F48091023790910337A0910437B0912C
:10DE100005378C57914EAF4FBF4F80930237909389
:10DE20000337A0930437B0930537209194003091C5
:10DE30009500241B350B8091023790910337A091F8
:10DE40000437B0910537820F931FA11DB11D809338
:10DE5000023790930337A0930437B093053710929D
:10DE60002537809127378823D9F1809194009091AC
:10DE7000950040913A3750913B3784179507A0F4AD
:10DE800080910A3790910B37A0910C37B0910D37E4
:10DE90008C57914EAF4FBF4F80930A3790930B37FB
:10DEA000A0930C37B0930D372091940030919500DA
:10DEB000241B350B80910A3790910B37A0910C37BA
:10DEC000B0910D37820F931FA11DB11D80930A37AA
:10DED00090930B37A0930C37B0930D3710922737E0
:10DEE00008958091A236882381F08091D4148823EC
:10DEF00031F081E08093D21481E090E008950E9497
:10DF00008E6E8823B1F30E94E76E80E090E0089562
:10DF1000809194009091950090933B3780933A378D
:10DF200081E0809327379091390191FD08C080915D
:10DF3000390181FD1AC086E10E94A76E16C0809348
:10DF4000A13620919400309195003093373720937B
:10DF5000363780932537809139018D7F8093390141
:10DF60008091A1368111FCCFE2CF81E08093A2366F
:10DF700008958091A23681110AC08091D41488231B
:10DF800021F081E08093D31402C00E94886F81E069
:10DF900090E008951F93CF93DF931F92CDB7DEB724
:10DFA0008FB789838091D41481111FC0F894809118
:10DFB000A236882351F08091390181FD14C00E945E
:10DFC0008E6E882381F080E003C00E94B96F81E0EB
:10DFD000909147019E3088F4882351F01FEF0E94F2
:10DFE000716F107429F489818FBF80E090E009C0BF
:10DFF00089818FBF81E090E004C08823A1F310E005
:10E00000EECF0F90DF91CF911F9108958091D3149F
:10E01000882321F00E94886F1092D3148091D2142B
:10E02000882321F00E94E76E1092D2141092D4142B
:10E0300008950F931F93AB0121E02093D414009116
:10E04000E6361091E7362091E8363091E9360F5FD9
:10E050001F4F2F4F3F4F0093E6361093E736209324
:10E06000E8363093E93622E0260F27FF0CC0809176
:10E070009F369091A03601969093A03680939F365C
:10E080000FEF1FEF07C0BC0181E594E10E942D9ABC
:10E0900000E010E00E940670C8011F910F910895E2
:10E0A0008093D61408950E944E6E823021F0823102
:10E0B00011F081E0089580E0089508958FEF809336
:10E0C0004E0122E044E060EF8CE691E00E94BC73D8
:10E0D00025E041E06EE08CE290E00E94BC7380E8B5
:10E0E00080936F018091460180936D0121E045E0AE
:10E0F00060E284E491E00C94BC73CF93DF93CDEFA6
:10E10000D3E0CE010197F1F70E94A7731092163564
:10E110001092983510921A361092153510921435C7
:10E12000E9E3F1E080818E7F808380818D7F808331
:10E130008DE090E00197F1F780818160808323E09A
:10E1400040E06FE182E491E00E94BC732197F1F717
:10E1500080915D0180915E010E945E7060E070E0E0
:10E160008CEC92E00E94255C0E94886F81E090E038
:10E17000DF91CF9108958091D5140895CF93DF93C7
:10E180001F92CDB7DEB789830E94A26E89818093EA
:10E19000D514282F40E06FE188E491E00F90DF91E3
:10E1A000CF910C94BC730E94BE708091390181FDA7
:10E1B00003C086E00C94A76E0895FA018093620173
:10E1C0009093630160936001709361013097C1F097
:10E1D000808180936B01818180936A018281809329
:10E1E00069018381809368018481809367018581BF
:10E1F00080936601868180936501878180936401A5
:10E2000008958CEC92E00E94465C81E080930D358D
:10E2100080910E3590910F35019690930F35809334
:10E220000E3581E090E008958091153592E8899F40
:10E23000F0011124EA5EFA4C10828F5F833018F4EB
:10E240008093153502C010921535E091153582E89E
:10E25000E89FF0011124EA5EFA4C808181110C9450
:10E26000017110920D3508951F93CF93DF93209184
:10E27000153512E8129F90011124F901EA5EFA4C5B
:10E280004081411103C00E94147192C05091390124
:10E2900051FD8EC05091A236552309F489C047FF25
:10E2A00016C00E9414718091D6369091D736A091F5
:10E2B000D836B091D9360196A11DB11D8093D636BE
:10E2C0009093D736A093D836B093D93671C04330E7
:10E2D000B0F40E9414718091D2369091D336A091FF
:10E2E000D436B091D5360196A11DB11D8093D2369A
:10E2F0009093D336A093D436B093D53659C050E01E
:10E30000EA0122976C177D07B0F40E941471809186
:10E31000CE369091CF36A091D036B091D1360196BD
:10E32000A11DB11D8093CE369093CF36A093D036E9
:10E33000B093D1363DC0B901695E7A4C0E942D9AE6
:10E34000E09115351E9FF0011124EA56FA4C8081A8
:10E35000809306350E9414718091470180930735A0
:10E3600090910C35992311F0891710F480930C3596
:10E370006091073570E084E00E94B16360910635DA
:10E3800070E083E00E94B1638091EA369091EB36B1
:10E39000A091EC36B091ED360196A11DB11D809390
:10E3A000EA369093EB36A093EC36B093ED3602C08C
:10E3B000C0E0D0E0CE01DF91CF911F910895CF93BF
:10E3C000DF93EC01888199810097E9F087309540CF
:10E3D00021F01982188283E026C06238C1F41092BD
:10E3E0000D350E9438630E949D6260E870E00E94D3
:10E3F0003471181619066CF40E949862E09161035A
:10E40000F0916203099587E095E09983888381E024
:10E410000AC080910A3590910B35019690930B3587
:10E4200080930A35F0CFDF91CF91089591E09093DA
:10E43000D4140E946A6E0C9406708091390181FD9B
:10E4400006C040E06FE085E491E00C94B17380E198
:10E4500008950F931F93CF93DF93C82F81E080938C
:10E46000D414D091A2369091390191FF16C0209119
:10E47000940030919500309337372093363780934E
:10E4800025378093A136809139018D7F80933901A2
:10E490008091A1368111FCCFD0E00E94A26E8091C4
:10E4A000A236882309F43FC0809127378823D9F109
:10E4B000809194009091950040913A3750913B376C
:10E4C00084179507A0F480910A3790910B37A0919B
:10E4D0000C37B0910D378C57914EAF4FBF4F809393
:10E4E0000A3790930B37A0930C37B0930D372091D8
:10E4F000940030919500241B350B80910A37909140
:10E500000B37A0910C37B0910D37820F931FA11DCF
:10E51000B11D80930A3790930B37A0930C37B093BB
:10E520000D37109227378091390181FD03C089E1B1
:10E530000E94A76E86E00E94BC63892B51F00E9466
:10E540001D72082F86E00E94BC6381500E946A6E93
:10E5500002C000E010E080919400909195009093AB
:10E5600039378093383781E080932637F89480914B
:10E570003901826080933901809139018D7F8093C8
:10E58000390162E06C0F81E594E10E94EC737894AC
:10E5900080919C3690919D36019690939D36809304
:10E5A0009C360E94A26E45E060EE82E491E00E94FB
:10E5B000B173C82F86E00E94BC63892B19F0802FAD
:10E5C0000E946A6EDD2319F00E94886F02C00E94CB
:10E5D000E76E809126378823D9F18091940090913D
:10E5E0009500409138375091393784179507A0F43A
:10E5F0008091063790910737A0910837B09109377D
:10E600008C57914EAF4FBF4F80930637909307378B
:10E61000A0930837B093093720919400309195006A
:10E62000241B350B8091063790910737A09108374E
:10E63000B0910937820F931FA11DB11D809306373A
:10E6400090930737A0930837B09309371092263775
:10E650008091A236882361F080919400909195007A
:10E6600090933B3780933A3781E08093273707C0F8
:10E6700023E040E06FE182E491E00E94BC730E94DD
:10E680000670C130E9F0C330A9F48091DE36909174
:10E69000DF36A091E036B091E1360196A11DB11DA3
:10E6A0008093DE369093DF36A093E036B093E13668
:10E6B000C2E009C0C53031F0C73029F4C1E003C061
:10E6C000C0E001C0C3E08C2F90E0DF91CF911F919B
:10E6D0000F910895CF93DF93EB010E94197000977B
:10E6E00029F4CE010E942972009751F020919F36A3
:10E6F0003091A0362F5F3F4F3093A03620939F3646
:10E70000DF91CF910895CF93DF938091A23681114D
:10E7100004C00E94B96FD1E001C0D0E00E944E6EEB
:10E72000863111F0813119F4C091470109C040E0F0
:10E730006FE186E491E00E94B173C82FCC0FC80F3F
:10E74000D1110E94716F8C2FDF91CF91089510929B
:10E75000D8141092D714EFE6F0E0808180628083B5
:10E760000895FC0180816823862F90E002C0959572
:10E7700087954A95E2F70895FC01922FF89420813D
:10E78000362F3095522F5323292F01C0220F4A953F
:10E79000EAF72623252B208378940895CF93DF93DF
:10E7A000E0917B01EC01E993A0E8B1E020E82E0FB5
:10E7B0003C91399311962A13FBCFE150F0E0E058D9
:10E7C000FE4F2181FC01E058FF4F2083319681E00C
:10E7D0008083DF91CF91089560938001E1E8F1E0BB
:10E7E0006158DC012D91CD01208331966E13F9CF54
:10E7F00008951F920F920FB60F9211240BB60F922D
:10E800002F933F934F935F936F937F938F939F9338
:10E81000AF93BF93EF93FF938091470180930735A8
:10E820008091143522E8829FC00111248A5E9A4C9F
:10E830000E94CE73809114358F5F833018F48093DB
:10E84000143502C0109214350E940171FF91EF91AE
:10E85000BF91AF919F918F917F916F915F914F91F8
:10E860003F912F910F900BBE0F900FBE0F901F90F6
:10E8700018951F920F920FB60F9211240F900FBE92
:10E880000F901F9018951F920F920FB60F921124A0
:10E890000F900FBE0F901F9018951F920F920FB6FA
:10E8A0000F9211240F900FBE0F901F9018951F927A
:10E8B0000F920FB60F9211241092A1360F900FBE37
:10E8C0000F901F9018951F920F920FB60F92112460
:10E8D0001092A1360F900FBE0F901F9018951F92A7
:10E8E0000F920FB60F9211248F9381E080930D3514
:10E8F0008F910F900FBE0F901F9018951F920F923F
:10E900000FB60F9211241092A1360F900FBE0F90E8
:10E910001F9018951F920F920FB60F9211248F938C
:10E920009F938091D7149091D81401969093D81406
:10E930008093D7149F918F910F900FBE0F901F90CF
:10E940001895CF92DF92EF92FF920F931F93CF9380
:10E95000DF937C018B016A0189ED94E10E94E65C02
:10E96000EC01892B51F0EC81FD81309711F0C80149
:10E970000995CE010E94925DF3CFA601B801C701AF
:10E98000DF91CF911F910F91FF90EF90DF90CF908B
:10E990000C946B5A0F931F93CF93DF9300D0CDB796
:10E9A000DEB78091AA369091AB36A091AC36B0918B
:10E9B000AD360196A11DB11D8093AA369093AB365A
:10E9C000A093AC36B093AD360E9431778C0189EDBF
:10E9D00094E10E94E65C009779F0DC011296ED91DB
:10E9E000FC911397309729F089839A8309959A812E
:10E9F00089810E94925DEFCF0115110549F0C80190
:10EA00000F900F90DF91CF911F910F910C94625A4C
:10EA10000F900F90DF91CF911F910F9108950E9459
:10EA20001C7C0E9438630E945B758DE493E0909398
:10EA3000A5368093A4360E942F772FEF31E040E077
:10EA40005EE160E074E082E090E00C94FC76BC0152
:10EA500089ED94E10C944A5DBC0189ED94E10C943C
:10EA60002B5DCF93DF93EC014091A6365091A736F2
:10EA70006091A8367091A9364F5F5F4F6F4F7F4FFF
:10EA80004093A6365093A7366093A8367093A93664
:10EA90000E944477009761F00E94B662E0915103B2
:10EAA000F0915203BE0181EA94E7099581E090E07C
:10EAB000DF91CF9108958FED94E10C94E25C0F9378
:10EAC000CF93DF93EC017B836A8318865F834E8349
:10EAD000BC018FED94E10E944A5DE091DB14F0915E
:10EAE000DC14309749F04C815D8101E020E030E09A
:10EAF00068858A819B810995DF91CF910F91089557
:10EB0000BC018FED94E10C942B5D0F93FC011086FA
:10EB1000E091DB14F091DC14309761F0DC0100E04F
:10EB200020E030E040E050E060E012968D919C9152
:10EB3000139709950F9108950F93DC0114962D9169
:10EB40003C91159781E018968C93189715967C93B5
:10EB50006E931497E091DB14F091DC14309741F040
:10EB6000AB0100E061E012968D919C91139709959D
:10EB70000F9108950F93E091DB14F091DC1430971E
:10EB800079F0DC0114964D915C91159701E09A01A2
:10EB900018966C91189712968D919C9113970995E0
:10EBA0000F910895E091DD14F091DE14309709F093
:10EBB000099408959093DE148093DD140895909342
:10EBC000DC148093DB1408958FED94E10C94E65CE3
:10EBD000EF92FF920F931F93CF93DF938C01EB0182
:10EBE0007A018FED94E10E94E65C0097D9F0DC0198
:10EBF00012962D913C9113972C173D0781F4169690
:10EC0000ED91FC911797309769F09701AE01B8012B
:10EC1000DF91CF911F910F91FF90EF9009940E9487
:10EC2000925DE3CFDF91CF911F910F91FF90EF9015
:10EC300008950895CF93DF93C1EED4E169A97AA92D
:10EC400020E030E049E356E78CEF94E10E946A5FF0
:10EC50000E941A7C69A97AA90E94E69320E030E01C
:10EC60004DE456E7BC018CEE94E1DF91CF910C941A
:10EC70006A5F8091121590911315209110153091B3
:10EC80001115880F991F2817390708F4C9019093A7
:10EC90001315809312150C941A76CF93DF930E946C
:10ECA00038630E949D62EC01198218820E94E4750B
:10ECB00028813981009719F1FC0140854423F9F03E
:10ECC000FC0142815381F901EE0FFF1FEE0FFF1F80
:10ECD000EC0FFD1F53834283FC01448155812F5F5C
:10ECE0003F4FF901EE0FFF1FEE0FFF1FEC0FFD1F4F
:10ECF00051834083398328830E94925DD9CFC90113
:10ED0000880F991F880F991F02960E949862888128
:10ED10009981892B31F081EE94E1DF91CF910C94B0
:10ED2000385ADF91CF910895AF92BF92CF92DF9280
:10ED3000EF92FF920F931F93CF93DF9300D0CDB745
:10ED4000DEB76B010E949D62FC01E080F180FA82D7
:10ED5000E982FCE0EF16F10418F400E010E00DC0C9
:10ED6000FF92EF928DE09AE09F938F930E94E89A32
:10ED70000F900F900F900F9022C00E151F05F9F005
:10ED80000E949D629801220F331F220F331F820FB2
:10ED9000931FFC01A280B3800E949D620F5F1F4FF2
:10EDA0009801220F331F220F331F820F931FFC0184
:10EDB00040815181B501C6010E94E875DECF0F90F8
:10EDC0000F90DF91CF911F910F91FF90EF90DF9007
:10EDD000CF90BF90AF9008950F93013059F4809178
:10EDE0000C1590910D1590931315809312150F919A
:10EDF0000C941A760F910895EF92FF920F931F9340
:10EE0000CF93DF937B018A01E9014AE353E0BC0120
:10EE100081EE94E10E941B5AE1EEF4E1F4A6E3A630
:10EE200016A705A7D0ABC7A78CEE96E7DF91CF91C9
:10EE30001F910F91FF90EF900C94DF758CEF94E190
:10EE40000E94EE5F8CEE94E10E94EE5F81EE94E111
:10EE50000C94365A809112159091131508950C94C4
:10EE6000775ACF93DF93E0913E03F0913F030995EA
:10EE7000EC01892B29F06A817B8181E00E94B163DA
:10EE8000CE01DF91CF9108950F931F93CF93DF931E
:10EE9000EC01E0914003F091410309958C016A81F6
:10EEA0007B8181E00E94B16381E090E0012B11F44D
:10EEB00080E090E0DF91CF911F910F910895E09154
:10EEC0004203F0914303099420E030E00296FC01F4
:10EED00032974081442331F0FC0131974081240F67
:10EEE000311DF4CFC9010895FC01208130E0322F9B
:10EEF00022278181282B02C0220F331F6A95E2F757
:10EF0000232F3327FA01EC5BFC4F808190E08223B2
:10EF1000932328E030E0241B350B02C0969587959B
:10EF20002A95E2F708956F927F928F929F92AF9207
:10EF3000BF92CF92DF92EF92FF920F931F93CF93E6
:10EF4000DF937C018B015A01E9012830310544F43B
:10EF5000A901B501C8010E947477F701808346C0FA
:10EF6000690183E0D594C7948A95E1F7452B21F098
:10EF70004701612C712C06C0FB01D701CB018C0D20
:10EF80009D1D1FC048E050E0B501C801860D971DCA
:10EF90000E947477F40181934F01FFEF6F1A7F0A8B
:10EFA0006C147D0479F7AE01477055274115510562
:10EFB000E9F0E701C60DD71DB501C801860D971D03
:10EFC00012C0E817F90719F021912D93FACFAE017D
:10EFD000477055274115510549F0E701CC0DDD1D5E
:10EFE00060E070E0CF010E9474778883DF91CF9159
:10EFF0001F910F91FF90EF90DF90CF90BF90AF9057
:10F000009F908F907F906F9008958F929F92AF9274
:10F01000BF92CF92DF92EF92FF920F931F93CF9305
:10F02000DF9300D0CDB7DEB70E949D628C0182E0F5
:10F0300090E00E947B62892B19F480E090E05FC031
:10F04000F801218130E0322F22278081A901480F69
:10F05000511DCA010E94885A7C01892B71F30E94BC
:10F060009D624C01F7019681292F269526952695BC
:10F0700030E0977041E050E011F440E050E0C90109
:10F08000840F951F0E947B62892BB9F2F7010481DE
:10F090001581A12CB12CF8018081882379F1F80128
:10F0A000C180D12CA50147705527B50193E0759516
:10F0B00067959A95E1F7680D791D883168F096019A
:10F0C000CE0101960E949377BE016F5F7F4FF801DA
:10F0D00080810E94C5630DC01A8219829601CE01FB
:10F0E00001960E94937769817A81F80180810E945C
:10F0F000B163AC0CBD1C0E5F1F4FCDCFC7010F908D
:10F100000F90DF91CF911F910F91FF90EF90DF90C3
:10F11000CF90BF90AF909F908F900895DC0150E00A
:10F12000E0E1F0E0CF01861B970B821B930B02C03E
:10F13000440F551F8A95E2F78C91852B8C9311967D
:10F140008C911197482B11964C9308956F927F9252
:10F150008F929F92AF92BF92CF92DF92EF92FF92E7
:10F160000F931F93CF93DF93283031051CF4FA01DE
:10F1700040815AC05901E3E0B594A794EA95E1F7BC
:10F180006115710541F03901EA018B017C014A01E9
:10F19000C12CD12C05C0EA01FC014A0D5B1D2AC01F
:10F1A000F40141914F0128E030E0B801C7018C0D16
:10F1B0009D1D0E948E78FFEFCF1ADF0ACA14DB0470
:10F1C00079F793012770332721153105E9F1CC0D2B
:10F1D000DD1D488150E0021B130B085F1F4F02C06A
:10F1E000559547950A95E2F760E070E0C7018C0DF0
:10F1F0009D1D1AC0C417D50719F069916193FACF04
:10F200002770332721153105F9F0488150E068E077
:10F2100070E0621B730B02C0559547956A95E2F743
:10F2200060E070E08A0D9B1DDF91CF911F910F91DF
:10F23000FF90EF90DF90CF90BF90AF909F908F9016
:10F240007F906F900C948E78DF91CF911F910F91EA
:10F25000FF90EF90DF90CF90BF90AF909F908F90F6
:10F260007F906F9008956F927F928F929F92AF924E
:10F27000BF92CF92DF92EF92FF920F931F93CF93A3
:10F28000DF9300D0CDB7DEB77C01FC018681082F6B
:10F29000069506950695202F30E0877001E010E076
:10F2A00011F400E010E0020F131FC80102960E9443
:10F2B0000163009709F448C00E94A462F70122810B
:10F2C000FC012083F7012381FC0121830E94A462B9
:10F2D00002965C01A80160E070E00E94369AF70196
:10F2E000048115810F5F1F4F812C912CF8013197FC
:10F2F0008081882339F1F801C080D12C3401F7E0F6
:10F300006F227724740193E0F594E7949A95E1F7DE
:10F31000EA0CFB1C883128F00E94CF639601AC01F7
:10F3200008C00E94BC639A8389839601AE014F5F37
:10F330005F4FB301C7010E94A6788C0C9D1C0E5F25
:10F340001F4FD4CF81E090E00F900F90DF91CF91CD
:10F350001F910F91FF90EF90DF90CF90BF90AF90F3
:10F360009F908F907F906F900895E0915F03F09150
:10F3700060030994E0913803F09139030994E09116
:10F380006303F09164030994E0916503F0916603CF
:10F39000099480E090E008950895E0913003F091A1
:10F3A0003103099480E090E008950F931F93CF9369
:10F3B000DF93CDB7DEB7E0970FB6F894DEBF0FBE90
:10F3C000CDBF0E94EA628C010E949D62AE014F5F38
:10F3D0005F4F602F0E94A081882309F442C088A952
:10F3E0009801281B3109C9010E947B62892BC9F150
:10F3F0008E8181110CC0BE016A5E7F4F88E10E9440
:10F40000C563E0915303F091540309952AC02A85FE
:10F410003B852D3C9BEA390719F02F3F3F4F09F5FB
:10F42000823019F088E090E002C082E090E001971D
:10F4300010F3E1E0F0E0EC0FFD1FE80FF91F23856A
:10F440002F3FA9F3BE01645F7F4F89E10E94C5632E
:10F4500089E10E94CF6367EB74E30E94D459892B42
:10F4600051F6E0960FB6F894DEBF0FBECDBFDF9128
:10F47000CF911F910F910895AF92BF92CF92DF92DB
:10F48000EF92FF920F931F93CF93DF93CDB7DEB729
:10F49000E0970FB6F894DEBF0FBECDBF8C016B01B5
:10F4A000CE0101967C0180E3F70111928A95E9F77C
:10F4B00081E089838CE00E94BC638C831D821F8263
:10F4C0008091161591E0980F90931615898783E027
:10F4D000B82EB8868DEC9BEA9B878A8789E10E94CB
:10F4E000CF636CE073E00E94D459892B31F082E045
:10F4F0008E838FEF8C878D8709C089E10E94CF634F
:10F50000BC01CE010C960E94CB59BE828DEC9BEAC9
:10F510009D8B8C8B67EB74E3CE0146960E94CB5992
:10F520000E949D629FA78EA70E94EA6288ABC701D6
:10F530000E94A080B82E90E00E940163892B31F1D7
:10F540000E94A4624B2DBC01C7010E94BE80E090C6
:10F550002603F09027030E94F4625C010E94A462DB
:10F56000B501F70109950115110581F0009739F0F2
:10F57000019761F441E050E064E070E004C041E0D4
:10F5800050E060E070E0C601F8010995E0960FB622
:10F59000F894DEBF0FBECDBFDF91CF911F910F91C9
:10F5A000FF90EF90DF90CF90BF90AF9008950E94B2
:10F5B0001A7C80931615E0913003F0913103099481
:10F5C000892B29F0E0913003F091310304C0E091E0
:10F5D0003203F09133030994CF93DF93EC018991C7
:10F5E0009991009729F060E070E00E94255CF7CFC8
:10F5F000DF91CF910895CF93DF93EC018991999199
:10F60000009719F00E94755BF9CFDF91CF910895B3
:10F61000CF93DF93EC017B836A830E94B96C99835B
:10F620008883DF91CF910895FC012081318182810F
:10F630009381820F931F918380830895CF93DF93EB
:10F64000EC010E94B96C99838883DF91CF91089572
:10F65000CF93DF93EC010E94B96C28813981821B22
:10F66000930B9C012F5F3F4F81E090E04A815B81CB
:10F670004217530710F080E090E0DF91CF9108959A
:10F68000CF93DF93FC01C281D38180819181C80F28
:10F69000D91F0E94B96C9E01281B390BC901DF914B
:10F6A000CF910895CF93DF93ECE2F7E3CEEED6E36C
:10F6B000A0E2B7E31192119219921992199219923C
:10F6C0001D9287E3E434F807A9F7DF91CF910895FD
:10F6D000CF93DF93FC01E05EF84C40819C01220F48
:10F6E000331F220F331F4423F9F0409194005091AF
:10F6F0009500E901C251D94C880F991FFC01E45DC6
:10F70000F84C80819181BA01681B790B88819981BD
:10F71000AA81BB81860F971FA11DB11D8883998384
:10F72000AA83BB8351834083F901E251F94C608184
:10F73000718182819381DF91CF91089560E070E0C3
:10F74000CB010895880F991F880F991FFC01E25182
:10F75000F94C40835183628373830895CF93DF9381
:10F76000C0E2D7E3EEEEF6E3ACE2B7E3899188239B
:10F77000D1F080919400909195002D913C9111973A
:10F78000AC01421B530B9A0140815181628173810C
:10F79000420F531F611D711D408351836283738328
:10F7A00011969C938E933496129657E3EE31F5079B
:10F7B000E9F6DF91CF9108950C9432800F931F9357
:10F7C000FC018091171590911815338322831583BE
:10F7D000048371836083F0931815E0931715892BC8
:10F7E00019F4CB010E944C8080E090E01F910F91B2
:10F7F000089580911715909118150097C1F01092F7
:10F80000181510921715DC0114966D917C911597BF
:10F810001296ED91FC9113970995E0911715F091CF
:10F820001815309721F0808191810C944C800895B7
:10F830000C94A4960C94A0968EED92E00E945C5CD1
:10F8400086ED92E00C945C5CCF93DF930E94AA62F9
:10F85000892BA9F086ED92E00E947A5CEC01892B5D
:10F8600021F10E94EA62998388830E94E5629B836A
:10F870008A83CE0104960E9426628CAB14C08EED62
:10F8800092E00E947A5CEC01009779F002960E9467
:10F89000386299838883BE016E547F4FCE018E57A4
:10F8A0009F4F0E948F63CE0102C080E090E0DF9105
:10F8B000CF910895BC016E547F4F8E579F4F0C948B
:10F8C0008F63CF93DF93EC01BC018EED92E00E9439
:10F8D000C55CBE01892B19F08EED92E009C086ED62
:10F8E00092E00E94C55C892B39F0BE0186ED92E062
:10F8F000DF91CF910C949F5CDF91CF9108950F938E
:10F900001F93CF93DF93EC01BC018EED92E00E9438
:10F91000C55C892B91F0FE0161917191CF010E942C
:10F920004B63BE016E547F4FCE018E579F4FDF91C8
:10F93000CF911F910F910C94A063BE0186ED92E0D0
:10F940000E94C55C892BD1F00E943863688179815F
:10F950008A819B810E944B638CA990E00E94016385
:10F960000CA910E00E94A462BE016C5F7F4FA80149
:10F97000DF91CF911F910F910C942D9ADF91CF9130
:10F980001F910F910895CF93DF93EC01BC018EED91
:10F9900092E00E94C55C892B19F0CE0102960CC042
:10F9A000BE0186ED92E00E94C55C892B19F08A8128
:10F9B0009B8102C080E090E0DF91CF910895FC012F
:10F9C000808191810895860F911D860F911D8E571C
:10F9D0009F4F0895860F911D860F911DFC01EE57D4
:10F9E000FF4F808191810895089586E79BE10E94F1
:10F9F000A35E892B21F086E79BE10C94905E08952D
:10FA0000E091621BF091631B309709F0099480E04C
:10FA10000895EF92FF920F931F93CF93DF938C0182
:10FA2000EA01FC0180819181009741F08C30934084
:10FA300071F1F8011182108283E0F6C080E024E0C9
:10FA4000829FF0011124EC59F44E118210828F5FD5
:10FA50008430A9F78093611B80919C1290919D1234
:10FA60009093751B8093741B0E946E5B8093443748
:10FA700060E470E086E79BE10E947C5E0E940D835B
:10FA80008CE093E0F8019183808381E0CDC0623007
:10FA9000D9F48091453790914637892B89F380912D
:10FAA0005637863029F480916E3781FD0E94F57CAF
:10FAB00081E00E9462848091453790914637892B7E
:10FAC000F9F20E94227FDCCF633060F5611114C02F
:10FAD0002097B1F2D093533CC093523C83E00E94F4
:10FAE00062848091453790914637892B11F00E94AE
:10FAF000007D0E94F57CC4CF613011F6209709F497
:10FB0000BFCFD0934F3CC0934E3C85E00E946284AF
:10FB10008091453790914637892B09F4B1CF0E94E7
:10FB2000007DAECF673809F040C01092601B84E6BC
:10FB3000E82E8BE1F82E8091601B8430C0F4F70131
:10FB4000828193818C179D0749F4808191810E9465
:10FB50002D84F7011182108213821282F4E0EF0EDD
:10FB6000F11C8091601B8F5F8093601BE4CFEDE6FA
:10FB7000FCE3838194818C179D0719F4148213820E
:10FB80001082B0962CE3ED3EF20799F7EAEEFCE323
:10FB9000818592858C179D0711F4158214823D96FC
:10FBA0008DE3EC36F807A1F76BCF683809F068CF22
:10FBB000C657DB4109F064CF86E79BE10E94A35E54
:10FBC000892B09F45DCF1092601BE091601BE4303B
:10FBD00008F056CF20E2E29FF0011124EC5AF34CDA
:10FBE000818D8823D9F086E79BE10E94905E809109
:10FBF000601BE0E28E9FC00111248C5A934C9093BD
:10FC0000533C8093523C82E00E946284809145374D
:10FC100090914637892B11F00E94007D8091601BE6
:10FC20008F5F8093601BD1CFDF91CF911F910F9198
:10FC3000FF90EF9008959093631B8093621B08954B
:10FC40009C0140919C1250919D1290E0E4E6FBE1F2
:10FC50009430A1F0608171816217730761F4628151
:10FC600073816417750739F490935F1B11821082BA
:10FC7000C9010C942D8434969F5FEACF90935F1B4B
:10FC800008959C0190E0E4E6FBE19430B1F081E05E
:10FC9000890F40815181452B69F490935E1B31831C
:10FCA000208380919C1290919D1293838283C9013D
:10FCB0000C9448843496982FE8CF90935E1B089557
:10FCC00020919C1230919D12FC01358F248F778FEB
:10FCD000668F089520919C1230919D12FC0132870D
:10FCE0002187748763870895CF93DF93EA010E9489
:10FCF000BC83009749F020919C1230919D12FC0129
:10FD000032872187D487C387DF91CF9108950F93DE
:10FD10001F93CF93DF9300D000D0CDB7DEB78C0117
:10FD2000AB019FEF99839A839B839C83B801CE019B
:10FD300001960E94747E009719F0FC0115830483DC
:10FD40000F900F900F900F90DF91CF911F910F9117
:10FD5000089540E050E062E086EE92E00E94165C7A
:10FD600010924637109245370895AC0161E086EE57
:10FD700092E00C94F75BAC0160E086EE92E00C94AC
:10FD8000F75B0F931F93CF93DF938A010E94398310
:10FD9000EC01892B59F080919C1290919D129D8FBE
:10FDA0008C8F1F8F0E8FCE010E94BB7ECE01DF9104
:10FDB000CF911F910F910895CF93DF93A091523C63
:10FDC000B091533C109719F0ED016C9605C0C091AD
:10FDD0004E3CD0914F3C299680914D3C86FF23C0EC
:10FDE00010925D1B80E0E4E6FBE18430C1F04081CD
:10FDF000518114962D913C9115974217530761F448
:10FE0000228133812115310539F080935D1B3983BF
:10FE100028831B821A8205C034968F5FE6CF8093B9
:10FE20005D1B0E94F57C88819981009741F04A8191
:10FE30005B8160914437DF91CF910C94165CDF9128
:10FE4000CF9108950F931F93CF93DF9380915637EF
:10FE5000863009F071C08091453790914637811501
:10FE6000954009F069C004E912E010934637009309
:10FE70004537D2E0D0934F37C4E9C0935037109242
:10FE80007237109271370E940783809590959093F6
:10FE900072378093713710925837109257370E94FB
:10FEA000F6828095909590935837809357370E94AB
:10FEB000007D1093463700934537D0934F37C0935A
:10FEC0005037A091503CB091513CFD01E459FD4F99
:10FED0008CE692E001900D920197E1F76CE672E0FA
:10FEE00085E697E30E94B682809149378093653713
:10FEF00080914A378093663780914B37809367377C
:10FF000080914C3780936837109272371092713716
:10FF10000E940783809590959093723780937137F4
:10FF200010925837109257370E94F682809590951C
:10FF30009093583780935737DF91CF911F910F914E
:10FF40000C94007DFC01680F791F80E048E1E61702
:10FF5000F70781F0219198E0322F3827532F517005
:10FF600030FD84278695513009F48068269591509C
:10FF700099F7EDCF08951F920F920FB60F921124AB
:10FF80000BB60F922F933F934F935F936F937F9393
:10FF90008F939F93AF93BF93EF93FF9380919400C0
:10FFA00090919500909331378093303781E0809322
:10FFB000223780917100807D809371000E94F97BCF
:10FFC000809122378823D9F18091940090919500F7
:10FFD000409130375091313784179507A0F48091C4
:10FFE000F6369091F736A091F836B091F9368C57E5
:10FFF000914EAF4FBF4F8093F6369093F736A09354
:020000021000EC
:10000000F836B093F9362091940030919500241B76
:10001000350B8091F6369091F736A091F836B09175
:10002000F936820F931FA11DB11D8093F636909370
:10003000F736A093F836B093F93610922237FF9135
:10004000EF91BF91AF919F918F917F916F915F9150
:100050004F913F912F910F900BBE0F900FBE0F90BD
:100060001F9018959FB7F894E1E7F0E08081807DBC
:10007000808388B38F6288BB10929000E1E9F0E042
:10008000108210929200109295001092940080813C
:10009000856080839FBF08959C019FB7F89430933B
:1000A00099002093980088B38F6288BBE1E7F0E065
:1000B0008081826080839FBF0895CF93DF93FC018E
:1000C000DB0185E0EB0119928A95E9F78581837060
:1000D00011F082E08C938781837021F082E0129688
:1000E0008C9312978581837081F08781837069F08A
:1000F00023893489818592852817390731F481E075
:10010000848312961C92129701C014828581837099
:10011000823029F0833011F488E001C080E011962C
:100120008C93119787818370823029F0833011F48A
:1001300088E001C080E013968C93DF91CF91089501
:10014000CF93DF9300D000D01F92CDB7DEB7BE01B2
:100150006F5F7F4F0E945D8099818A81890F8D5FDB
:100160009B81890F9C81890F9D81890F0F900F9032
:100170000F900F900F90DF91CF9108954F925F9263
:100180006F927F928F929F92AF92BF92CF92DF92A7
:10019000EF92FF920F931F93CF93DF9300D000D085
:1001A00000D0CDB7DEB78C017B01BE016F5F7F4F02
:1001B0004E830E945D80B9815A80652D70E0AB81CD
:1001C0004C80242D30E08B2F90E00396860F971FF4
:1001D0008A0F911D820F931F5D81850F911D4E81A6
:1001E00050E0481759070CF493C0F801818180FB57
:1001F000882480F8912C83E0880C991C8A95E1F77B
:10020000828180FBAA24A0F8B12C94E0AA0CBB1C2C
:100210009A95E1F78A2880818770882A838180FBFC
:10022000CC24C0F8D12C45E0CC0CDD1C4A95E1F77C
:10023000C828848180FB662460F8712C56E0660C27
:10024000771C5A95E1F76C28F7016082F8018581E7
:100250008370F4E08F9FA0011124F80196819370C0
:10026000F0E19F9FC0011124842BF8014781F0E445
:100270004F9FA0011124842BF7018183F801808511
:10028000F7018283B23051F4F8018185F70183834D
:10029000F8018285F701848385E001C083E0580E70
:1002A000852D952D961B6115710561F061507109C1
:1002B000A801460F571FFA014385F701E90FF11D09
:1002C0004083EECFA23089F4F701E50DF11DD8018E
:1002D00053969C915397908391E0950DF701E90F08
:1002E000F11D8E5F54969C919083B42DB80F8B2F87
:1002F0009B2F921B2115310561F021503109F80126
:10030000E20FF31F8589F701E90FF11D8083EFCF1D
:1003100080E026960FB6F894DEBF0FBECDBFDF910A
:10032000CF911F910F91FF90EF90DF90CF90BF90F2
:10033000AF909F908F907F906F905F904F900895B7
:10034000BF92CF92DF92EF92FF920F931F93CF93C2
:10035000DF93633008F4AEC0EA01D62E7C01FC01C5
:10036000908196FBBB24B0F88181282F2695269595
:100370002370C82EC294C694C69453E0C522392F68
:100380003770388393FB332730F9398394FB332755
:1003900030F93A8395FB992790F99B83BC822D8392
:1003A000829583708E83CF8282818887222379F120
:1003B0003381848190E0982F8827830F911D9A873D
:1003C000898787010B5F1F4F223071F46CE073E067
:1003D000CE010B960E94CB59F70186818B878581D0
:1003E0008C870E5F1F4F1EC02330E1F4F7013D964E
:1003F000DE011B969E012D5E3F4F9E2F8F2F429157
:100400004D93A217B307D9F7092F182F0BC08701F7
:100410000D5F1F4F6CE073E0CE010B960E94CB592D
:100420001A861986CC20A1F1B1100DC0F8012081E7
:10043000818190E0982F8827820F911D9C8B8B8B58
:100440000E5F1F4F04C089859A859C8B8B8BF2E0D1
:10045000CF120EC06CE073E0CE0145960E94CB59DE
:10046000F80181818D8B80818E8B0E5F1F4F18C0AC
:10047000F3E0CF1215C0085F1F4FD801FE0175963B
:10048000CE014D962E912193E817F907D9F708C0B0
:100490006CE073E0CE0145960E94CB591C8A1B8A02
:1004A000C8018E199F092D2D281B2FA71EA70DA748
:1004B000D81608F480E0DF91CF911F910F91FF9043
:1004C000EF90DF90CF90BF900895FB01415051090C
:1004D000460F571FE417F50778F4208130E0322FDC
:1004E00022276181260F311D820F931F82179307E8
:1004F00008F401963296EECFE417F50751F4208107
:1005000030E0322F2227820F931F8217930708F4BF
:1005100001960895CF93DF93C0915037D0E0649750
:1005200020914F3730E0322F2227C20FD31F48E0EF
:1005300050E069E577E39E01280F311DC9010E9453
:100540006582AE0161E677E30E946582009721F043
:1005500098278927982702C08FEF9FEFDF91CF91CF
:10056000089590938F1B80938E1B0895FC01238127
:10057000260F20934C37A72FBB2792819A0F909379
:100580004B37318130934A37408140934937E92FC7
:10059000F0E0EA17FB0748F481E0830F80934A37C5
:1005A000811103C04F5F4093493730E0772726170A
:1005B000370788F49F5F90934B3791110CC080915F
:1005C0004A378F5F80934A37811105C08091493740
:1005D0008F5F809349370895AB01BC0180E090E0C4
:1005E0000E946582982789279827089544E150E062
:1005F0006DE477E380E090E00E946582009721F04F
:1006000098278927982708958FEF9FEF089586E010
:100610000C948A8281E10C948A8280E0E82FF0E0D9
:10062000EE0FFF1FEC52F34C118210828F5F84306B
:10063000A9F780E090E2899FF0011124EC5AF34C75
:10064000118E8F5F8430B1F780E094E09093891B26
:100650008093881B80E09DE0989FF0011124E65173
:10066000F34C158214828F5F8A30B1F78093871B19
:100670000895CF93DF93EC012091881B3091891B63
:100680002F5F3F4F21158DE7380710F020E030E154
:10069000522F432FE4E5FCE390E0943059F0818D34
:1006A000882329F0A481B581A417B50749F39F5F7A
:1006B000B096F3CF3093891B2093881B1092871B31
:1006C00090E0E0E0F0E09430E9F080E2989FD00123
:1006D0001124AC5AB34C59968C915997811104C08E
:1006E0009093871BFD0110C0873041F4309739F09B
:1006F0005A962C915A97828D821708F0DF019F5FDE
:10070000FD01E1CF9093871B309791F182E0818FBB
:1007100080918A1B848780918B1B858780918C1B9D
:10072000868780918D1B878788ED94E0938B828BE1
:10073000958B848B81E090E0918B808B138E828FE0
:1007400083E0808F168A80E1878B2091881B30910F
:10075000891B3227232732273583248377836683B7
:1007600088819981AA81BB8180839183A283B3838D
:10077000CF01DF91CF9108950F931F93CF93DF9314
:10078000DC012091881B3091891B2F5F3F4F211581
:100790008DE7380710F020E030E1522F432FEAEECA
:1007A000FCE390E09A3041F0C481D5819F5F3D9693
:1007B000C417D507B9F7E9CF3093891B2093881B5D
:1007C00090E08DE09A30D1F0492F50E021E0290FE0
:1007D000849FF001859FF00D1124E651F34CEF0149
:1007E000249604811581012B39F49093871B30974F
:1007F00041F480E090E02CC0922FE4CF9093871BCF
:10080000F8CF2091881B3091891B3227232732276C
:100810003983288377836683109729F410821182A5
:100820001282138209C08D919D910D90BC91A02DD3
:1008300080839183A283B3838DE0849FD001859FC1
:10084000B00D1124A651B34C80E418968C93CF01BF
:10085000DF91CF911F910F9108959C0190E094300A
:10086000A1F0E92FF0E081E0890FEE0FFF1FEC52BD
:10087000F34C408151814217530729F49093871B11
:10088000118210820895982FEACF9093871B0895C4
:100890009C0190E0943099F0E92FF0E081E0890F1D
:1008A000EE0FFF1FEC52F34C40815181452B29F490
:1008B0009093871B318320830895982FEBCF9093DB
:1008C000871B0895AF92BF92CF92DF92EF92FF9273
:1008D0000F931F93CF93DF93C091523CD091533C21
:1008E000843009F4DBC125E737E33093513C209392
:1008F000503C3093483720934737833059F4898DE3
:100900008F70833009F06AC088899989892B09F032
:10091000D5C67EC0823009F07FC080918D1B8F5F6D
:1009200080938D1B811113C080918C1B8F5F8093EE
:100930008C1B81110CC080918B1B8F5F80938B1B54
:10094000811105C080918A1B8F5F80938A1B109252
:100950004637109245371092E93C1092E83C898D59
:10096000982F9D7F953041F48A8D8F5F8A8F8431D7
:1009700009F0A4C6198EA2C6882309F49FC6288947
:100980003989232B09F440C09A8D2FEF290F2A8F24
:10099000911194C69B8D983031F02FEF280F2230A3
:1009A00048F4953039F4198E80E880934D3C0E94CC
:1009B000DC7E3DC5953038F423E0092E01C0220FBE
:1009C0000A94EAF701C020E32A8F9F5F9B8F8F7004
:1009D0008330A1F048F4813009F445C3823009F036
:1009E0006DC610926E3742C3863009F4BCC488309D
:1009F00009F4B9C4843009F061C6B5C484E08093B9
:100A00004D3C0E94DC7E45C58F70833009F056C690
:100A100088E080934D3C00C5853019F5E0914E3C4F
:100A2000F0914F3C84819581892B09F447C610923F
:100A3000533C1092523C89E697E39093513C80934B
:100A4000503C90934837809347371092E93C10927E
:100A5000E83C109246371092453788E080934D3C31
:100A60001BC180914D37853409F028C600914F375E
:100A700010E0102F002780915037080F111D809132
:100A80004537909146378017910708F417C61093A1
:100A9000463700934537809153378F7309F00EC660
:100AA000F0905437F1100AC68091E43C9091E53CF7
:100AB000C0916903D0916A038C179D0759F4409146
:100AC000E63C5091E73C20916B0330916C03421758
:100AD0005307A1F020915D3730915E372817390711
:100AE00009F0ECC520915F37309160378091E63C8A
:100AF0009091E73C2817390709F0E0C50E94F6827B
:100B0000019609F0DBC580915637863009F429C17A
:100B10008131E9F1813009F0D1C5809161378830A8
:100B200009F0CCC51092613780916337909164379A
:100B3000873F6FEF960710F0099601C008969093D3
:100B40006437809363378091593790915A37A091D9
:100B50005B37B0915C3780935D3790935E37A0939D
:100B60005F37B09360378091E43C9091E53CA09171
:100B7000E63CB091E73C8093593790935A37A09365
:100B80005B37B0935C3780E48093553774C50C5164
:100B90001109109346370093453789E697E3909300
:100BA000513C8093503C8091673790916837892BF6
:100BB00029F00E940A83019609F080C520916337CD
:100BC000309164372115310509F478C58AEE9CE32C
:100BD00090934F3C80934E3CA0906137B090623729
:100BE00040916D0350916E0360916F03709170039B
:100BF000A0915937B0915A3700915B3710915C370B
:100C0000E0906B03F0906C03E0914E3CF0914F3C10
:100C10008DE3EC36F80708F051C584819581009783
:100C200021F12817390709F586819781009719F076
:100C3000A816B906D1F4808191818C179D0729F4FB
:100C4000C280D380CE14DF04B1F08417950729F455
:100C5000C280D380C616D70671F0A817B90729F449
:100C6000828193810817190731F03D96F0934F3C2C
:100C7000E0934E3CC9CF1092533C1092523C82E01C
:100C800080934D3C89E697E39093483780934737AC
:100C90001092E93C1092E83C0E94DC7E8091E83C96
:100CA0009091E93C009709F409C59C01245E3F4FEF
:100CB000309346372093453730934F372093503742
:100CC000E0914E3CF0914F3C20852093553721E137
:100CD0002093563708969827892798279093663748
:100CE00080936537109268371092673784819581B9
:100CF00090936237809361378681978190936437B0
:100D0000809363378091E43C9091E53CA091E63C70
:100D1000B091E73C8093593790935A37A0935B3753
:100D2000B0935C3780819181A281B38180935D37DC
:100D300090935E37A0935F37B093603785E797E372
:100D40009093513C8093503C0E940A8380959095EB
:100D5000009711F48FEF9FEF909368378093673778
:100D60008AC40E940783019609F0A8C440916337A2
:100D7000509164374115510509F4A0C48091613741
:100D800090916237009709F499C460915937709136
:100D90005A37E0915B37F0915C37C4E5DCE3298D8D
:100DA0002223A9F0AC81BD814A175B0781F4AE8193
:100DB000BF818A179B0759F4A881B9816A177B07FD
:100DC00031F4AA81BB81EA17FB0709F467C1A09639
:100DD0002CE3C43DD20719F780916E378F738230B0
:100DE000D9F45093851B4093841B80E0843091F0AC
:100DF000E82FF0E0EE0FFF1FEC52F34C2081318121
:100E00008F5F4217530791F71092871B80E0C0E075
:100E1000D0E07CC08093871B80916E3782FD4EC4EA
:100E200084E180936E3788E290E090934637809318
:100E3000453780E580936D373091683780916C3706
:100E4000809368372091673780916B37809367373D
:100E500020936B379091663780916A37809366371D
:100E600090936A37809165378093871B40916937EB
:100E700040936537809369373F5F30936C3731110A
:100E80000DC02F5F20936B37211108C09F5F909397
:100E90006A37911103C08F5F809369378091613702
:100EA000909162379093851B8093841B20916337C8
:100EB0003091643730936237209361379093643771
:100EC000809363378091593790915A37A0915B375F
:100ED000B0915C3780935D3790935E37A0935F3716
:100EE000B09360378091E43C9091E53CA091E63C62
:100EF000B091E73C8093593790935A37A0935B3772
:100F0000B0935C379DC3973089F08F5F8430C1F018
:100F100060E2869F90011124F901EC5AF34C918D07
:100F20009111F1CF8093871BEF010CC0209721F026
:100F3000428D9A8D941748F7E901CC5AD34CE5CFEE
:100F40008093871B209709F4B9C3D093533CC09377
:100F5000523C83E08A8F888F1E8A84E08F8B1B8EA1
:100F600080916337909164379D838C838091613742
:100F7000909162379F838E838091593790915A3731
:100F8000A0915B37B0915C3788839983AA83BB8338
:100F900081E0898F80918A1B8C8780918B1B8D8744
:100FA00080918C1B8E8780918D1B8F8781E090E0D4
:100FB000998B888B809168378B87809167378A8778
:100FC00080916637898780916537888781E090E0D6
:100FD0000E94A98B80916D37982F907F913508F4EE
:100FE00042C082958F7090E00597880F991F880FF7
:100FF000991F2091861BEF2DF0E0E817F9077CF58B
:10100000E35BF84C20A5211103C01092861B29C078
:10101000213011F4F394EFCF2230E1F431A53430D4
:10102000C9F42093861BF092871B82A590E0982F2D
:10103000882723A5822B9093851B8093841B893D51
:1010400074E0970710F088ED94E09B8B8A8B9D8B62
:101050008C8B09C031A5332311F0F30ECCCF209334
:10106000861BF092871B80E180936E3780916E37EC
:10107000826080936E3782E08093753784E080933E
:1010800076378093773788ED809378378CE290E0DD
:10109000909346378093453780E67FC2D093533C88
:1010A000C093523C10924D3C80916E37982F9470B3
:1010B000F92E82FF03C0198E80E218C290916D371D
:1010C00092959F70990F990F9093871B091B110997
:1010D000045111091093463700934537922F9F70A2
:1010E000923029F4982F9F73923139F41FC09130B8
:1010F00021F4982F9F739230C9F0012B19F4982F87
:101100009370A1F020916537988529133CC22091F6
:1011100066379985291337C2209167379A85291335
:1011200032C2209168379B8529132DC284FF49C0A4
:10113000688979896115710509F443C0CE010C965F
:101140000E94B6823091693780914937381339C08F
:1011500020916A3780914A37281333C090916B37BA
:1011600080914B3798132DC080916C3740914C374C
:10117000841327C03C872D879E878F878B8D811195
:1011800019C09E89888D2A8D821B292F2695269528
:101190002695821B980F9E8B87FD81952F89322F74
:1011A00036953695231B820F8F8B9695969596953F
:1011B000890F888F81E080934D3C888D8A8F198AB2
:1011C000188A298DE22FEF708E2F90E0FC01319765
:1011D000E830F10508F072C2E057FF4F0C944F94CD
:1011E00080914D3C80FF14C083E0898F80E4809320
:1011F0004D3C198A188A809145379091463700975F
:1012000009F406C122E420934D3C0E94A98B00C141
:1012100080916E378F73823009F050C224CF809155
:101220004D3C80FF6BC080916E378F73823109F027
:1012300065C080916D37982F907F913508F442C03A
:1012400082958F7090E00597880F991F880F991FDE
:101250002091861BEF2DF0E0E817F9077CF5E35BA2
:10126000F84C20A5211103C01092861B29C0213003
:1012700011F4F394EFCF2230E1F431A53430C9F406
:101280002093861BF092871B82A590E0982F8827D9
:1012900023A5822B9093851B8093841B893D24E09A
:1012A000920710F088ED94E09B8B8A8B9D8B8C8B42
:1012B00009C031A5332311F0F30ECCCF2093861B48
:1012C000F092871B83E0898F8091653788878091B2
:1012D00066378987809167378A87809168378B87DF
:1012E00081E090E00E94A98B82E480934D3C198AB2
:1012F000188A10924637109245378AC080E2809350
:101300004D3C0E94DC7EE091523CF091533C118EAA
:1013100083CD80916E3780FF28C024FD26C0888948
:101320009989892B09F0CAC1809145379091463738
:1013300001960E94A98B80914D3C982F90619093CB
:101340004D3C2091453730914637232B19F082616F
:1013500080934D3C0E94DC7E81E090E0998B888BED
:1013600088E0898F1B8E81E10FC185FF1DC08091B0
:10137000733790E0982F882730917437832B4091F2
:10138000503C5091513C480F591F5093513C409351
:10139000503C4091453750914637BA01681B790B54
:1013A00070934637609345374091453750914637A3
:1013B0004115510551F024FD08C090914D3C9260BB
:1013C00090934D3CCA010E94A98B80916F3790E0A9
:1013D000982F882720917037820F911D9093851B3D
:1013E0008093841B2C893D892817390710F0892B9D
:1013F00021F43093851B2093841B8091841B909152
:10140000851B9B8B8A8B80914D3C837009F456C160
:101410001092E93C1092E83C0E94DC7E80914D3CA9
:1014200085FF07C01092E93C1092E83C198E84E1D8
:10143000ABC084FF0AC01092E93C1092E83C81E006
:1014400090E0998B888B84E08CCF2091E83C3091A0
:10145000E93C21153105E1F080FF02C0198A188AA4
:1014600088899989009781F48A899B8982179307D3
:1014700020F49093E93C8093E83C8091E83C909183
:10148000E93C998B888B04C09093E93C8093E83CBD
:101490001B8E80914737909148379093513C8093B1
:1014A000503C8091E83C9091E93C892B59F0888927
:1014B0009989009739F088969093463780934537FD
:1014C00088E10BC080914D3C81FFF8C088E290E03C
:1014D000909346378093453780E180936E375CC0A8
:1014E00080914D3C80FFEAC0198E80E180934D3C95
:1014F0000E94DC7EE3C0809145379091463700978B
:1015000011F00E94A98B90916E3780914D3C90FF15
:101510000BC080FF06C087E0898F1A8E198A188A4F
:1015200019C086E0898F16C080FF1EC085E0898FB4
:10153000198A188AC3C08091453790914637009721
:1015400011F00E94A98B80916E3780FF0DC087E05B
:10155000898F1A8E81E090E00E94A98B80E18093B0
:101560004D3C0E94DC7E0FC08091453790914637FC
:10157000892B49F4A3C080914D3C80FF9FC087E038
:10158000898F1A8E9BC080E180936E3788E290E04D
:10159000909346378093453780E580936D378885F3
:1015A00080936937898580936A378A8580936B3702
:1015B0008B8580936C378C85809365378D85809380
:1015C00066378E85809367378F858093683786E08E
:1015D000809356378C819D819093623780936137D9
:1015E0008E819F8190936437809363378091E43C30
:1015F0009091E53CA091E63CB091E73C809359374F
:1016000090935A37A0935B37B0935C378881998168
:10161000AA81BB8180935D3790935E37A0935F373B
:10162000B0936037898D84FF05C010927037109297
:101630006F3706C084E080936F3788ED80937037F2
:1016400080E4809355378091453790914637909349
:101650004F3780935037109274371092733710922F
:101660007237109271370E940783809590959093FE
:1016700072378093713785E480934D3710924E37DF
:10168000109254371092533780918E1B90918F1B7C
:10169000019690938F1B80938E1B9093513780936C
:1016A000523710925837109257370E94F682809521
:1016B0009095909358378093573704C010924637CF
:1016C0001092453710924D3CDF91CF911F910F91B1
:1016D000FF90EF90DF90CF90BF90AF900895982744
:1016E0008927982708950E9458940895FC018091B5
:1016F0004737909148372DE43CE3281B390BAB0169
:10170000261737070CF4A9011416150654F4509344
:10171000E93C4093E83CE817F90719F0BF010C9445
:101720002D9A089580E880936100109261000E94D4
:10173000496A0E948B5B0E942E6E8091F8349091D2
:10174000F9340097B1F301979093F9348093F8340A
:10175000F0CF2091523C3091533CBC01C901089616
:101760000E94B682E091523CF091533CA9E4B7E369
:101770008C91808711968C911197818712968C910C
:101780001297828713968C91838708952F923F92A8
:101790004F925F926F927F928F929F92AF92BF9281
:1017A000CF92DF92EF92FF920F931F93CF93DF932D
:1017B000CDB7DEB763970FB6F894DEBF0FBECDBFCF
:1017C0006C014B012A01FC0117821682838181FF83
:1017D00043C3AE014F5F5F4F3A01F6019381F401BD
:1017E00093FD859193FF81914F01882309F430C3C4
:1017F000853239F493FD859193FF81914F018532B4
:1018000039F4B60190E00E94B09A52012501E5CF6B
:1018100010E0F12C20E02032A0F48B3269F030F49B
:10182000803259F0833269F420612CC08D3239F056
:10183000803339F4216026C02260246023C02860F0
:1018400021C027FD27C030ED380F3A3078F426FF4D
:1018500006C0FAE01F9F300D1124132F13C04AE079
:10186000F49E300D1124F32E20620CC08E3221F430
:1018700026FDEEC2206406C08C3611F4206802C03A
:10188000883641F4F40193FD859193FF81914F01D6
:101890008111C1CF9BEB980F933018F42061805ECB
:1018A00006C09BE9980F933008F071C12F7E26FF88
:1018B00016E02F73322E853619F42064322E08C0BC
:1018C000863621F4F22FF0683F2E02C0111111501C
:1018D00037FE07C01C3350F4EE24E394E10E27E0FA
:1018E0000BC0183038F027E017E005C027E04CE3C4
:1018F000E42E02C0212FE12C520144E0A40EB11CC1
:10190000F20160817181828193810E2DA3010E9479
:1019100034992C01098100FF02C003FF07C031FC8C
:1019200008C032FE09C030E2232E07C02DE2222E6D
:1019300004C09BE2292E01C0212C802F8C7019F04D
:10194000211068C2A8C237FE0FC0E40C04FF04C017
:101950008A81813309F4EA941E1474F5F8E0FE15C7
:1019600078F588E0E82E2CC036FC2AC0812F90E064
:10197000841595059CF02CEF42162FEF520674F05B
:10198000432D4068342E0AC0E2E0F0E0EC0FFD1F6A
:10199000E10FF11D8081803319F411501111F4CF42
:1019A00037FE0EC0EE24E394E10E812F90E048163E
:1019B00059062CF4141904C0EE24E39401C010E07D
:1019C00037FE06C01414150434F4C201019605C094
:1019D00085E090E002C081E090E0211001961123A3
:1019E00031F0212F30E02F5F3F4F820F931F2F2DBB
:1019F00030E08217930714F4F81A01C0F12C832DFC
:101A0000897049F4FF2039F0B60180E290E00E942D
:101A1000B09AFA94F7CF222029F0B601822D90E0F7
:101A20000E94B09A33FC09C0FF2039F0B60180E370
:101A300090E00E94B09AFA94F7CF37FE5AC0942DE6
:101A4000852D57FE02C090E080E0292E382E20E040
:101A500030E0A2014E1951095D874C87A20142195D
:101A600053095F874E87612F70E044275527461B37
:101A7000570B598B488B5FEF2516350649F4B60195
:101A80008EE290E02A8B3B8B0E94B09A3B892A8998
:101A9000421453046CF04C855D854215530544F4A3
:101AA000EE85FF85E20FF31FE60DF71D818101C072
:101AB00080E351E0251A31082F5F3F4F488959894B
:101AC000241635064CF0B60190E02A8B3B8B0E9421
:101AD000B09A2A893B89CFCF2414350439F49A81EE
:101AE000963318F4953311F404FF81E3B60190E0C6
:101AF0004BC08A81813309F00F7EB60190E00E94CD
:101B0000B09A111105C034FC18C085E690E017C0EA
:101B1000B6018EE290E00E94B09A82E0EE24E39457
:101B2000E80EF301E80FF11D8081B60190E00E94FC
:101B3000B09A11508E2D91F7E6CF85E490E0B60172
:101B40000E94B09A57FC05C04114510439F404FFB7
:101B500005C05194419451088DE201C08BE2B60159
:101B600090E00E94B09A80E39AE0491651042CF06C
:101B70008F5F5AE0451A5108F7CFB60190E00E94F6
:101B8000B09AB601C201C0960E94B09A57C183367E
:101B900031F0833779F0833509F058C021C0520104
:101BA000E2E0AE0EB11CF2018081898301E010E019
:101BB000230114C05201F2E0AF0EB11CF2014080CB
:101BC000518026FF03C0612F70E002C06FEF7FEFEE
:101BD000C2012A8B0E945C9A8C012A892F7715C03A
:101BE0005201F2E0AF0EB11CF2014080518026FF9D
:101BF00003C0612F70E002C06FEF7FEFC2012A8B3C
:101C00000E941E9A8C012A892068322E23FD1AC058
